:1000000000400020FD8600003D8700003F87000083
:1000100000000000000000000000000000000000E0
:100020000000000000000000000000004187000008
:10003000000000000000000043870000458700002A
:1000400047870000AD5F0000A98A000047870000D5
:100050004787000000000000478700004787000036
:10006000E53C00007D8E00004787000047870000C8
:100070004787000047870000478700004787000048
:10008000478700002D8B000047870000478700004E
:100090004787000047870000478700004787000028
:1000A00047870000478700000000000000000000B4
:1000B0000000000000000000000000000000000040
:1000C00010B5064C2378002B07D1054B002B02D02E
:1000D000044800E000BF0123237010BD700200201F
:1000E000000000006CFD0000044B10B5002B03D095
:1000F0000349044800E000BF10BDC04600000000F6
:10010000740200206CFD0000164B002B00D1144B34
:100110009D46402292029A1A924600218B460F4633
:100120001348144A121A0CF0E7FC0F4B002B00D0B6
:1001300098470E4B002B00D0984700200021040068
:100140000D000D48002802D00C4800E000BF0CF064
:1001500093FC2000290008F0F9FC0CF067FCC04675
:100160000000080000400020000000000000000027
:1001700070020020D42F00200000000000000000CA
:1001800002000120104011D1042A0ED91368180969
:1001900080B2002809D001388000031D11180979A8
:1001A000002902D001309842F8D170470020FCE7C6
:1001B0000378002B03D05AB2002A01DB01307047CC
:1001C0003F229343C03B59424B41C01803789343AD
:1001D000802BF4D10130F9E710B500240378002B0F
:1001E00001D1200010BDFFF7E3FF0134F6E770B541
:1001F000002204000D00411C092004F09BF8002897
:1002000006D001236200134343600023A34200DBB6
:1002100070BD9A00A958821891600133F6E770B555
:10022000012803DC1C2001F0B7FA70BD01230D6822
:1002300011201D42F7D04868184206D1042804D97D
:100240000F2302681340042B01D00E20EBE703F0CC
:10025000CFFE6D100400002D03DDFFF7BDFFA842A7
:1002600006DA1220DFE72000FFF7A2FF0400013DBD
:10027000012DF8D120787F2809DDDF280BDCF82359
:100280003F22DB00800118406378134018430123AC
:1002900040001843C9E7EF280BDCFC226378120109
:1002A0009B0113403F220007000C0343A07810403D
:1002B000ECE7F72812DCFC22637892021B03134060
:1002C000E0228004520310403F221843E378134099
:1002D000FC220343A07812018001E8E7012040429C
:1002E000D5E7F8B54D680F00EB0706D4042D04D907
:1002F0000F232E683340092B03D00B2001F04CFA5A
:10030000F8BD6B683609B6B25C10731EA3420FD8F5
:10031000032120000AF0ACFA6421642803DC010008
:10032000032800DA03212800891904F035F80500B4
:100330002B6800201B099BB2013B9C42E0D23A682B
:10034000A31C9B005A510123013464001C436C60C0
:10035000D6E7F0B585B0012803DC1C2001F01CFABB
:1003600012E001274B683A000093022806D08B6800
:100370003B4203D05F10002F00DC17000125009BDB
:100380002B4203D00120404205B0F0BD009B042B5E
:10039000F8D91B680C680F261900314004292DD1AB
:1003A0002C4205D1042C03D923681E40042E01D011
:1003B0000E20D3E70098FFF7E3FEB842E2DB009897
:1003C00003F016FE0600200003F012FE0378010081
:1003D000002BD7D0781E30180CF044FF041ED1D06B
:1003E0003378002B01D0A64202D36800012521E01A
:1003F0003000FFF7DDFE01350600F1E709293ED1A7
:10040000009B5B685B1001939F42BBDC2C422ED1AA
:10041000042C2CD923683340042B28D1200003F06E
:10042000E7FD039602907E1C009AB300D0588442E8
:1004300002D178002843A7E728420ED104280CD91E
:100440000368039A1340042B07D103F0D1FD010088
:1004500002980CF0D1FE0028EBD0019B37009E42A1
:10046000E1DD8FE71F00019B9F4200DD8AE77B1CD7
:1004700000999A008A58A242F4D17800B6E703297D
:1004800000D07FE71A0992B25B0F92000B40D31A9B
:1004900001939F4200DD75E72C4229D1042C27D916
:1004A00022681640032E19D1100980B2520F800025
:1004B0003240251D801A019B2E181B1A0193009BA8
:1004C000781E0433019A904200DD5BE72A00191878
:1004D000B2420FD316D10130400087E7042E07D176
:1004E000200003F085FD05002000FFF749FEE2E74C
:1004F0000F2033E70C78A4461478A44502D10131CB
:100500000132E5E70130DDE7F0B50D0085B00128E7
:1005100004DC1C2001F040F905B0F0BD012708689B
:10052000384206D1042804D90F2102680A40042A5F
:1005300001D00E20EEE76A681740FAD1042AF8D9F4
:1005400013680B40042BF4D103F052FD04006868DB
:1005500003F04EFD02900CF059FE039000280FD1DD
:100560002000FFF739FE0190019B0122591C092050
:1005700003F0E0FE364E3060002815D10020CBE7B6
:10058000029920000CF06EFE001B43424341200004
:100590000193019B5E1C0028E6D0039B0299C018C2
:1005A0000CF060FE0196F4E70122019B5B0013430F
:1005B0004360039B002B18D12000FFF7F9FD019B3E
:1005C0000500BB4201DC3068A6E7291B200003F0D0
:1005D0002FFF0028D2D0BB1C32689B009850280007
:1005E000FFF7E6FD01372C00E9E7019B012B02D163
:1005F0002B68836090E7029920000CF033FE012500
:100600000700019B002F13D0AB42DCDB391B20001D
:1006100003F00EFF0028B1D032680135AB009850CE
:10062000039B0299FC1820000CF01CFE0700E8E771
:10063000AB42C8DB20000CF0E9FD0100200003F014
:10064000F7FE00289AD001353368AD00E850BAE7CC
:10065000E40F002010B503F0AFFC43000120184365
:1006600010BD0000C30711D404280FD90F2302685E
:100670001340032B0AD119400133591AC0234907EB
:10068000DB051940024B1A40114301607047C04618
:10069000FFFFFF9F70B5002805DC1C2001F07CF8EF
:1006A0000500280070BD01220C68144201D10D2004
:1006B000F4E701281CD04B681342F8D05B101320DC
:1006C000FF2BEBD81A0619040A431A431B021343E3
:1006D0006410E243D2171440E11C89101A00032071
:1006E00003F028FE051EDCD02100FFF7BBFFD8E792
:1006F0000023EDE7F7B507000E001C20012F06DDF3
:100700004C68012322001A40009203D10D2001F011
:1007100043F853E0022F02D08A681A42F6D0012330
:1007200035681D4200D0A9E0042D00D8A6E01C4188
:10073000002C00DC1C000F2029680840092828D163
:100740006B685B100093022F05D0B368009A5B10B2
:100750009A4200DD0093009B01221D1B0135EB43F3
:10076000DB171D40691C092003F0E4FD071E09D0BA
:1007700001236D001D430300326808334560009972
:10078000A14201DA3800FEBD0134A100515802C374
:10079000F5E7042845D1280003F02AFCFFF71CFDEB
:1007A0000190022F04D0B3685B10984200DD0193E2
:1007B000019BA34204DA002003F02EFE0700E1E7CC
:1007C000280003F015FC0700009BA34221DB280052
:1007D000009703F00DFC05003800FFF7E9FC019BD2
:1007E00001340700A342F7DA009BC41A200003F08B
:1007F00013FE071EC6D003F0FBFB0190306803F028
:10080000F7FB2200009B591B411801980CF058F986
:10081000B8E73800FFF7CCFC009B070001330093DA
:10082000D2E703282AD10B099BB2490F9B00014054
:10083000591A022F04D0B2685210914200DD110003
:10084000A14205DA00220320110003F073FDB5E791
:1008500003200E1B331DD9170140C918891000222F
:1008600003F068FD071E00D18CE701363100033428
:10087000FFF7F8FE381D29193200C7E7212046E7A7
:10088000F7B5002804DC1C2000F086FF040014E00B
:100890000D6801272E003E4011D03D41FF2D01D9AA
:1008A0001320F1E700223900032003F043FD041E6A
:1008B00003D03900FFF7D6FE25712000FEBD042DC0
:1008C000EED90F232A681340042B1BD12800FFF711
:1008D00057FCC31C07000320D9170140C918891011
:1008E000320003F027FD041EE7D03900FFF7BAFEFF
:1008F000280003F07DFB231D01003A0018000CF0D6
:10090000DFF8DAE7092B1FD103206B6832005B1098
:1009100001930333D9170140C918891003F00AFD68
:10092000041ECAD00199FFF79DFE019B9E42C4DAC6
:10093000B300EB189B683B4204D05B10FF2BAFD891
:10094000A21913710136F0E7032BA9D12C00B4E7EB
:1009500010B57F2902DC0170013010BD1A4B99429D
:100960000CDC40238A115B42134303703F230B408E
:1009700080214942194341700230EEE7134B9942FE
:1009800010DC20230A135B4213433F2480220370B0
:100990008B1152422340214013430A43437082701B
:1009A0000330DAE70A4B9942D7DCF0230370603B4F
:1009B0004370113B8A11FF3B1A4382703F22114062
:1009C0001943C1700430C8E7FF070000FFFF0000B3
:1009D000FF0F010010B50124044002D04410200094
:1009E00010BD042810D90F2302681340042B07D12F
:1009F00003F0FEFA21000A220CF0D0FC0400EEE71E
:100A0000032B01D10430F5E70D2000F0C5FEE6E729
:100A1000F0B50E0085B0002803DC1C2000F0BCFE01
:100A200017E00F6801243D00254006D1042F1ED990
:100A30000F233A681340042B0DD13800FFF7CAFF8B
:100A400002AC01002000FFF783FF011B200003F030
:100A5000EFFC040032E0092B09D17B685B100193A5
:100A6000019B9C4205DD00F09DFE002819D02A2044
:100A7000D4E70134A300F858FFF7ACFF01237F2827
:100A80000DDD154ADB18904209DD144A013390420E
:100A900005DD0021124AC30F82424B419B00ED1835
:100AA000DEE7280003F0B8FC041E07D0376803F027
:100AB0009FFA01250600019B9D4202DD200005B042
:100AC000F0BD0135AB00F858FFF784FF010030009E
:100AD000FFF73EFF0600EEE7FF070000FFFF000004
:100AE000FF0F0100F7B5030001900E001C20012B41
:100AF00011DD0868FFF76EFF07007068FFF76AFFF7
:100B0000019B05000124022B08D0B068FFF762FFAB
:100B1000041E03DC292000F03FFEFEBDAF421CDCBA
:100B2000E81B210009F0A4FE451C691C00220920D5
:100B300003F000FC0028F0D001226B001343436057
:100B40009440002379009D42E7DD17009E000F438B
:100B50008619B76001330919F5E7781B210009F000
:100B600087FE6442451CE0E710B504000120084000
:100B700010D104290DD90F230A681340042B08D182
:100B8000080003F035FA010020000CF035FB434269
:100B9000584110BD0020FCE7F7B50E00012803DC2A
:100BA0001C2000F0F9FDFEBD4D68EB0706D4042DB6
:100BB00004D90F222B681A40092A01D00B20F0E734
:100BC0006A681B099BB25410A34200D85C1E01271F
:100BD00031680F404810002F35D12648FFF7C4FF79
:100BE00001230190002813D131682348FFF7BCFF8F
:100BF000002811D0002C0DD00122631C013C944030
:100C00009B005A5114436C6004E00137BA00AB50AA
:100C1000BC42FADA0020C6E701233068184223D12B
:100C2000042821D902680E331340042B1CD1FFF78E
:100C3000D1FE002807D131681048FFF795FF002842
:100C400012D01220ADE70028FBDD8442F9DB8300DF
:100C5000EB180433844209DC0123621C013C9C40F4
:100C6000920053511C43CEE711209AE75A68013095
:100C70001A60EEE7A3E10000A7E100004DF40000D8
:100C8000002310B50C000B70C30705D50D494210A9
:100C900020000CF075FA08E00B49002802D0042867
:100CA00004D10A4920000CF08BFA10BD0428FCD9AD
:100CB0000F2302681340042BF7D103F099F904497C
:100CC0000200E5E724EE0000ACE10000B2E1000024
:100CD000B7E10000F0B593B0060002911C20012E90
:100CE0001DDD029B01251B681C002C4000D0ADE0DF
:100CF000042B00D8E6E01A680F231A40092A4AD1CB
:100D00000394039A029992008A5817002F4005D144
:100D1000042A03D910681840092806D0222000F0C0
:100D20003BFD0190019813B0F0BD52685210A41819
:100D3000039A013203929642E3D1611C012203F02F
:100D4000F9FA0190002802D100230193EAE7019B00
:100D50006400190025435D600831029ABB00D05839
:100D600002684368120992B25B109A4200D8531E7F
:100D70000022934209DCDA43D21713409B00C918C2
:100D8000039B01379F42E8DBCCE794000519AD686F
:100D900001320D51EDE72700032A59D10193029A40
:100DA000BB00D3582B42B9D1042BB7D9186801998D
:100DB0000140032939D1020992B2430F92000B403E
:100DC000D31A1C190137BE42E9D10320E31CD917FD
:100DD0000140C9188910002203F0ACFA01900028E4
:100DE000B2D000252100FFF73DFC019B1E1D029A99
:100DF000AB00D45801231C421FD1042C1DD90F2154
:100E000023681940032918D1180980B25B0F8000AC
:100E10000B40C01A0023834213DBC343DB17184087
:100E200001353618BD42E2DB7CE7042900D075E7C6
:100E30001800FFF7A5F92418C4E72000FFF7A0F970
:100E4000E8E7E2181279F2540133E4E700273C00A6
:100E50000F25029ABB00D3580122134234D1042B30
:100E600032D9186801002940042935D11800FFF74C
:100E700087F924180137BE42EBD1200003F0CCFAE9
:100E80000190002800D15FE7029FB600BB19041D46
:100E9000029301233D681D4229D1042D27D90F2635
:100EA0002B681E40042E37D12800FFF769F9060091
:100EB000280003F09DF80100200032000BF000FE36
:100EC000A41922E02700C3E7180005A9FFF7D8FE00
:100ED00005A80CF09BF9CCE7032900D01EE7020916
:100EE00092B2430F92000B40D31A1C19C2E705A916
:100EF0002800FFF7C5FE05A80CF088F905A9050034
:100F0000020020000BF0DCFD6419029B0437BB4299
:100F1000BFD10023237005E7032EF6D11A0992B240
:100F20005B0F92001E40961B291DC5E7F0B50D0012
:100F300097B0002806DC1C2000F02EFC07003800CB
:100F400017B0F0BD0C68012123000B40009306D1BF
:100F5000042C04D922680F331A40092A01D00B202F
:100F6000EAE7626852100392002A03DC009803F05B
:100F700053FAE3E7504A019201280BD0686808420F
:100F800008D1042806D902681340042B02D103F0CB
:100F90002FF8019001980CF039F906000F27039BF8
:100FA0000834013B05935E43039B02909B00E318CA
:100FB000049301232068184273D1042871D9016871
:100FC0000B003B409C46042B03D1FFF7D9F8861950
:100FD00009E0032B6CD162460B099BB2490F9B00C1
:100FE00011405A1A9619049B0434A342E1D13000EF
:100FF00003F012FA071EA2D02B680793029B002B66
:1010000003D0686802F0F4FF0190380002F0F0FFAE
:101010000400009B079A9B00D3189E68300002F0E2
:10102000E7FF0123334005000693002B01D1042E76
:1010300004D809A93000FFF723FE09AD28000CF001
:10104000E5F8069B0490002B0ED1042E0CD90F213D
:1010500033681940032907D11A0992B25B0F920035
:101060000B40D31A351D04932000049A29000BF07D
:1010700027FD049BE418029B002B0AD0059B009AD5
:10108000934206DD2000029A01990BF019FD029BA4
:10109000E418009B01330093009A039B9342B8D15C
:1010A0004DE709A9FFF7ECFD09A80CF0AFF88EE7B2
:1010B00002F09EFFF9E7C046F8E6000010B50122F5
:1010C000002400280BDD0B681A40141E03D05C10AE
:1010D000E343DB171C400122904200D04A68611CA8
:1010E000092003F027F9002803D0012364001C43E2
:1010F000446010BD0A6870B510000125284034D145
:10110000042A32D90F24136849681C40092C17D1CE
:1011100054681B099BB22C41A34200D85C1E844238
:1011200005DC02200133984206DB00200FE0850039
:101130005519A9600130F2E7840011510130F2E73E
:10114000032C12D1294203D1132000F025FB70BDDE
:101150004910FF29F8D81B099BB204329B00D31811
:101160009342E2D911700132FAE70B2000F014FB30
:10117000DBE700000123F7B500254E680C00334083
:101180000193AB420ED11D00042E0BD90F22336800
:101190001A40092A26D172681B099BB25510AB422E
:1011A00000D85D1E27687C10FB0746D439003D48F7
:1011B000FFF7DAFC002826D00BF07EFF290009F0AB
:1011C0003DFC4C1C019B002B00D069E0042E67D92C
:1011D00032680F331340092B3BD10134A400A459CA
:1011E0002000FEBD042A04D13000FEF7C9FF05002F
:1011F000D8E7019D032AD5D11D09ADB25B0FAD0023
:101200001340ED1ACEE739002748FFF7ADFC002860
:101210001DD1042F16D90F233A681340042B11D186
:101220003800FFF7D7FB041E07D139001F48FFF72E
:101230009BFC002806D0122005E0002CFBDDA54217
:10124000C0DAF8E7112000F0A7FA0400C8E72C0084
:10125000B8E7042B1CD1300002F0CAFE0500012CB7
:101260000EDCFEF7A5FF461B300003F0D5F8041E88
:10127000B6D002F0BDFE320029000BF021FCAFE732
:101280002B78013C002BD6D02800FEF791FFE5E734
:10129000032B05D13419E37801245B001C439FE73D
:1012A0000B20D0E79CE10000A7E100004DF4000016
:1012B000F7B54D680E002A0001210A402FD1042DF8
:1012C0002DD90F242B68B7681C40092C14D16968EC
:1012D0001B099BB24C100192A34200D85C1E3168DE
:1012E0003448FFF741FC00282DD00F232A68134013
:1012F000092B1DD1012317E0032C10D10F4203D17C
:10130000132000F049FAFEBD7A100192FF2AF7D8A7
:101310001A0992B25B0F92001C40141BDFE70B20EE
:10132000EFE701339A00AF509C42FADA0020EAE777
:10133000032BFBD12B0001335A1BA242F6DC6A4679
:101340001279DA70F7E736687010F30719D43100B4
:101350001948FFF709FC002822D1042E1ED90F23BB
:1013600032681340042B19D13000FFF733FB0028FB
:1013700007D131001148FFF7F7FB00280ED01220EB
:10138000BFE70028FBDD8442F9DB0F232A68134006
:10139000092B07D1013080004751C7E71120B0E782
:1013A0002000F2E7032BC1D16B461B792D18EB709F
:1013B000BCE7C046A3E10000A7E100004DF4000037
:1013C00070B501240868204207D1042805D90F25EB
:1013D00001680D40092D02D14468200070BD032D25
:1013E00008D10A0992B24B0F92002B40D31A5B002E
:1013F0001C43F2E7042DF0D102F0FAFDFEF7ECFEFB
:1014000040000443E9E7000010B5034A0E210348F9
:1014100004F0CAFE10BDC0462CE1000024E100002B
:1014200000207047042070470120704710B500204D
:1014300002F0F2FF10BD002070470020704700202E
:101440007047002070470020704700207047002040
:1014500070470020704700207047000010B5034A15
:101460000D21034804F0A0FE10BDC04644E2000078
:10147000ACE2000070470378002B03D05AB2002A78
:1014800001DB013070473F229343C03B59424B413F
:10149000C01803789343802BF4D10130F9E70000A2
:1014A000F8B50127060014000800394227D10429A5
:1014B0003FD90F230A681A40042A3AD13C4213D17B
:1014C000042C11D922681340042B0DD102F090FD99
:1014D0000500200002F08CFD010028000BF08CFEBE
:1014E00000282EDB1FD127E0E30722D502F080FD84
:1014F0000A2200210BF052FF0500601010E0174097
:1015000015D1042A15D90F2312681340042B10D1CA
:1015100020004D1002F06CFD0A2239000BF03EFF56
:1015200085420EDB08DD002E09DC00200CE04D10AA
:10153000E3E70F22054B1A700136022EF5D804207E
:1015400002E0042076173040F8BDC046B00200200B
:10155000F8B5060000242B4BE500ED182B79032B82
:1015600009D00134FF2CF6D1300004F031FE041E06
:1015700046D1013C44E030000BF048FEE3B20200EB
:101580003100180004F0A4FE002839D12A685168FF
:101590008842E6D08300D3189B680130F02BF7D146
:1015A00001238000083012181A42DAD1042AD8D94F
:1015B0000F21136819400429D3D11B0998B20123C4
:1015C0000130800010181842CBD10428C9D90F224D
:1015D00003681340042BC4D102F00AFD0327050061
:1015E000092128000BF0FAFD0028BAD0013F451C64
:1015F000002FF5D1310028000BF034FE8542B0D128
:101600002000F8BDA825002010B50124044002D018
:101610004410200010BD042810D90F230268134085
:10162000042B07D102F0E4FC21000A220BF0B6FEE5
:101630000400EEE7032B01D10430F5E70D22014B46
:101640001A70E6E7B0020020012210B5024018D15E
:10165000042802D903681A0992B201230B4012D15F
:10166000042902D90B681B099BB20024934206D1BE
:1016700004309B000431C318984206D30124200093
:1016800010BD0022E9E70023EFE704780A78002C78
:1016900001D1002AF2D0013001319442ECD0002473
:1016A000EDE70000F7B50700009101933049314B99
:1016B000002A02D002220A70013A00261A601B6832
:1016C000CE54BE4200DBF7BD009AB300D058294B80
:1016D000274D1C68C8239B0065191C1B0123184259
:1016E00006D0254A4310210028000BF017FD09E021
:1016F000224A002802D004281BD1214A21002800B8
:101700000BF00CFD1A4C20000BF080FD194A019BD8
:101710001060002B0BD07B1EB34208DD194B9842A2
:1017200005D8431C1360202222540022E2540136C3
:10173000C7E7042819D90F2301680B40042B04D1F3
:1017400002F056FC104A0300CDE7092B03D1436891
:101750000E4A5B10C7E7032B08D10A0992B2490F62
:1017600092000B40D31A0A4ABDE70123094ABAE79F
:10177000B1020020D405002024EE0000ACE10000FE
:10178000B2E100001F03000053F4000024E5000054
:1017900033E500003EE50000014B18700020704763
:1017A000B0020020024B1878431E98417047C04693
:1017B000B0020020002310B51A00FFF773FF034B9F
:1017C0000348196805F0E9F9002010BDD405002090
:1017D000B102002070B502F0ABF9094C0100251DE3
:1017E0001F2228000BF02AFD28000BF00FFD042318
:1017F00004308008000118432060200070BDC046FE
:101800008C020020C368F0B59D00836889B05D1923
:101810000300183306930369069A9F00069B029003
:10182000DF19436901939B00D3180393D04B1B78B6
:10183000002B26D17F222B68CE491C1213409B001F
:101840005B58043501929F46029B587805F084F955
:101850000023029A137027E0C54B1B78002B10D190
:101860002B68019A1C121340C24A9B009B580435F6
:10187000E9E7069B3A1DD11ABD4BD82928DD1A226B
:101880001A70029BBA4C9B6821780193EA1A029B5A
:1018900092109B7812021A43029B587805F064F963
:1018A0000023029A23701370029B069A9B6801938F
:1018B000ED1A029BAD10DD60069BFE1A029BB6106E
:1018C0001E61039B9B1A029A9B10536109B0F0BDE5
:1018D00039001B7817000C60002BD2D12B68019ABD
:1018E0001C121340A34A9B009B580435ABE7069B90
:1018F0003A1DD11A9E4BD82902DD1A221A70C0E770
:1019000038001B7817002A68291D0260002B01D0BF
:101910000D00B6E76B68019A1C121340954A9B00B4
:101920009B5808358FE7069B3A1DD11A904BD82952
:1019300002DD1A221A70A4E73900A4001B782C19C2
:1019400017000C60002B9CD12B68019A1C121340CD
:10195000884A9B009B58043575E7069B3A1DD11AAF
:10196000834BD82902DD1A221A708AE73900170042
:10197000814AA400A2581B780A60002B00D080E79F
:101980002B68019A1C1213407A4A9B009B5804351D
:1019900059E7043F784B3A68A400E250744B1B7837
:1019A000002B00D06DE72B68019A1C121340714A7E
:1019B0009B009B58043546E76F4BA400E058FFF7A7
:1019C00023FE6B4B06001B78002B09D1043F3868BF
:1019D000FFF71AFE0123861976001E43664BE65078
:1019E000634B1B78002B00D04BE72B68019A1C122D
:1019F0001340604A9B009B58043524E7069B391D21
:101A0000CA1A5B4BD82A02DD1A221A7039E70698E7
:101A1000039C0122A04202D222000C3A1268380034
:101A20001B780F000260002B00D02AE72B68019A78
:101A30001C1213404F4A9B009B58043503E7069A3B
:101A40003B1D991A4A4AD82902DD1A23137018E758
:101A500006990398814218D202000C3A126847494D
:101A600052106418A41AA40022583A601F00404B78
:101A70001B78002B00D004E72B68019A1C1213403E
:101A80003C4A9B009B580435DDE61821117000226A
:101A9000EBE7069B039A934219D213000C3B1B6899
:101AA000364A5B10A418043FE41A3A68039BA4006A
:101AB000E2502F4B1B78002B00D0E2E62B68019AF6
:101AC0001C1213402B4A9B009B580435BBE618227E
:101AD000274B1A70EDE7069B039A934228D2274BB7
:101AE000043FE61814000C3C23685B10F31A9B00BB
:101AF0009858FFF789FD04903868FFF785FD246842
:101B0000049B6410341B1E18012376001E43039BA4
:101B1000A400E650164B1B78002B00D0B1E62B68D2
:101B2000019A1C121340134A9B009B5804358AE605
:101B300018220F4B1A70EDE7069B3A1DD11A0C4B79
:101B4000D82902DD1A221A709BE639001700039A81
:101B5000A400A2581B780A60002B00D091E62B68E5
:101B6000019A1C121340034A9B009B5804356AE6F5
:101B7000B002002024E30000A02D0020FDFFFF3F65
:101B8000043F039B3A68A400E250D64B1B78002B1D
:101B900000D076E62B68019A1C121340D24A9B00B3
:101BA0009B5804354FE6039BA4001C192368043F8F
:101BB00038685E10FFF728FD0123361876001E43B3
:101BC000C84B26601B78002B00D05AE62B68019A80
:101BD0001C121340C44A9B009B58043533E6069BF5
:101BE000A4003F1BBF4CBB420CD82378002B00D075
:101BF00047E62B68019A1C121340BB4A9B009B5876
:101C0000043520E6B94802F0E3F92378002B00D030
:101C100037E62B68019A1C121340B34A9B009B586D
:101C2000043510E6A300ED18002C00DA3CE6AD4BBD
:101C30001B78002B00D024E62B68019A1C1213405D
:101C4000A94A9B009B580435FDE5043F3B68042BE3
:101C500004D1A300ED18002C00DA25E6A14B1B7877
:101C6000002B00D00DE62B68019A1C1213409E4AEF
:101C70009B009B580435E6E5043F3B68042B04D0E9
:101C8000A300ED18002C00DA0EE6964B1B78002B13
:101C900000D0F6E52B68019A1C121340924A9B0073
:101CA0009B580435CFE501233E1F306818420AD007
:101CB00018410138002809DB01234000A400184323
:101CC0002D193060F0E5FFF79FFCF2E7854B1B789C
:101CD000002B01D03700D4E52B68019A1C12134069
:101CE000814A9B009B5837000435ACE5069E03995A
:101CF000891B3E008910049106990C36711AD82967
:101D000002DD1A231370BCE53900FF2764007F0051
:101D10003C40FE3FFF3F3C430C60029C1278A468AD
:101D200003942D1B029CAD10A4782D022543BD40C9
:101D30003D434D600125049C370064002C438C60BA
:101D4000644602998C701B588B60002A03D00833BC
:101D50001D00039695E51D00019A9B680C351C1229
:101D60001340614A9B009B5803966CE53B1F1C681F
:101D7000039A069B934232D10A20E30711D4042C24
:101D800018D90F2322681340042B16D1200002F02B
:101D90002FF90BF03BFAC8239B00984200D918009A
:101DA0000630643004F0DCFA00280FD1043D069BB5
:101DB000039379E50720042CF3D02000431E9841BB
:101DC000FA234042FF3318400730EAE7029B210024
:101DD000587804F0DBFE0023029A1370E7E7039BB8
:101DE000039A0C3B1B6802995B109B00D31A0C3BB7
:101DF0001C601F1D1300083B1B685A108A70D2B26A
:101E00003B49D2005B0055589B0A029A9B009560A3
:101E1000ED18039B069A043B1B685B109B00D318CC
:101E20000393304B1B78002B00D02AE52B68019AD6
:101E30001C1213402C4A9B009B58043503E53B1FA2
:101E40001868FFF7E1FBA40006003F1B1E2827DCF3
:101E500000280DDC234B1B78002B00D011E52B68EC
:101E6000019A1C121340204A9B009B580435EAE457
:101E700001F046FE033E361801F042FE1D4B801B6A
:101E80009842F9D8174B1B78002B00D0F9E42B6847
:101E9000019A1C121340144A9B009B580435D2E44B
:101EA0000123029A137001F02BFE029B0A38861957
:101EB0005E60F9E43B1F1868FFF7A6FBA40006006C
:101EC0003F1B002818DC074B1B78002B00D0D8E400
:101ED0002B68019A1C121340034A9B009B5804353F
:101EE000B1E4C046B002002024E3000050E5000049
:101EF000A82500203F420F00D64B984203DD1D224B
:101F0000D54B1A70BDE40123029A137001F0F8FD5D
:101F1000FA239B005E430A3E3018029B5860C3E4DC
:101F2000A300FF1A002320001A003900FFF7BAFBB4
:101F3000CA4ECB4C3168200002F07AFAC94B3168A6
:101F40001860200004F0D2FC3168200004F025FE67
:101F5000C14B1B78002B00D093E42B68019A1C1214
:101F60001340C14A9B009B5804356CE4BA4BA40053
:101F70001B783F1B002B00D083E42B68019A1C12B6
:101F80001340B94A9B009B5804355CE4029804F066
:101F90004BFAB14B1B78002B00D072E42B68019AEE
:101FA0001C121340B04A9B009B5804354BE43B1F66
:101FB0001B68002B58D13B0001260C3B18680640DB
:101FC0002FD046103A0001217300083A0B431360EA
:101FD000002E00DC95E0012173000B433A1F1360D3
:101FE0003B00083B1B680B419B1B04933B000C3BD5
:101FF000186808423BD0049BA4005B188B400B433D
:10200000039AA350944B1B78002B00D039E42B6823
:10201000019A1C121340944A9B009B580435FFF709
:1020200012FC04281BD90F2302681340092B02D18C
:1020300043685E10C6E7042B08D101F0D9FF03788E
:10204000002BBFD0FFF717FA0136F8E7032B06D1B4
:102050001609B6B2520FB6001340F61AB2E71922AB
:102060007D4B1A70FFF70DFC5B105E1EB0E7042875
:1020700042D90F2302681340092B05D1049BA40009
:1020800002339B001B58BBE7042B2BD1039BA400FE
:102090001B19079301F0ACFF0600049C0134012CCE
:1020A00010DC3000FFF7E7F9831B1800049302F0FF
:1020B000B3F9041E0ED001F09BFF049A31000AF020
:1020C000FFFC07E03178013C002906D112220C0008
:1020D000614B1A70079B1C6094E73000FFF7CBF947
:1020E0000600DCE7032B07D10122049BA400C018E3
:1020F00003795B00134383E71922574B1A70FFF7EC
:10210000C0FB04357EE7A300069AFB189B1AD82B68
:1021100008DD1A22504B1A70FFF7B3FB01221C0096
:102120003A600437631E002CF8DC4B4B1B78002B05
:1021300001D0FFF7A6FB2B68019A1C1213404A4AF4
:102140009B009B580435FFF77EFB069A3B1D9B1AAC
:10215000414ED82B03DD1A233370FFF792FB069B09
:10216000039AA40093422AD23B1F1868FFF74CFA47
:10217000011E21DD039B0C3B1A68521082421BDBBF
:102180009007801A394B4018C018039B8000C25832
:102190003B1B1A60304B3F1B1B780437002B01D0D0
:1021A000FFF76FFB2B68019A1C1213402E4A9B000D
:1021B0009B580435FFF747FB20233370EAE71823C9
:1021C000FBE7284BA4001A683B1B1F001A60224B38
:1021D00004371B78002B01D0FFF753FB2B68019AC3
:1021E0001C121340204A9B009B580435FFF72BFB21
:1021F0003A1F1368042B02D13A00A4002D19164B84
:102200001B78002B02D01700FFF73BFB2B680199CE
:102210001C120B4014499B005B5817000435FFF754
:1022200012FB043F3B68042B04D00023A4003B6056
:102230002D190437084B1B78002B01D0FFF721FB29
:102240002B68019A1C121340074A9B009B580435C7
:10225000FFF7F9FA80EE3600B0020020D405002026
:10226000B10200200800002024E30000FCFFFF3F33
:10227000A3009C46F81A002C17DC1C220026D34B26
:102280001A706346FF1AD14B06601B780437002B87
:1022900001D0FFF7F6FA2B68019A1C121340CC4AC2
:1022A0009B009B580435FFF7CEFA002103685B10B2
:1022B00001268A008258164003D10D22C34B1A70A2
:1022C000DFE75210934200DD130001318C42EFDC56
:1022D0005E0001231E43D4E7A3009C46F81A002C9D
:1022E00017DC1C220026B94B1A706346FF1AB74B45
:1022F00006601B780437002B01D0FFF7C2FA2B6869
:10230000019A1C121340B24A9B009B580435FFF7F8
:102310009AFA002103685B1001268A008258164051
:1023200003D10D22A94B1A70DFE75210934200DA55
:10233000130001318C42EFDC5E0001231E43D4E721
:102340003B000122083B1968A40011421DD03B1F2D
:102350001B68134219D0114113410022994200DA3F
:1023600004323B1B1A60994B3F1B1B780437002B30
:1023700001D0FFF786FA2B68019A1C121340944A89
:102380009B009B580435FFF75EFA02203B1F1A683A
:102390004042FFF785F83E1B3060E4E73B00012038
:1023A000083B1968A40001421ED03B1F1A68024274
:1023B0001AD001415010CB0FD217884253413A1B1B
:1023C0009B001360814B3F1B1B780437002B01D00F
:1023D000FFF757FA2B68019A1C1213407C4A9B00A6
:1023E0009B580435FFF72FFA01203B1F1A68404223
:1023F000FFF756F83E1B3060E4E73B00083B1868E7
:102400003B1F1968A600BE1B0423814202D004288A
:1024100002D80023336016E001231842F9D10F23BC
:1024200002681A40042AF4D1033A1142F1D1042976
:10243000EFD90A681340042BEBD1FFF705F9431ECF
:10244000984180003060614BA4001B783F1B04372B
:10245000002B01D0FFF715FA2B68019A1C121340CC
:102460005B4A9B009B580435FFF7EDF93B00083BA6
:1024700018683B1F1968A600BE1B0023814202D0CA
:10248000042802D80423336016E001231842F9D14E
:102490000F2302681A40042AF4D1033A1142F1D101
:1024A0000429EFD90A681340042BEBD1FFF7CCF8CD
:1024B0004342584180003060444BA4001B783F1BCE
:1024C0000437002B01D0FFF7DCF92B68019A1C12AE
:1024D00013403F4A9B009B580435FFF7B4F93B007B
:1024E0000122083B1968A40011421ED03B1F1B6843
:1024F00013421AD05B104A10D80FC9179A424141B3
:102500003B1B89001960314B3F1B1B780437002BA4
:1025100001D0FFF7B6F92B68019A1C1213402C4A20
:102520009B009B580435FFF78EF93B1F1A6801206A
:10253000FEF7B6FF3E1B3060E5E73B000122083B9B
:102540001968A40011421DD03B1F1B68134219D00B
:10255000114113410022994200DD04323B1B1A60F5
:102560001A4B3F1B1B780437002B01D0FFF789F96A
:102570002B68019A1C121340154A9B009B58043586
:10258000FFF761F93B1F1A680220FEF789FF3E1B27
:102590003060E5E73B1F1B68A400043B5A1E9341D3
:1025A0003A1B17009B001360084B04371B78002B65
:1025B00001D0FFF766F92B68019A1C121340044AF8
:1025C0009B009B580435FFF73EF9C046B00200203F
:1025D00024E300003B00083B1868FFF715F83B1F99
:1025E00006001868FFF710F80121A4003B1B1F002C
:1025F000321852000A431A60EA4B04371B78002B4A
:1026000001D0FFF73EF92B68019A1C121340E64AED
:102610009B009B580435FFF716F93B00083B1868F0
:10262000FEF7F2FF3B1F06001868FEF7EDFF0121E1
:10263000A4003B1B1F00321A52000A431A60D94BF8
:1026400004371B78002B01D0FFF71BF92B68019A88
:102650001C121340D44A9B009B580435FFF7F3F833
:102660003B00083B1868FEF7CFFF3B1F06001868C9
:10267000FEF7CAFF02000121A4003B1B1F007243AA
:1026800052000A431A60C74B04371B78002B01D055
:10269000FFF7F7F82B68019A1C121340C24A9B00FF
:1026A0009B580435FFF7CFF83B1F1868FEF7ACFFC7
:1026B000061E17D11F23BB4A1370A4003B1B1F002B
:1026C0001E60B84B04371B78002B01D0FFF7D9F8F8
:1026D0002B68019A1C121340B34A9B009B58043587
:1026E000FFF7B1F83B00083B1868FEF78DFF31009B
:1026F00008F0BEF8012346001E43DEE73B1F1868C2
:10270000FEF782FF061E17D11F23A64A1370A400EE
:102710003B1B1F001E60A34B04371B78002B01D00E
:10272000FFF7AFF82B68019A1C1213409E4A9B00DA
:102730009B580435FFF787F83B00083B1868FEF705
:1027400063FF310008F07AF901234E001E43DEE7F3
:102750003B1F1868FEF758FFC2178018504001222F
:10276000A4003B1B1F004000104318608D4B043732
:102770001B78002B01D0FFF784F82B68019A1C12FC
:102780001340894A9B009B580435FFF75CF8A3006F
:102790000793FB1A0493012C2CD11868FEF734FF21
:1027A00001230600C4179C43E418B44202DC330042
:1027B00026001C000134A41B0AF07EFC210008F056
:1027C0003DF901238E1976001E43049B1E60079B72
:1027D000FF1A744B04371B78002B01D0FFF751F818
:1027E0002B68019A1C1213406F4A9B009B580435BA
:1027F000FFF729F8022C0AD1049B1868FEF704FFA2
:10280000049B04005868FEF7FFFE0600CDE7642431
:102810000126CFE7A300FE1A31002000049301F047
:1028200055FF049B3060FF1A5E4B04371B78002B6A
:1028300001D0FFF726F82B68019A1C1213405A4A60
:102840009B009B580435FEF7FEFF3B00083B1868D1
:10285000FEF7DAFE3B1F06001868FEF7D5FE020001
:102860000121A4003B1B1F00324052000A431A60A2
:102870004C4B04371B78002B01D0FFF702F82B6874
:10288000019A1C121340484A9B009B580435FEF7DE
:10289000DAFF3B00083B1868FEF7B6FE06003B1F58
:1028A0001868FEF7B1FE32000121A4003B1B1F0097
:1028B000024352000A431A603A4B04371B78002B3C
:1028C00001D0FEF7DEFF2B68019A1C121340364A36
:1028D0009B009B580435FEF7B6FF3B00083B186889
:1028E000FEF792FE06003B1F1868FEF78DFE3200D1
:1028F0000121A4003B1B1F00424052000A431A6002
:10290000284B04371B78002B01D0FEF7BAFF2B6849
:10291000019A1C121340244A9B009B580435FEF771
:1029200092FF3B1F1868FEF76FFEC0430122A40010
:102930003B1B1F004000104318601A4B04371B78E4
:10294000002B01D0FEF79DFF2B68019A1C1213404B
:10295000154A9B009B580435FEF775FF3B00083B6A
:102960001868FEF751FE06003B1F1868FEF74CFE84
:10297000320082400121A4003B1B1F0052000A4389
:102980001A60084B04371B78002B01D0FEF779FF43
:102990002B68019A1C121340034A9B009B58043574
:1029A000FEF751FFB002002024E300003B00083B8B
:1029B0001868FEF729FE06003B1F1868FEF724FE84
:1029C000320002410121A4003B1B1F0052000A43B8
:1029D0001A60EA4B04371B78002B01D0FEF751FF39
:1029E0002B68019A1C121340E54A9B009B58043542
:1029F000FEF729FF3B000C3B1868FEF705FE3B0085
:102A0000083B06001868FEF7FFFDF1170200C31728
:102A1000300008F065F83B1F049005911868FEF738
:102A2000F3FD02000498059908F00EF80123A400B4
:102A30003E1B370040001843D04B30601B780437F2
:102A4000002B01D0FEF71DFF2B68019A1C121340CA
:102A5000CB4A9B009B580435FEF7F5FEA300FE1AF7
:102A6000310020000493FEF729FB049B3060FF1A1D
:102A7000C24B04371B78002B01D0FEF702FF2B68F6
:102A8000019A1C121340BE4A9B009B580435FEF766
:102A9000DAFEA300FF1A39002000FEF72BFBB74B2C
:102AA0001B78002B01D0FEF7ECFE2B68019A1C125C
:102AB0001340B34A9B009B580435FEF7C4FEA300A5
:102AC000FE1A310020000493FEF754FB049B306093
:102AD000FF1AAA4B04371B78002B01D0FEF7D1FE5A
:102AE0002B68019A1C121340A54A9B009B58043581
:102AF000FEF7A9FEA300FF1A39002000FEF7D8FB5D
:102B00009E4B1B78002B01D0FEF7BBFE2B68019A71
:102B10001C1213409A4A9B009B580435FEF793FE03
:102B2000A300FE1A310020000493FEF749FC049B29
:102B30003060FF1A914B04371B78002B01D0FEF751
:102B4000A0FE2B68019A1C1213408D4A9B009B58D3
:102B50000435FEF778FE3B1F186801F049FA3A0089
:102B60000121083A12680300A4000A4229D1042A6C
:102B70000CD910680F221040013808280FD807F030
:102B8000D9FD052026220E0E0E0E24007D491800C8
:102B90000AF032FB434258413B1B80001860774BE0
:102BA0003F1B1B780437002B01D0FEF76AFE2B6811
:102BB000019A1C121340724A9B009B580435FEF781
:102BC00042FE7149E3E77149E1E77149DFE7714985
:102BD000DDE7069B3E1DF31A684CD82B03DD1A2354
:102BE0002370FEF74EFE00F095FF01223B004000EF
:102BF0001043186023783700002B01D0FEF741FE08
:102C00002B68019A1C1213405D4A9B009B580435A7
:102C1000FEF719FE069B3E1DF31A584CD82B03DD18
:102C20001A232370FEF72DFE00F06AFF5A4A400077
:102C3000104001223B001043186023783700002B1E
:102C400001D0FEF71EFE2B68019A1C1213404C4A5D
:102C50009B009B580435FEF7F6FD069A3B1D9B1A18
:102C6000464CD82B03DD1A232370FEF70AFE00F032
:102C700051FF4A4B1A68831A904201D2484A9B1866
:102C800001213A005B000B43136023780437002BCB
:102C900001D0FEF7F6FD2B68019A1C121340384A4A
:102CA0009B009B580435FEF7CEFD00F033FF3B4BF5
:102CB000A4001860314B3F1B1B78002B01D0FEF79E
:102CC000E0FD2B68019A1C1213402D4A9B009B5873
:102CD0000435FEF7B8FD03F02FFBA300002810D148
:102CE000FF1A264B1B78002B01D0FEF7CAFD2B687C
:102CF000019A1C121340224A9B009B580435FEF790
:102D0000A2FD3E00FF1A012320001A003900FEF741
:102D1000C9FC244C2068643003F022FB002803D156
:102D2000043D3700FEF7C0FD029B21685A781E481B
:102D300003F045FF0123029A137000F0E1FE1B4BE4
:102D400022681B68063253431818FFF7E6F803F0B1
:102D5000F3FAA30000282BD1FF1A084B1B78002B95
:102D600001D0FEF78EFD2B68019A1C121340044A15
:102D70009B009B580435FEF766FDC046B00200205C
:102D800024E3000060E5000068E500006FE5000056
:102D900076E500007BE50000FEFFFF7FDC050020FC
:102DA00037894100D4050020B10200200400002032
:102DB0003E00FF1A2000012300223900FEF772FCBA
:102DC000F14C2068643003F0CBFA0028A8D0EF481B
:102DD00003F072FCAEE7A4003E1BFEF7FBFC3700DD
:102DE000EB4B30601B780437002B01D0FEF749FD18
:102DF0002B68019A1C121340E64A9B009B5804352D
:102E0000FEF721FDE24BA4001B783F1B002B01D0F5
:102E1000FEF737FD2B68019A1C121340DD4A9B0018
:102E20009B580435FEF70FFDA4003E1B300000F058
:102E3000AAFE3700D64B30601B780437002B01D038
:102E4000FEF71FFD2B68019A1C121340D14A9B000C
:102E50009B580435FEF7F7FCA4003E1B300000F041
:102E600094FE3700CA4B30601B780437002B01D02A
:102E7000FEF707FD2B68019A1C121340C54A9B0000
:102E80009B580435FEF7DFFCA300FE1A310020003A
:102E9000049300F02DFC049B3060FF1ABC4B0437F8
:102EA0001B78002B01D0FEF7ECFC2B68019A1C125A
:102EB0001340B84A9B009B580435FEF7C4FCA4009D
:102EC0003F1B380000F064FEB14B1B78002B01D093
:102ED000FEF7D7FC2B68019A1C121340AD4A9B00E9
:102EE0009B580435FEF7AFFCA300FE1A310020000A
:102EF000049300F02FFC049B3060FF1AA44B0437AE
:102F00001B78002B01D0FEF7BCFC2B68019A1C1229
:102F10001340A04A9B009B580435FEF794FCA40084
:102F20003F1B380000F07AFE994B1B78002B01D034
:102F3000FEF7A7FC2B68019A1C121340954A9B00D0
:102F40009B580435FEF77FFC0121200000F04EFE67
:102F50008F4B1B78002B01D0FEF793FC2B68019A56
:102F60001C1213408B4A9B009B580435FEF76BFCE8
:102F70000021200000F03AFE854B1B78002B01D089
:102F8000FEF77FFC2B68019A1C121340814A9B00BC
:102F90009B580435FEF757FCA4003E1B300000F0A0
:102FA0006BFE37007A4B30601B780437002B01D062
:102FB000FEF767FC2B68019A1C121340754A9B00B0
:102FC0009B580435FEF73FFCA4003E1B300000F088
:102FD00067FE37006E4B30601B780437002B01D042
:102FE000FEF74FFC2B68019A1C121340694A9B00A4
:102FF0009B580435FEF727FCA4003F1B380000F067
:1030000023FE634B1B78002B01D0FEF73AFC2B68A4
:10301000019A1C1213405F4A9B009B580435FEF72F
:1030200012FCA4003F1B380004F054FA584B1B78E4
:10303000002B01D0FEF725FC2B68019A1C121340CF
:10304000544A9B009B580435FEF7FDFBA4003E1B31
:10305000300004F0F9FA37004D4B30601B7804372C
:10306000002B01D0FEF70DFC2B68019A1C121340B7
:10307000484A9B009B580435FEF7E5FBA4003F1B24
:10308000380004F0CFF9424B1B78002B01D0FEF73B
:10309000F8FB2B68019A1C1213403E4A9B009B5878
:1030A0000435FEF7D0FBA4003E1B300004F0D4F939
:1030B0003700374B30601B780437002B01D0FEF708
:1030C000E0FB2B68019A1C121340324A9B009B586C
:1030D0000435FEF7B8FBA300FF1A3900200001F009
:1030E0001DFF2B4B1B78002B01D0FEF7CAFB2B6872
:1030F000019A1C121340274A9B009B580435FEF787
:10310000A2FBA300FF1A3900200001F00DFD204BA7
:103110001B78002B01D0FEF7B4FB2B68019A1C1220
:1031200013401C4A9B009B580435FEF78CFBA30000
:10313000FF1A3900200001F0A9FD154B1B78002B68
:1031400001D0FEF79EFB2B68019A1C121340114A16
:103150009B009B580435FEF776FBA300FF1A39004D
:10316000200001F0BBFD0A4B1B78002B01D0FEF7BD
:1031700088FB2B68019A1C121340064A9B009B583F
:103180000435FEF760FBC046D4050020B1020020E4
:10319000B002002024E30000A300FE1A310020004A
:1031A000049304F03BFB049B3060FF1AC64B0437CA
:1031B0001B78002B01D0FEF764FB2B68019A1C12D0
:1031C0001340C24A9B009B580435FEF73CFBA3000A
:1031D000FE1A31002000049304F028FB049B3060A9
:1031E000FF1AB94B04371B78002B01D0FEF749FBBF
:1031F0002B68019A1C121340B44A9B009B5804355B
:10320000FEF721FBA300FE1A31002000049304F016
:1032100015FB049B3060FF1AAB4B04371B78002B67
:1032200001D0FEF72EFB2B68019A1C121340A74A0F
:103230009B009B580435FEF706FBA300FE1A3100E5
:103240002000049303F0A8FF049B3060FF1A9E4BFC
:1032500004371B78002B01D0FEF713FB2B68019A73
:103260001C121340994A9B009B580435FEF7EBFA59
:10327000A300FF1A3900200001F0D0FD924B1B780B
:10328000002B01D0FEF7FDFA2B68019A1C121340A7
:103290008E4A9B009B580435FEF7D5FAA300FF1A0F
:1032A0003900200001F042FD874B1B78002B01D034
:1032B000FEF7E7FA2B68019A1C121340834A9B0021
:1032C0009B580435FEF7BFFAA300FE1A3100200018
:1032D000049301F0A7FC049B3060FF1A7A4B04377B
:1032E0001B78002B01D0FEF7CCFA2B68019A1C1238
:1032F0001340764A9B009B580435FEF7A4FAA300BE
:10330000FF1A3900200001F03BFC6F4B1B78002BAB
:1033100001D0FEF7B6FA2B68019A1C1213406B4AD3
:103320009B009B580435FEF78EFA002C7CDD3B1F7A
:103330001E68012C0CD1264207D1042E05D90F237B
:10334000326830001340042B11D001235B4213E09C
:10335000022CFAD13B00083B186801231842F4D133
:103360000428F2D902680E331340042BEDD100F08B
:103370003FFEFEF7EDF80300A200BF1A5A1C53D01F
:103380000020022C11D101223240824226D1042E8B
:1033900024D90F213068014009291FD171684810D4
:1033A000C0B28100914214D17F18FF2B1ED81C029D
:1033B000044323129C464648DBB2DB00C218117955
:1033C000414A032901D1FEF791FC02231370FEF755
:1033D00058FAB418A468BC500432E3E70B223A4B05
:1033E0001A7000233B600437FEF74BFA069A0299E5
:1033F000BA1A86009210BE1B0A613100984700225B
:10340000344B371D1A60304B30601B78934201D02B
:10341000FEF737FA2B68019A1C1213402B4A9B00C7
:103420009B580435FEF70FFA00233B60264B3A1DEC
:103430001B78002B02D01700FEF723FA2B680199A6
:103440001C120B4021499B005B5817000435FEF706
:10345000FAF9069B029AFB1A9B101361A300FF1A4C
:103460003900200003F06AF9174B1B78002B01D0BC
:10347000FEF707FA2B68019A1C121340134A9B00AF
:103480009B580435FEF7DFF9069B029AFB1A9B1046
:103490001361A300FE1A31002000049303F04EF9DB
:1034A000049B3060FF1A084B04371B78002B01D0B7
:1034B000FEF7E7F92B68019A1C121340034A9B00A0
:1034C0009B580435FEF7BFF9B002002024E300004A
:1034D000A8250020E40F00200023F7B55A1E019212
:1034E000002B07DA01F030FD03F040FA03F018FC7E
:1034F0001923019300263000194B1968B14212DDDF
:10350000184B1A6801328A420FDAF0241A601D68DB
:10351000154F6C43E35D002B1FD0E419022B06D13D
:103520002000FEF76FF9019BD8E70022EDE7012BA1
:103530000DD1002801D100F0E3FAF0226A43BB1854
:103540005B680A49C31A8B4201D80223BB54F0239B
:103550005D43054BEB5C022BE2D00136CCE7C04665
:10356000D805002000000020481C00203F420F002A
:1035700080220B4B52001A600121A822A920094B7E
:10358000D20019649A58C00005321A5006481A50E1
:10359000C122C020920000039850044B197070475C
:1035A00000E100E0008000404C0500000306002020
:1035B00004207047F8B550C9012322001A40101E9C
:1035C0002DD03340181E2AD0641000201C2C26D881
:1035D0001D4B761035009E4200DD1D001B4F3B5DEC
:1035E000012B05D00121200005F094FC01233B555F
:1035F000174B1B78002B01D1FFF7BAFF0023154AA8
:103600009E420DDCFF2514491448D65CB44202D119
:103610005E007052D5540133042BF6D10420F8BD5E
:10362000D15C8C4203D10C4A5B009D52F6E701331A
:10363000042BF5D10023D15CFF2901D1D454F2E74A
:103640000133042BF7D1E9E788130000E4050020DB
:10365000030600201C0000200E000020DC050000F6
:1036600070B530C9012322001A40101E1BD02B4018
:10367000181E18D064101C2C00D90024154E335D80
:10368000012B05D00121200005F044FC0123335516
:1036900069100800104A1038104B904204D90122DA
:1036A00052421A60042070BD1C600D4807F0E0F81B
:1036B0000C4B040018800C4B1B78002B01D1FFF73A
:1036C00057FF0122094B9A64A922D2009958641825
:1036D0009C50E7E7E40500209086010018000020D8
:1036E00020A107000C0000200306002000800040FD
:1036F000F8B501240B6806000D00234204D10D200B
:10370000FEF74AF82000F8BD5B102000052BFAD820
:103710000E4A9B009C580E4F3B5D002B05D00021AC
:10372000200005F0F7FB00233B55012E06DD6B68FA
:10373000042B03D10221200005F0ECFB200005F052
:1037400097FA012440002043DDE7C046F8E5000079
:10375000E405002070B501240D68254204D10D2038
:10376000FEF71AF8200070BD6D101C2D17D800242C
:10377000012804DD4C68043C63425C416400094E4E
:10378000735DA34204D02100280005F0C3FB7455EB
:10379000280005F0F3FB03000420012BE3D00020F8
:1037A000E1E7C046E4050020F8B501260D683400C5
:1037B000B04200DD4C682B003340181E0BD02300B4
:1037C0003340181E07D06D10002D05DCA12300200A
:1037D0001E4ADB00D650F8BD641000201C2CFAD81D
:1037E0001B4F3B5D012B04D00121200005F092FB13
:1037F0003E552900174807F03BF80A21053007F02D
:1038000037F8154BA400E258144B12021343A222BE
:103810001349D2008B50134C0C4B9C50124C195135
:10382000012412495C50124B196900219950114A28
:10383000904200DD1000A8228021D2009850012281
:1038400089005A5004201A60C5E7C04600F00140C4
:10385000E405002000B4C40428F8000003000300BD
:103860000060004040A10040140500000405000075
:1038700000A00040FFFF0000030010B50120002B56
:1038800002DC1B30FDF788FF10BD10B50124044099
:1038900002D04410200010BD042810D90F23026864
:1038A0001340042B07D100F0A3FB21000A2209F0EA
:1038B00075FD0400EEE7032B01D10430F5E70D2080
:1038C000FDF76AFFE6E70000F8B50C00022803DC0C
:1038D0001C20FDF761FFF8BD0868FFF7D6FF060062
:1038E0006068FFF7D2FF0500A068FFF7CEFF010078
:1038F000794806F0BDFF04001C2D01D90020EAE73D
:10390000764F7B5D012B05D00121280005F002FBDD
:1039100001237B550021280005F01AFB002C0ED056
:1039200020000138C046C046C046C046C046C0461A
:10393000C046C046C046C046C046C046F1D1012779
:1039400031002800394005F003FB002C0ED0200088
:103950000138C046C046C046C046C046C046C04604
:10396000C046C046C046C046C046F1D1711039407D
:10397000280005F0EDFA002C0ED020000138C046DA
:10398000C046C046C046C046C046C046C046C04607
:10399000C046C046C046F1D10127B11039402800C9
:1039A00005F0D6FA002C0ED020000138C046C046E3
:1039B000C046C046C046C046C046C046C046C046D7
:1039C000C046C046F1D1F1103940280005F0C0FAD8
:1039D000002C0ED020000138C046C046C046C0466C
:1039E000C046C046C046C046C046C046C046C046A7
:1039F000F1D1012731113940280005F0A9FA002C36
:103A00000ED020000138C046C046C046C046C04661
:103A1000C046C046C046C046C046C046C046F1D1BA
:103A200071113940280005F093FA002C0ED02000C7
:103A30000138C046C046C046C046C046C046C04623
:103A4000C046C046C046C046C046F1D10127B111AC
:103A50003940280005F07CFA3900002C0ED02000F7
:103A60000138C046C046C046C046C046C046C046F3
:103A7000C046C046C046C046C046F1D1F6113140EE
:103A8000280005F065FA002C0ED020000138C04651
:103A9000C046C046C046C046C046C046C046C046F6
:103AA000C046C046C046F1D10121280005F050FAB9
:103AB000002C00D122E720000138C046C046C04695
:103AC000C046C046C046C046C046C046C046C046C6
:103AD000C046F1D112E7C04640420F00E405002085
:103AE0000420704710B5002803DC1C20FDF754FEAD
:103AF00010BD0B680020DB07FAD40D30F6E700009C
:103B00000122034B1A64A822D20098587047C0467D
:103B1000008000400122054B10B51A64A822FA214A
:103B2000D2009858890006F019FE10BD00800040B0
:103B30000048704710E600001D20704770B5054E24
:103B40000400335C0D008B4202D005F0E3F93555DB
:103B500070BDC046E405002070B50024084D635DCB
:103B6000012B09D10021200005F0F2F900212000ED
:103B700005F0D0F90023635501341D2CEED170BD42
:103B8000E405002070470D2070473B20704700007F
:103B9000F8B501260568354202D04468344203D1A5
:103BA0000D20FDF7F9FDF8BD6D101C2DFBD80A4F57
:103BB0007B5D012B04D03100280005F0ABF97E5568
:103BC000064964108C4202DCE143C91721402800F9
:103BD00005F0D4F8E7E7C046E4050020FF03000045
:103BE00010B50800FFF7D4FF002010BD70B5040029
:103BF0000D001C280ED8084E335C012B04D0012187
:103C000005F088F901233355290020004D1EA941F4
:103C100005F09EF970BDC046E4050020036810B5AC
:103C2000DA0703D40D20FDF7B7FD10BD4168581029
:103C300004394A425141FFF7D9FFF6E710B50800B1
:103C4000FFF7ECFF002010BD37B569460A00064BB0
:103C500030CB30C203680220042B02D101F016F8E9
:103C600037BD01F03BF8FBE788E5000010B5080020
:103C7000FFF7EAFF002010BD10B5084C6379002B58
:103C800005D00021052005F045F9002363710520CA
:103C900005F074F943425841800010BDE40500204E
:103CA00010B5084CE37A002B05D000210B2005F05D
:103CB00031F90023E3720B2005F060F943425841CB
:103CC000800010BDE4050020A02200230349D2009B
:103CD0008B50034910328B507047C04600F00140B2
:103CE00000600040F7B52F4D2F4EEB6C002B14D029
:103CF000A9240023E4003759EB642C4B18680028F2
:103D00000BDB2B4B19784A425141C9B2197005F0AF
:103D10001FF9284B1B88DF1937512B6D002B38D02A
:103D20000021254B254FF45829653A780193244DFD
:103D30008A4206D02B68032B03D8224AD05C05F0B8
:103D400007F92B68204A0133134004D50422013BB4
:103D50005242134301331B4900228C462B60042B33
:103D600018D06046C05C591CFF2802D10B0001220C
:103D7000F5E7002A00D02B60012105F0E9F80123C6
:103D80003B702B68114A5B009B5A0C34E418019B72
:103D9000F450F7BD01235B422B6000233B700C4BBA
:103DA000F4E7C046FC80004000800040180000207E
:103DB000020600200C0000204C0500000106002037
:103DC000E00500201C000020030000800E00002001
:103DD0005C460000084B094AFF201A805A809A80EE
:103DE000DA800023064A07491370074A08704870B2
:103DF0008870C870136070470E000020DC0500005A
:103E0000010600201C000020E00500200122024BDA
:103E100052421A607047C0461800002010B5034A8D
:103E20000D21034802F0C0F910BDC04690E5000026
:103E30005BEF0000E12170B54902194804F08EFCE7
:103E4000002401220320174B17491A615C500431EA
:103E500058508018083158501A60063004F002FF9C
:103E6000FF21124AA15401341D2CFBD10122002054
:103E70000F4B01001A6004230E4A0F4D1468002CEA
:103E8000FCD02C680002013B20431160002BF5D1CF
:103E900001220A4B1A6004F01DFE01F09BF970BD6F
:103EA000D01B00200080004004050000E405002035
:103EB00000D0004000D1004008D5004004D00040B0
:103EC000F8B50B4E070030000D0004F08FFC040025
:103ED000A84200DD2C003D00EB1B9C4205DD3000BC
:103EE00004F08EFC28700135F6E72000F8BDC046CE
:103EF000D01B002010B50100014804F037FC10BDB4
:103F0000D01B002010B5054C200004F03DFCE12141
:103F10002000490204F022FC10BDC046D01B002046
:103F2000C3070CD4064B1B68834208D8054B1B689B
:103F3000984204D8031F1B68002B00D0180070475C
:103F40000C060020080600200023012210B50A48B4
:103F5000990001334250642BFAD1084C084B0021E0
:103F60001A602000074A08F0C7FD074B074A636044
:103F7000074B1A6010BDC046A02D0020100600207F
:103F800008000020D409000030270000140600209B
:103F90000406002010B5044B044A1A60044B054A7D
:103FA0001A60FFF7D1FF10BD0C060020100600209C
:103FB00008060020E40F0020044B1B681868000965
:103FC00080B20238C343DB17184070470406002054
:103FD00000B59BB00200054901A809F0D1F801A87D
:103FE00002F086FB02F09CFEFCE7C046E8E600001B
:103FF0000B4BC20704D4042804D80A4B00D00A4B48
:10400000180070470F2203681A40031D042AF7D0D6
:10401000064B092AF4D0064B032AF1D0054BEFE7F3
:10402000C2E60000B2E10000ACE10000CCE6000016
:10403000DCE60000D3E600000020064A0649131F14
:10404000186013681B099BB202339B00D2188A4286
:10405000F5D3704714060020E40F0020F7B50F24B5
:104060000126314B314A1968314B324D18681368BB
:104070001F002740072F26D813681B099BB2023365
:104080009B00D218AA42F2D300242B4EA500AD19F2
:104090002868FFF745FF01342860642CF6D1274CCF
:1040A0002068FFF73DFF2060254C2068002802D0E3
:1040B000FFF736FF20600025224B1B680093009B12
:1040C0009D4214DBF7BD1B099BB29B00D3189A429B
:1040D000D2D01F68374208D1B94206D2B84204D3C1
:1040E000043F3F68002F00D01F60043BEFE7F02340
:1040F0006B43154A9B181A78002A01D10135DEE777
:104100001F693C2300266B43DB199B00019301369A
:10411000BB1BF3D4019BB4001C1B0B4B1C19A069E7
:10412000FFF7FEFEA061F2E70C0600201406002057
:1041300008060020E40F0020A02D00200800002029
:10414000E40F0020D8050020481C0020F7B501240A
:10415000204246D1234B1B689C46984241D3224BB8
:104160001B68019398423CD8031F1B68002B38D171
:104170000200036800941B099BB2002B0FD1009929
:10418000131F196090422CD015682B1F1B689900D3
:1041900069180C68013B14600A602A00EDE79D0075
:1041A00055192968009C214219D18C4517D8019CCA
:1041B0008C4214D30E1F3468002C10D10F680F34BA
:1041C0003C40072C08D92F60151F2B600B680A6034
:1041D0001B099BB20A00D0E700993160CDE7013B93
:1041E000CBE7F7BD0C060020080600200D4970B58E
:1041F0000A000D4D1368141F1B0926689BB2981CFA
:10420000002E0BD000238A4200D00B0023608300D5
:10421000C91880001218AA42ECD370BD1B011360AC
:10422000F7E7C04614060020E40F0020F8B5124C52
:1042300027000F223B681D09ADB213420DD06E1C42
:10424000B600A74204D032003900200008F041FC3B
:104250000022A3190436A4191A600235AD00074BD9
:104260007F199F42E5D31B1B9B10013B1B01236061
:10427000034B1C60F8BDC04614060020E40F00206C
:1042800004060020F0B59BB0FFF73AFC00240700BD
:10429000214AA300D0580134FFF758FF642CF7D10E
:1042A0001E4B1868FFF752FF1D4B1868002801D0FD
:1042B000FFF74CFF00261B4B1B689E4217DBFFF7E6
:1042C00095FFFFF7CBFEFFF7B1FFFFF719FC164B89
:1042D000C21B1B6815491B6801A81B099BB2023B46
:1042E00008F04EFF01A802F003FA1BB0F0BDF02564
:1042F00075430F4BED182B78002B01D10136DAE70F
:104300002B695C1E002CF9DBA300EB189869FFF702
:104310001DFF013CF6E7C046A02D0020080000204C
:10432000E40F0020D805002004060020A2E60000CB
:10433000481C0020F7B5174D4F1C2B6806001B6862
:104340000C001B099BB201929F420BDBFFF79AFF07
:104350002B681B681B099BB29F4203DB0A20FDF7F9
:104360001BFAFEBD2868A71CBA00DB1B81181B01C5
:104370000B6029600021031F19600F231E400300FA
:104380002401264340C3083A9A189A42E9D9019970
:1043900002C3FAE704060020F7B503000122134028
:1043A00004000D000193002B2BD1174B1B68834297
:1043B00027D8164B1B68834223D90F23144F38602C
:1043C00000681840FFF7B6FF019B3C68061E3B6083
:1043D00017D0236804301B099BB29D4200DD1D00ED
:1043E000AA00211D251F08F06BFBFFF725FE2E609C
:1043F000FFF734FE00232B602268064B1340236036
:1044000034002000FEBDC0460C0600200806002037
:10441000E40F0020F0FF0F000323043010B5C11794
:1044200019400918891000220420FFF783FF10BDEE
:1044300070B5050008000C00FFF7EEFF0023002810
:1044400004D170BDE95CC21811710133A342F9DBDC
:10445000E343DB171C40002304192371F1E7F0B597
:104460000C009BB0022804DC1C20FDF795F91BB062
:10447000F0BD01230868184206D1042804D90F268C
:1044800001683140042901D00E20EEE761680D007B
:104490001D40F9D10429F7D90A683240042AF3D122
:1044A000A2681A4201D10D20DFE7FFF7A1FD060047
:1044B0006068FFF79DFDA768010001AC7F10300028
:1044C000257003F075FD39006423220003F0D5FD4B
:1044D000200008F09BFE01002000FFF7A9FFC6E7BF
:1044E00010B51C4CA544041E02D1FFF795FF0BE04C
:1044F00003F076FC0138062828D806F01BF90909D4
:1045000011182904240000208023DB009D4410BDE5
:10451000200003F0E1FC011B2000FFF789FFF3E717
:10452000200003F087FC430001201843ECE78022C1
:104530006946D200200003F094FC684608F066FE4D
:1045400001006846E9E704210348E6E70020CCE7DC
:104550000420D9E700FCFFFF40E7000070B50C0025
:10456000022803DC1C20FDF717F970BD0123086841
:10457000184206D1042804D90F25016829400429CE
:1045800001D00E20EFE761681942FAD10429F8D969
:104590000A682A40042AF4D1A2681A4201D10D20E7
:1045A000E1E7FFF725FD05006068FFF721FDA4683E
:1045B00001006410280003F0FBFC210003F038FD2B
:1045C000FFF78EFFD1E770B50D00012803DC1C203A
:1045D000FDF7E2F870BD01240868204206D10428E6
:1045E00004D90F2102680A40042A01D00E20EFE707
:1045F0006A682242FAD1042AF8D913680B40042BC6
:10460000F4D1FFF7F5FC06006868FFF7F1FC010044
:10461000300003F0CDFC03F04FFD40002043D9E70C
:10462000F8B507000C001C20012F0BDD01250868E0
:10463000284206D1042804D90F2102680A40042A1E
:1046400003D00E20FDF7A8F8F8BD62682A42F8D121
:10465000042AF6D913680B40042BF2D1FFF7C8FCEB
:1046600006006068FFF7C4FC0100022F14D0A468A4
:104670002C4211D06410300003F09AFC050003F0C6
:10468000AFFB012811D1002C02DD0135012C06D130
:104690002800FFF725FFD7E701246442EBE7280055
:1046A00003F027FC013C0500F0E70228F0D1002CC4
:1046B000EEDD0135012CEBD000222800110003F0C3
:1046C0004AFC03F016FC013C0500F3E7086870B5EE
:1046D00001240500254006D1042804D90F230268CF
:1046E0001340042B03D00E20FDF756F870BDFFF7E2
:1046F0007FFC03782900233B5A4253411022C01803
:1047000008F04CFE80239B05C218044B9A4201D945
:104710001420E9E740002043E8E7C046FFFFFF3FE1
:1047200010B50124044002D04410200010BD04281C
:1047300010D90F2302681340042B07D1FFF758FC50
:1047400021000A2208F02AFE0400EEE7032B01D123
:104750000430F5E70D20FDF71FF8E6E710B508680F
:10476000FFF7DEFF06F018FB094906F0E3F908F051
:10477000C9F804F011FD074B002207F07DFA04F0A0
:10478000B3FC08F04FF843000120184310BDC046A9
:10479000D30237390000D040F7B50C00042803DC01
:1047A0001C20FCF7F9FFFEBD0868FFF7B9FF019078
:1047B0006068FFF7B5FF0600A068FFF7B1FF0500CE
:1047C000E068FFF7ADFF07002069FFF7A9FFAE42E1
:1047D00001D11F20E5E7019BC01B9B1B5843A91B70
:1047E00006F046F8C71901207F003843DBE70000D8
:1047F00010B5034A0821034801F0D6FC10BDC0469D
:1048000000E70000F9E600000020704710B51E2008
:10481000FCF7C2FF10BD10B51E20FCF7BDFF10BD98
:1048200010B51E20FCF7B8FF10BD10B51E20FCF718
:10483000B3FF10BD10B51E20FCF7AEFF10BD10B5C4
:104840001E20FCF7A9FF10BD10B51E20FCF7A4FF29
:1048500010BD10B51E20FCF79FFF10BD10B51E2027
:10486000FCF79AFF10BD10B51E20FCF795FF10BD98
:1048700010B51E20FCF790FF10BD10B51E20FCF7F0
:104880008BFF10BD10B51E20FCF786FF10BD10B5C4
:104890001E20FCF781FF10BD10B51E20FCF77CFF29
:1048A00010BD10B51E20FCF777FF10BD10B51E20FF
:1048B000FCF772FF10BD10B51E20FCF76DFF10BD98
:1048C00010B51E20FCF768FF10BD10B51E20FCF7C8
:1048D00063FF10BD10B51E20FCF75EFF10BD10B5C4
:1048E0001E20FCF759FF10BD10B51E20FCF754FF29
:1048F00010BD10B51E20FCF74FFF10BD10B51E20D7
:10490000FCF74AFF10BD10B51E20FCF745FF10BD97
:1049100010B51E20FCF740FF10BD10B51E20FCF79F
:104920003BFF10BD10B51E20FCF736FF10BD000088
:1049300010B5034A1E21034801F036FC10BDC046E5
:1049400094E7000084E800000120034B1860034B4B
:104950001B6883401843704704100020E80F0020B4
:10496000F0B5EFF310810123194083F31088134A47
:10497000A1261268124D013A9340A022114FD20590
:10498000F600002B17D02C68945103420BD0C04680
:10499000C046C046C046C046C046C046C0462C6859
:1049A000D4515B08EDE7D451C046C046C046C0466E
:1049B000C046C046F5E781F31088F0BD2000002016
:1049C000F40F00200C05000030B585B001AD0C22BD
:1049D0000649280008F074F80024285D01210134FC
:1049E000FFF7ACF80C2CF8D105B030BD11EA00008F
:1049F00030B585B001AD0C220649280008F060F8FA
:104A00000024285D00210134FFF798F80C2CF8D120
:104A100005B030BD11EA0000F7B56A463B4B01AE68
:104A200013800A2393703A4B33801C23B370FFF733
:104A300067F8384B384DC0182B68984201D20023D4
:104A40002B602C68002C41D1375D01213800FFF725
:104A500075F801340021380004F07AFA032CF3D100
:104A6000002401276B461E5D39003000FFF766F811
:104A700001343900300004F06BFA032CF2D1C82065
:104A80000138C046C046C046C046C046C046C046C3
:104A9000C046C046C046C046C046F1D16B46002164
:104AA0001878FFF74BF86B4600215878FFF746F867
:104AB0006B4600219878FFF741F8FFF721F8FA23B9
:104AC00000241B01C01828602000FEBDFFF718F865
:104AD0002B6800249842F7D3032004F0C9F806009D
:104AE000042004F0C5F836180A2004F0C1F80B4B76
:104AF0009B1B181A0A4BA04206DB18600023094AC8
:104B00002B6013600124DFE71C60F7E7030400005B
:104B10001A1B000010270000FC0F0020E303000018
:104B2000E80F0020041000200022054B10B51A6089
:104B3000044B1B68934201D003F0F2F8002010BD33
:104B400000100020F41A002010B5041E0CDA002416
:104B5000084BA400E2581F231A401E3B9340064A0C
:104B60001360064A136010BDFEF7E6FFA042EEDDBB
:104B7000EEE7C04628F80000F40F002018050050AA
:104B80000200086810B5C3070FD540101823012A8A
:104B900003DD4A68042A00D10833054A1360FEF792
:104BA000F1FFFFF7D1FF002010BD01204042EDE7EB
:104BB0002000002010B500280CDD0A68131F591EC4
:104BC0008B4107490B60042A06D0FFF711FF002232
:104BD000044B1A60002010BDFFF7F6FEFAE7C0464E
:104BE000F80F0020E80F002010B50124044002D087
:104BF0004410200010BD042810D90F230268134070
:104C0000042B07D1FFF7F4F921000A2208F0C6FBB4
:104C10000400EEE7032B01D10430F5E70D20FCF78B
:104C2000BBFDE6E70868F8B5C3071AD5FFF7DCFF58
:104C30000300203B5E2B25D80520434301221D188D
:104C40000020114E9D4219D005211024F75C3C42F2
:104C500000D080180139520064100029F7D10133C7
:104C6000F0E704280ED90F2203681A40042A09D15C
:104C70001B099BB2002B05D00379DAE70123400022
:104C80001843F8BD0120FCE71DEA000070B5086874
:104C90000D00FFF7A9FF04006868FFF7A5FF621E7B
:104CA0000100042A14D8451E042D11D805236B4396
:104CB0009B18012215009D402B00064805682B43D8
:104CC0000360054B1B68002B02D0200003F029F87D
:104CD000002070BD00100020F41A002070B5086894
:104CE0000D00FFF781FF04006868FFF77DFF621E7B
:104CF0000100042A13D8451E042D10D805236B4348
:104D00009B1801229A400748036893430360064BAF
:104D10001B68002B03D00022200003F002F80020C3
:104D200070BDC04600100020F41A0020F0B5050048
:104D300089B008680C00FFF757FF0690022D36DD9A
:104D40006068FFF751FF0190A068FFF74DFF040076
:104D50000127231D661E0793731C0293079B9E4227
:104D600035D0052373430593019B019D05330493BF
:104D7000049BAB421ED0042E16D86B1E042B13D8F6
:104D80000122059B2349013B5B199A409446224A24
:104D90000B681068069A3A4003920DD062461A4397
:104DA0000A60012200280DD17F000135E0E70124CF
:104DB0000194CDE7029ECFE7624693430B60002843
:104DC000F2D0039A0299280002F0ABFFECE7019BB6
:104DD0001E1D042E1AD8012C18D1002505273B00D2
:104DE00021006B439B1999400B000A4A0135116859
:104DF0009943094B11601B68002B05D0019B0022D1
:104E0000581D290002F08DFF052DE8D1002009B0C2
:104E1000F0BDC04600100020F41A0020F0B53B4B56
:104E200085B01B680C00002B03D101204042FFF726
:104E30008BFE012627683E403CD1042F3AD90F2330
:104E40003A681340092B35D17B685B100293029BB3
:104E50009E4258DAB300FB189868FFF7C5FEFF239F
:104E600005000414001218401C4029492B404043FF
:104E7000019305F0FDFC03042000254960430393E2
:104E800005F0F6FC039C00020443019820494043CE
:104E900005F0EEFC1F4B20431B68202B06D1AD0014
:104EA000AD0E1D4BAD00EC5800022043FFF758FD3E
:104EB0000136CCE73800FFF797FEFF260500071400
:104EC000001230401249404305F0D2FC3740040440
:104ED00038000F49784305F0CBFC2E400002044314
:104EE00030000B49704305F0C3FC0A4B20431B689C
:104EF000202B06D1AB009B0E074A9B009B5800025B
:104F00001843FFF72DFD002005B0F0BDF40F002081
:104F10005906000020000020F8EB0000086810B5DA
:104F2000C30703D5FFF760FE054B1860054B1B68F0
:104F3000002B03D0024B186802F0F4FE002010BDD5
:104F400000100020F41A00209D4B70B51B68002B48
:104F50000DD19C4C2368002B0AD19B4A1268002A71
:104F600006D19A4B1B68002B01D0FFF755FD70BD91
:104F7000974D2A68002A1BD1944A1268002A10D043
:104F8000FFF74AFD0028F2D0FFF71EFD8E4B226886
:104F900019681A6000290BD0002A09D1FFF728FDF3
:104FA000E5E7894A1268002AF0D1002BEED0EBE742
:104FB00000211A2003F0CCFF00211B2003F0C8FFC2
:104FC00000211C2003F0C4FF2E68012E5CD0022EAD
:104FD00000D1A2E0002E50D1013631007A4C0320DE
:104FE0002368994303F0B4FF0420216801404B4239
:104FF000594103F0ADFF102123680A2019404B42AC
:10500000594103F0A5FF80212368090119404B4253
:105010005941062003F09CFF8021236809021940B2
:105020004B425941072003F093FF80212368490236
:1050300019404B425941092003F08AFF802123681F
:10504000890219404B425941192003F081FF802108
:105050002368C90219404B425941182003F078FFD8
:10506000802321681B0319404B425941172003F04C
:105070006FFF31001A2003F06BFF2B680321581CCF
:1050800005F0DCFC296072E702214F4C17202368F1
:1050900019404B42594103F05BFF08212368182057
:1050A00019404B42594103F053FF80212368C90046
:1050B00019404B425941042003F04AFF80212368E4
:1050C000490119404B4259410A2003F041FF802118
:1050D0002368C90119404B425941032003F038FFAE
:1050E00080212368890319404B425941092003F06C
:1050F0002FFF802321681B0419404B42594119207E
:1051000003F026FF3100062003F022FF31000720C4
:1051100003F01EFF31001B20ADE720212A4C172091
:10512000236819404B42594103F012FF4021236884
:10513000182019404B42594103F00AFF802123688F
:10514000192019404B42594103F002FF8021236886
:10515000490019404B425941092003F0F9FE8021D2
:105160002368890019404B425941072003F0F0FEA3
:1051700080212368890119404B425941062003F0E0
:10518000E7FE80212368490319404B4259410A2018
:1051900003F0DEFE80212368C90319404B425941C8
:1051A000032003F0D5FE802321685B0419404B42A5
:1051B0005941042003F0CCFE01211C205BE7C046CE
:1051C000F80F002000100020F00F00200410002035
:1051D000EC0F0020012010B54042FFF7B5FC10BDD8
:1051E00010B5034A0A21034800F0DEFF10BDC04697
:1051F000F8EC000048ED00008023F0B502255B05C7
:105200001A690A4C0A4BA1261D5103278025F60076
:10521000ED00BA43884202D300221A51F0BD5F5913
:10522000002FFCD098518018F4E7C0460405000018
:1052300000E0014010B5002806D1C020B021400296
:105240008902FFF7D9FF10BDB02080218002C9027A
:10525000F7E7000043425841064B40421840B02354
:105260009B02C018036800201A0E532A01D11B02AA
:10527000180A704700C0FEFF30B501248025054B99
:10528000054AED009C505C59002CFCD001600021C7
:10529000995030BD00E001400405000043425841F0
:1052A000074B40421840B0239B02C018A62310B5FC
:1052B0000902DB05090A1943FFF7DEFF10BDC046EE
:1052C00000C0FEFFF0B5012480260D4B0D4DF60009
:1052D0005C51002902DC00225A51F0BD5778147845
:1052E0003F022743947824042743D47804322406C9
:1052F0003C439F59002FFCD010C00139E9E7C0465C
:1053000000E001400405000070B505004B680A008C
:105310009C1C2100A400FFF7D5FF281970BD0000D8
:10532000134B1B68002B0CD08022B023D2029B02AF
:1053300000280BD11A1D5B681B0E522B00D11000E8
:105340007047B022C02392025B02F1E782420DD97E
:1053500003681B0E522B09D1436802339B00C0180F
:10536000824203D903681B0E522BE9D00020E7E7E5
:1053700008110020F0B50020B7B00024FFF7D0FFDF
:10538000270005002600002D2ED1284D2868FFF7A4
:1053900061FF32003B0001900094254904A807F00A
:1053A000EFFE04A801F0A4F9224B64201C682B68CE
:1053B000A0215A425341204A5B421340B02292023C
:1053C0009B18E41A6043490205F052FAA0225202E7
:1053D000030000921949220004A807F0D1FE04A896
:1053E00001F086F937B0F0BDFF226B6829689C4652
:1053F0000233FF180B12013613409C4200DA1C00E6
:10540000FF200A140240039262460140019200917B
:10541000039A0B4904A807F0B3FE04A801F068F949
:105420002800FFF77DFF0500ADE7C046081100200A
:1054300062EE00000C11002000C0FEFF0CEE000028
:105440004EEE000070B50020FFF704FF04000120BD
:10545000FFF700FF844200DA04000A4B1D686A422D
:10546000554128001D60FFF7E5FEA0226B42520265
:105470001340054A28009B18044A611C1360FFF77B
:105480000DFF70BD08110020048001000C110020E8
:10549000F8B50020FFF7DEFE07000120FFF7DAFE77
:1054A0003E00204D0643204C0DD18021C020C90272
:1054B0004002FFF7A1FE01213000FFF7EFFE1B4B7A
:1054C0002E6023601DE0874209DD0023B0212B60A0
:1054D000164B8902236023680020012517E0012371
:1054E00080212B60124BC9022360F4E7120E522A6E
:1054F00008D0002800D023600E4801F0F9F8FFF72B
:10550000A1FFF8BD28005A68023292009B188B4216
:1055100005D21A68561CE9D10028F2D0D1E72160E3
:10552000EFE7C046081100200C11002004800100A4
:1055300004C0020027EE000070B50020FFF7F0FE67
:10554000FF260500002801D1280070BD03681C1447
:105550003440FFF7E5FEDA2CF4D10500F2E7000055
:10556000FF2270B51F4CD2000021200007F0C4FAC2
:10557000FF25FFF7E1FF0026002818D1F0210A22BD
:10558000194849420B00962553432D011B185D19FC
:105590002D78002D07D0154D154E5D199B191B78E0
:1055A000DB00E3582B60013A002AEBD170BD0368A1
:1055B0001A142A400A2A0AD11A122A40FF2A03D0B2
:1055C000D200A1180B71A050FFF7AAFED4E7132A4E
:1055D000FAD11B122B40FF2BF6D0DB00E21816711C
:1055E000E650F1E7A8250020481C002068090000CB
:1055F0006109000010B59AB0FFF74AFFFFF7B0FF4E
:1056000000231A000A48D900415801334C1EA14119
:105610005218FF2BF7D1074901A807F0B1FD01A8E7
:1056200001F066F8044801F063F81AB010BDC046F6
:10563000A825002097EE0000ABEE00008022F0B518
:105640005200A1B00021684807F056FA80220021DC
:105650005200664807F050FA654BFF271B681A0096
:10566000049353425A4110000592FFF7E3FD049C56
:105670000020631E9C415F4B64421C405E4BE4185B
:10568000FFF75AFF0600002E2FD10498FFF7E2FD26
:10569000411C0598FFF702FE059A554B574D1A60BD
:1056A0002C60FFF75DFFFEF72DFC514B64201B685B
:1056B000A0215A4253414F4A5B421340B0222C680A
:1056C00092029B18E41A6043490205F0D1F8A02227
:1056D0005202030000924A49220007A807F050FD39
:1056E00007A801F005F821B0F0BD326813141212BA
:1056F0003A403B4003921A000A3A092A49D83A4BE9
:10570000039A995C002931D110223E4807F0F4F940
:1057100035002B6803991A123A40914209D11A14A4
:105720003A400B2A27D0132A2DD00A2A01D1354B13
:105730001D602800FFF7F4FD051EEAD1314B196802
:1057400000290FD02000FFF7DFFD04002D4B5B196F
:105750005968002903D02000FFF7D6FD0400043566
:105760000C2DF3D1204B0121039A99543000FFF7FF
:10577000D7FD060087E73B40022BDADC214A9B007D
:10578000D3185D60D5E7102200211E4807F0B4F958
:10579000CFE71A00153A082AE8D8144A0399525C50
:1057A000002AE3D13500152B00D015003000036826
:1057B0001A143A40152A0FD01D2A00D10025FFF7F0
:1057C000AFFD0028F3D1002D04D020002900FFF701
:1057D0009BFD0400054BC6E7039A1B123B409A420F
:1057E000EDD10500EBE7C0460810002010110020A5
:1057F0000811002000C0FEFF04C002000C110020B0
:10580000F1ED0000302F002010B5FFF717FF10BD9D
:10581000F0B585B0039203220333DC17294D144001
:10582000E4182B68284F5A42534180225B42D2022F
:10583000A4103B409B18A21C0291244E91000091A1
:105840000190316800980A18934215D2FFF7F6FECE
:105850002B685A42534180225B421F40D202BF183C
:105860003368009A9B189F4206D2194800F040FF07
:105870000025280005B0F0BD029B356819066B466F
:105880001A7BA423DB051343FF222F00090C1943C5
:10589000019B12041B04134019432800FFF7ECFC82
:1058A0000837281D21003760FFF7E6FC002C04D0E4
:1058B0000A9A21003800FFF705FD009B083BFF18FE
:1058C0003760D6E70811002000C0FEFF0C11002051
:1058D000CBED0000704770470021094B094A596021
:1058E0000131516059680029FCD000211961012360
:1058F00093600222044B8131FF315A501A60704785
:10590000FC1000400010004000E100E00222064BC5
:105910000121DA670022054B5A61054A11615A6973
:10592000002AFCD07047C04604E100E0FC100040B3
:105930000010004010B5044C2378002B01D0FFF775
:10594000E5FF0020207010BD111200200120024B45
:105950001B685B0018437047941200200120024B23
:105960001B685B0018437047240000201FB5064BDE
:1059700006491A6801A807F003FC082101A8FEF7F0
:1059800057FD05B000BDC046981200203CEF000056
:105990001FB580235B051A6E044901A807F0F0FBD0
:1059A000082101A8FEF744FD05B000BD3CEF000052
:1059B00010B5044C200007F029FC01002000FEF780
:1059C00037FD10BD9D1200200E4B10B51B680E4C0C
:1059D0005A1C0FD00D4C002B0CD00D4C012B09D0B4
:1059E0000C4C022B06D0094C042B03D00A4C052B7F
:1059F00000D1074C200007F009FC01002000FEF751
:105A000017FD10BD2800002041EF000068E50000F0
:105A10004CEF00006FE5000046EF000070B5040099
:105A20000D001600FEF776F88023012200215B05A9
:105A30001B6E6270E270020AA271020CE2711A0A15
:105A400060716372000EA2721A0C1B0E2670257113
:105A5000A1702072E272237370BD000070B5214CFA
:105A60002278002A3DD1204B01215A608022D205A4
:105A700011605A68002AFCD0002207201B4B1C49E9
:105A800001255A500439585008315A5019481A49BA
:105A900058501A491A485A501A495A50A622D20048
:105AA0009D50082218495A50043158500220174975
:105AB000585017491748585017480439585018205B
:105AC00016495850C12189005A500539FF39585894
:105AD000921802435A501249124A9950FFF7FCFE9D
:105AE000257070BD11120020FC0000400010004025
:105AF0000C050000746962751C0500002405000097
:105B0000200004022C0500001405000034050000EC
:105B10003C050000FFFF00002110010054050000BB
:105B2000121200200405000013B5094B0400009375
:105B3000084B019307280AD8074B1B78002B01D18B
:105B4000FFF78CFF6B46054A1957054BD15013BD23
:105B5000E2ECF0F4F8FC0004111200200010004008
:105B60000C05000070B50E4B06001B78002B01D110
:105B7000FFF774FF00200B4D2C7884420ED00A4BA7
:105B8000202219780323091B1940084B4901C91821
:105B9000300006F095FF0120013C2C7070BDC0461E
:105BA000111200209C12002010120020121200205E
:105BB000002370B588B0984235DD0D6801262C00B1
:105BC00034409C422FD12300042D2CD90F222B6866
:105BD0001A402300092A26D16A683F2A23DD684635
:105BE000FFF7C0FF230000281DD06B461978330053
:105BF000A14203DB6B461B5D5B003343A200AA1886
:105C000001349360202CF2D1092169444A780B7841
:105C100012021A438B781B041A43CB781B061343DA
:105C2000024A13600423180008B070BD98120020C7
:105C300070B5454B8AB01B78002B01D1FFF70EFFE2
:105C400002AC2000FFF78EFF002802D100200AB02E
:105C500070BD23780B2BF9D96378012BF6D1E3784B
:105C6000012BF3D100231120384E394D33602B70B6
:105C700068442379374A4178136002780902114356
:105C8000827812041143C27812060A4332490A602C
:105C9000002B0ED1152169444A780B7812021A4361
:105CA0008B781B041A43CB781B0613433360002305
:105CB00018E0012B1AD1152169444A780B78120299
:105CC0001A438B781B041A43CB781A211B06134303
:105CD00033600E23627C6944934200DD130000228E
:105CE0009A422CD100220420EA54B0E7022B03D1BF
:105CF000627B10331621EEE7042B0DD1152108220B
:105D00006944684606F0DCFE0098019903F05CF9EE
:105D100006F088FD3060CAE7052BC8D1152108229E
:105D20006944684606F0CCFE0098019903F04CF9EE
:105D300006F078FD3060627D0A231E21CBE7885C87
:105D4000A8540132CCE7C046111200209412002062
:105D50009D120020280000209812002010B5134B3F
:105D600004001B78002B01D1FFF778FEFFF7CEFD72
:105D700000200F4A0F49104B5450586001301060FA
:105D800058680028FCD00020186101309060186924
:105D90000028FCD0094B0A481B785B011B185350A4
:105DA000FFF7B4FDFFF798FD10BDC04611120020AB
:105DB0000010004004050000FC10004010120020FC
:105DC0001212002010B588B000281DDD0A680121DC
:105DD00013000B4018D1042A16D90F201468204054
:105DE000092811D150683F280EDD980010188068EE
:105DF0000024084201D04010C4B26846C4540133A4
:105E0000202BF2D1FFF7AAFF002008B010BD000040
:105E100010B5002813DD0C68E30710D56410532C6F
:105E20000DD8084B1B78002B01D1FFF717FEFFF7A9
:105E30006DFDA123044ADB00D450FFF74DFD002087
:105E400010BDC046111200200010004010B50028FF
:105E50000EDD0C68E3070BD56410FF2C08D8054B4A
:105E60001B78002B01D1FFF7F9FD034A034BD450F7
:105E7000002010BD11120020001000402405000079
:105E800010B5002805DD0868C30702D54010FFF7EC
:105E90004BFE002010BD70B588B0002820DD012425
:105EA000086804401CD104281AD90F230268134043
:105EB000042B15D1FEF79CF8060007F0A7F90500A2
:105EC000122800D912252A0002210D326846FFF758
:105ED000A5FD6B465D73A54205DC6846FFF73EFFF6
:105EE000002008B070BD2300325D6B449A7301340A
:105EF000F1E7F0B50D008BB0012832DD0868012212
:105F0000040014402DD104282BD90F2301680B4025
:105F1000042B26D16B68134223D0FEF769F86E6814
:105F200007007310019307F071F905000E2800D9DE
:105F30000E252A000121113202A8FFF76FFD6A46E3
:105F4000127902AB5A7302AA73129373019B7614EF
:105F50001B0ED67313745574A54205DC02A8FFF717
:105F6000FDFE00200BB0F0BD3A5D02A963189A74E3
:105F70000134F1E730B589B0002814DD0C68E3077F
:105F800011D5102268460021FFF748FD6B466A468E
:105F900065105D73684663122D0E64149373D47399
:105FA0001574FFF7DBFE002009B030BD174B184A0F
:105FB0005968002903D000215960013191601969A5
:105FC00000291FD0002018618023DB00D35811491D
:105FD000012B18D1A923DB00D3585B420B600E497B
:105FE0000B78032B01D801330B7003200B490B787E
:105FF000013303400B700A495B015B180949535098
:106000000123936070470860FAE7C046FC10004027
:1060100000100040240000209C12002010120020DC
:10602000121200200405000010B50A4B1B78002B4B
:106030000ED0FFF76BFCA1230722074CDB00E250D8
:10604000FFF74AFC0022054B0620E250FFF76CFDEB
:1060500010BDC046111200200010004024050000B1
:1060600010B5034A1021034800F09EF810BDC04649
:10607000BCEE0000B3EE0000044A05491368C854A2
:1060800001339B059B0D13607047C046D01600205E
:10609000D012002070B5124C124A2368834202DCF1
:1060A0000023236018E0115C451C0E00FA3E012E0F
:1060B00007D8AB4211DD515D002902D028399F2954
:1060C00001D82800EAE70100151A565C6E54013128
:1060D0008B42FADC181A206070BD1170FAE7C046D6
:1060E000DC1A0020DC16002010B5FDF709FD064B78
:1060F0001A68824201D900221A601B68C31A034839
:1061000098428041404210BDC8120020204E00003D
:1061100070B5FFF711FAFF250400002801D1200017
:1061200070BD03681B142B401D2B00D10400FFF72A
:10613000F7F8F2E770B5002601250D4C0D4A2368EB
:106140001268934205D00C4AD05CFDF7D3FE0028BC
:1061500006D1002E03D0FDF7DDFC084B186070BDA2
:1061600023682E0001339B059B0D2360E5E7C046A5
:10617000D4160020D0160020D0120020CC1200200F
:1061800010B50400064B074A1B6812689B1ADB43D4
:106190009B059B0DA34200DB10BDFFF7CBFFF1E792
:1061A000D0160020D416002070B5074E33680B2B94
:1061B00008DC0C255D43054C0133285164196160EE
:1061C000A260336070BDC046D8160020402F00206A
:1061D000F0B5B7B0040007F019F8012802D8002084
:1061E00037B0F0BD23785B2BF9D1013825182B7817
:1061F0005D2BF4D101343A21200006F0EFFF061E9A
:10620000EDD0071B002FEADD210000243A0004A88E
:1062100007F014F804AB711CDC556F1AA742DEDDE1
:106220001DAD3A00280007F009F8134BEC551B6828
:1062300003950193019BA342D1DD0C2666430F4BCE
:1062400004A9F618306806F0D7FF051E05D173685B
:10625000B6680293029B9D4201DB0134EAE7306895
:10626000039906F0C9FF37000836002801D1786885
:10627000B6E70135EEE7C046D8160020402F0020D3
:1062800010B5FBF7C1F8FEF7ABFFFBF7E7F8FDF73A
:10629000C5FDFEF7ADFAFEF74BFBFFF7E1FE01F09F
:1062A000EDF801F013FD01F03FFD01F089FF10BD95
:1062B000962210B512010021034806F01DFC0022B1
:1062C000024B1A6010BDC046481C0020D8050020B3
:1062D00070B514007F22174BC000C0580D008368B2
:1062E00013401C2B01D0002070BDC3681900114061
:1062F0000429F8D101690A40192AF4D11B0A013393
:106300009B000C30C018FDF773FE037806000120D7
:10631000002BE9D0300006F079FF0023A042E2D143
:10632000A34201DB0120DFE7F15CEA5C9142DAD1B4
:106330000133F5E7A825002010B5FDF7EBFB064B70
:106340001A68824201D900221A601B68034AC31AE4
:1063500000209A42404110BDCC120020CF0700001F
:10636000064B074A1B6812689B1ADB439B059B0D73
:106370000122834200DC002210007047D01600206A
:10638000D4160020F8B505000C0016001F1E0ED113
:106390000320FFF7E5FF002808D0FA20FFF76CFE86
:1063A000E8B2FFF769FEE0B2FFF766FEF8BD501DE8
:1063B000FFF7D6FF0028F9D0FB20FFF75DFEE8B21B
:1063C000FFF75AFEE0B2FFF757FEF0B2FFF754FEB8
:1063D0003012C0B2FFF750FE3C00E31B9E42E5DDE9
:1063E0002078FFF749FE0134F7E7000070B500247C
:1063F000F0250B4B1B68A34202DCFFF759FF70BD71
:106400002B006343074A9B181A78002A05D0597855
:10641000002311201A00FFF7B5FF0134E9E7C04659
:10642000D8050020481C0020F8B507000024F025FE
:106430002B0063430C4A01349E18B74211D03178C7
:1064400000290BD00133D15C002311201A00FFF783
:1064500099FF2A000021300006F04EFB0A2CE7D1FC
:10646000F8BD024B1C60F9E7481C0020D80500204D
:10647000F0B5150001222F007A4C1740A544019079
:106480000291002F11D005AB1A706A105A70120ECB
:106490001A710522691299706D140299DD70FFF767
:1064A00071FFCF239B009D44F0BD042D2AD90F24FA
:1064B00028680440042C32D1022304AA2800137156
:1064C000FDF796FD050006F0A1FEC82302009B0023
:1064D000984200DD1A007C1C97420DD1984206D9E3
:1064E000614804AB03226149C01806F0E9FA2200B2
:1064F00005AB02990198D2E72700611E695C05ACE3
:10650000E155E8E7042D00D0A7E0032304AA043DE9
:1065100013716B425D4105AB55710222E9E7092C0D
:106520007ED1042205AB1A706A6851100091694649
:10653000521209789A70009A59701F2A01DD2022A0
:1065400000926A46127806ACDA70009BBB4202DC0D
:1065500005ABE21ACDE70126BB00EB1898680640B0
:1065600006D1042837D90F210368194002290CD11C
:10657000012323704310637042121B0E4014A2705B
:10658000E070237105340137DFE7042921D10223AC
:106590002370FDF72DFD039006F038FEA31C0C2898
:1065A00009D86070864201D19C19ECE7039A925D8C
:1065B0009A550136F6E70C226270039A925D9A555D
:1065C0000136092EF9D12E23E372237363730E343F
:1065D000D9E7012907D103230438237043425841E6
:1065E00060700234CFE7092909D10423237043687E
:1065F0005A1062705B12A370E6700434C3E703297B
:106600000BD1052323700068020992B2430F920058
:106610000B40D31A63701B12EDE726700134B2E70A
:10662000032C00D03DE7052205AB01091A7089B2A1
:10663000420F890022408A1A11125A709970642AF6
:1066400000DD64220421DA70081F824201DC04327A
:106650004FE7685C58540131F6E7002D00D020E781
:1066600053E7C046C4FCFFFF22030000BCE100006A
:1066700070B502000024F0210D4E0800604380191F
:106680004578954203D001340A2CF6D170BDF02232
:10669000002106F031FA074A1368013BA34200D1FA
:1066A0001460002329001A001120FFF76BFEEDE7AC
:1066B000481C0020D805002010B5B2B002236A465D
:1066C0000400137006F0A2FDC72800D9C7200023DC
:1066D000984207DC421C6B46FE211420FFF752FE55
:1066E00032B010BD694601335A1EA25CCA54EFE7AE
:1066F00030B5B3B00500FFF71FFE002816D0022307
:106700006A462800137006F081FD0400C72800D9EE
:10671000C7240023A3420BDB20003230FFF730FDFB
:10672000621C6B46FF211420FFF72CFE33B030BDF6
:10673000694601335A1EAA5CCA54EBE7F0B5BDB0F6
:1067400005900C00012803DC1B20FBF725F855E021
:106750002C4B08680393C30709D4042807D90F23D7
:1067600002681340042B02D1FDF742FC0390254B35
:1067700060680493C30709D4042807D90F2302686B
:106780001340042B02D1FDF733FC049000261E4B6E
:106790001B680893089BB3420BDC049B1B4A0093C5
:1067A000C821039B0AA806F0B9FC0AA8FFF7A0FFBE
:1067B000CAE70C257543164B0399ED18286806F0B7
:1067C0001BFD071E05D16B68AD680993099B9F42AD
:1067D00001DB0136DEE728680499079506F00CFD19
:1067E0000835069000280BD121000598079B083139
:1067F0005B6802389847074B069A1A603DB0F0BDB7
:106800000137E3E7F8E60000D81600201DF000008D
:10681000402F0020E40F0020F7B5234B06001B6833
:10682000F02100930023009A9A4211DC0024F02307
:106830001A006243019201991C4A55182F78002FC3
:1068400012D001340A2CF3D11948FFF751FF29E087
:106850000A005A43154882185078B04202D1127883
:10686000002A1FD10133DEE7F0223900280006F0AC
:1068700043F902230D4A0199EB6053540D4AF1008C
:106880008A58009B6E70AE70AA602F616F61A34240
:1068900002DC054B01341C60002331001A0010207B
:1068A000FFF770FDF7BDC046D8050020481C00204A
:1068B00065F40000A825002010B5FFF797FDFF2420
:1068C000084AE3005B429B18074AD35C043B012B58
:1068D00003D8E043C0B2FFF79FFF013C002CEFD18B
:1068E00010BDC046FC070000A8250020F8B5050033
:1068F0000E00FDF79DFDFF240D4B18600D4AE300CF
:106900005B429B180C4AD35C062B01D0032B0BD1A6
:10691000E743FFB2320029003800FFF7D9FC002816
:1069200002D03800FFF778FF013C002CE6D1F8BD1B
:1069300008000020FC070000A825002070B5050015
:10694000FF24084AE3005B429B18074AD35CAB4232
:1069500003D1E043C0B2FFF75FFF013C002CF0D150
:1069600070BDC046FC070000A8250020F7B5FDF764
:10697000C7F8574B1A68824201D900221A601A6878
:106980005449821A8A420DD9FF2253491860D30014
:106990005248CB1A1B181B78073B022B0CD9013A23
:1069A000002AF4D1F7BD0720FFF7C8FF4C4B27E0C2
:1069B0000820FFF7C3FF38E0FDF7ACF8071E00D151
:1069C00001270020FDF758F901900020FDF768F934
:1069D000019B0090434C444D002B12D02368002BA8
:1069E0006ED12B682760002B6ED0404B01261B78A0
:1069F000002BD8D10920FFF7A1FF394B1E703B4B6C
:106A00001E70009B002B12D02B68002B0FD1236827
:106A10002F60002B1ED0324B01261B78002BC7D1D4
:106A20000920FFF78BFF2E4B1E70304B1E70236822
:106A3000002B0FD02A4E3278002A0BD19F4200D271
:106A400027602368FB1A312B04D90720FFF776FF54
:106A5000012333702B68002B0FD0244E3278002A8C
:106A60000BD1BB4200D92F602B68FF1A312F04D9FC
:106A70000820FFF763FF012333702368002B0CD03D
:106A8000019B002B09D1164E3378002B02D1072031
:106A9000FFF754FF0023236033702B68002B00D1D5
:106AA00080E7009B002B00D07CE7104C2378002B64
:106AB00002D10820FFF742FF00232B60237071E70B
:106AC000009A002AA0D1B5E7009B002B9FD1AEE72A
:106AD000C41200200F270000A8250020FC0700009A
:106AE000B8120020B4120020BC120020C0120020F6
:106AF00013B50400FFF77AFCFEF7EDFE00230093C8
:106B0000134B1B68002B02D16846FDF79DF8042348
:106B100001A901200193FEF74DF800210800FEF7BE
:106B200003F8FEF711FAFFF77FFAFDF7CDF8FDF74E
:106B300051F9FDF76BF9FEF74DFBFDF70DF8002C51
:106B400004D0FDF701FA0348FFF7D2FD13BDC0469C
:106B5000F41A002056F40000002310B501001A00BA
:106B60001120FFF70FFC10BD07B56B461970694681
:106B70005A7013128B701314120ECB700A716B467D
:106B8000010005221320FFF7FDFB07BD10B50A0029
:106B900001001220FFF76CFC10BD70B505000C0061
:106BA000FFF7CAFB002809D020003230FFF7E8FACF
:106BB0002B00220000211B20FFF7E4FB70BD10B565
:106BC0000C000300110014202200FFF7DBFB10BDB6
:106BD000012370B5FF24084A41185B42884201D363
:106BE000D84370BD06781D0A234073409B009B5814
:106BF00001306B40F2E7C04638F0000013B50400E6
:106C0000FE2813D80A4BC200D05800280ED0436883
:106C100008309900FFF7DCFF01900920FFF7B0FA78
:106C200001AB042221001720FFF7ACFB13BDC046C7
:106C3000A8250020F8B500231800254DDA00AA5831
:106C40000133511E8A418018FF2BF7D1052444439C
:106C50000A20FFF795FAFB20FFF70EFA2720FFF72F
:106C60000BFA0020FFF708FAE0B22412FFF704FA4B
:106C7000E0B2FFF701FA174BFA21186803F0F8FDAC
:106C800000260700F300E85800281CD043680830AD
:106C90009900FFF79DFF04000520FFF771FAF0B29D
:106CA000FFF7EAF9E0B2FFF7E7F92004000EFFF77B
:106CB000E3F92002000EFFF7DFF9200EFFF7DCF901
:106CC000380001F025FF0136FF2EDBD1F8BDC046AC
:106CD000A825002004000020F7B50190FFF718FA5E
:106CE00001250400FF276D42002C01D12800FEBDC4
:106CF000266833143B40152B0DD121000198083133
:106D000006F07AFA002801D135123D402000FEF746
:106D100007FB0400E8E71D2BF8D101256D42F5E7DC
:106D2000F0B5A1B0FFF706FA8021A64CA64F206867
:106D3000C900091AC019FDF7C3F82368C0182060FC
:106D4000002811D0FCF7DCFEA04B18603B78FA2B32
:106D500000D049E12368022B08DCFFF7C5F90028C1
:106D600002D00120FFF796F921B0F0BD7B78BC7806
:106D7000981E242800D919E103F0E6FC250038000C
:106D80003C00400043004C0018015600880092006F
:106D90009900AF00EE000501180118011801180153
:106DA0001801180118011801180118011301180120
:106DB000180118011801180118011801180118010B
:106DC000180118019600FF2C0ED02000FFF750FC90
:106DD00000227F4BE100CA505B181A71210000921B
:106DE00013001320FEF714FD0320BBE72000FFF77C
:106DF00013FDF9E72000FFF73BFCF5E7FFF75CFD2B
:106E0000F2E7FFF7F3FA0020FFF772FE7148FFF791
:106E10006FFCE9E7632CE7D86F4BA200D258210042
:106E20001520FFF725FBDFE7FFF772F9FF270400C6
:106E3000002CD9D025682B143B40152B04D0200002
:106E4000FEF76EFA0400F3E72000083006F0DEF9E2
:106E500006000530FFF794F9FB20FFF70DF92D121E
:106E60001D20FFF709F9E8B2FFF706F9F0B2FFF7C6
:106E700003F93012C0B2FFF7FFF825002B1B9E422A
:106E8000DDDD287AFFF7F8F80135F7E700211D204E
:106E900000910B000A00FEF7BBFCFDF755F8A3E7D5
:106EA0002000FFF7ABFE9FE7FFF7C4FE9CE7FCF76F
:106EB0003FFE07AC494A64210090494B200006F090
:106EC0002DF902232000237006F0A0F92300020010
:106ED00000211620FFF756FA86E7424BFA21186880
:106EE00003F0C6FC00260490394AF3009B181C6886
:106EF000002C28D01B790593636808349F00B81DC7
:106F00000393FFF73DF9FB20FFF7B6F801207D1C46
:106F1000FFF7B2F8F0B2FFF7AFF8E8B22D12FFF7C3
:106F2000ABF8E8B2FFF7A8F80598FFF7A5F8E7195E
:106F3000A7420CD8FFF7FEF8049B0398584301F0D2
:106F4000E7FDFFF7F7F80136FF2ECDD14CE72078AB
:106F5000FFF792F80134EBE70024FFF747FA23002C
:106F6000220021000094DA20FEF752FCFF222100CB
:106F7000D200174805F0C0FDFCF7E6FF2100200015
:106F8000FDF7D2FD30E7012C02D1FEF7F3F92BE734
:106F9000022C02D1FEF738FC26E70120FFF7A8FDFE
:106FA00022E7002321001A001A2093E71A00C83AAA
:106FB000052A00D918E7002218001100FAF75AFA3A
:106FC00012E7C046DC1A0020DC160020C8120020A0
:106FD000A825002038F40000A02D00204FF4000068
:106FE0004AF4000004000020FB2B00D0B9E6226820
:106FF000042A00DCB1E63E79F878614B360206439C
:107000009E4200DDADE6331D9A4200DCA5E6FB5C46
:10701000FE2B00D0A5E67878BC78751E1B2869D0B9
:107020001AD807284FD0082824D0012819D1FF2CBE
:1070300010D02000FFF71CFB7D79524AB31E00924E
:1070400021002A000A20FEF7E3FB4F4BE400E0504A
:107050001B191D71701D85E61D285DD04FD31E289C
:1070600071D00300C83B052BF4D8484A2900FAF731
:1070700001FAEFE7632CEDD87A79022A13D0032ABC
:107080001BD0012AE6D1F979BB79090219433B7A71
:10709000A4001B0419437B7A1B060B435B001343BC
:1070A0003B4AA350D6E7002DD4DDB11E3548FDF78D
:1070B000BFF9374BA400E050CCE7BB79A4005A1EBF
:1070C00093419B00ECE7632DC4DC07AF2A002F49F6
:1070D000380005F0F5FC002338007B55FFF7FCFD78
:1070E0000028B7DB2A4B8000C25821001520FFF78B
:1070F000BFF9AFE729002548FFF7F8FBAAE7FF2C07
:10710000A8D07A79022AA5D81E490B200091210027
:10711000B31EFEF77DFB9DE7632D00DD6325002395
:1071200007A99D420ADCEB430022DB172B40CB185A
:107130001A70152000916B1C2100EAE7FA185279A9
:10714000CA540133EDE7022C13D0032C14D0012CC8
:1071500000D07FE7002D00DC7CE77B79002B03D09B
:107160001C00322B00DD322464235C43094B1C607D
:1071700070E7FEF7AFFB6DE7FEF7ADFB6AE7C046D1
:10718000F6030000E2160020A8250020E1160020EA
:10719000A02D0020040000200122094B1A60094A9A
:1071A0001368002BFCD00322074B1B68D817104034
:1071B000C018012380100638400018437047C046AD
:1071C00000C0004000C1004008C5004001207047D9
:1071D00010B5064C200001F007F90549200001F028
:1071E00037F90122034B1A6010BDC046181B00205E
:1071F000801A0600E01A00201FB500210E20FCF7BF
:107200009DFC01210F20FCF799FC01210D20FCF7CA
:1072100095FC1C4C200001F045F81B4B1B4A1B68D9
:1072200012681B49D2B28B420BD880239B04019376
:1072300001AB1A710199029A0023200001F04EF867
:107240001FBD14498B4202D88023DB04EFE71249AB
:107250008B4202D880231B05E9E710498B4202D8F4
:1072600080235B05E3E70E498B4202D880239B0510
:10727000DDE70C498B4202D88023DB05D7E780236A
:107280001B06D4E7F81A0020300000202C00002054
:1072900048E8010090D0030020A1070040420F0001
:1072A00080841E0000093D0010B5002815DD012472
:1072B0000B68234211D023410C4A13600C4AA042B0
:1072C00009D04B68234206D02341022B09D0032B5F
:1072D00009D0A34203D002231360002010BD002375
:1072E000FAE70323F8E71460F7E7C0463000002010
:1072F0002C00002010B500280FDD0C68E3070CD52A
:107300006410012C09DD064B1B68002B01D1FFF72F
:107310005FFF2100034801F09BF8002010BDC0462C
:10732000E01A0020181B0020F8B501250868284243
:1073300003D10D20FAF730FAF8BD4010FCF722FC1B
:10734000041E14DBFCF7F8FBA04210DB0221200036
:10735000FCF7F4FBFA222900D200200001F00AFC1D
:107360000025A84205D101002000FCF7E7FB002022
:10737000E2E700270726FA2201219200200001F00F
:10738000F9FB0028F3D0282802DD0123B3401F4376
:10739000013EF0D20E4EAF550135052DE9D1002149
:1073A0002000FCF7CBFB012206210920FCF7C2FFDD
:1073B0000028DCD00B23012443600023F25C9900F9
:1073C00052004118224301338A60052BF6D1B3E7FE
:1073D000E41A002070B500281EDD0D68EB071BD4F1
:1073E000042D19D90F242B681C40032C14D11A0921
:1073F00092B25B0F92001C40141B2E00FFF7FCFEA4
:10740000731B06489C4205DD317900F06DFF0136A3
:10741000F070F5E700F067FF002070BDF81A00205B
:107420000120704710B504680D20E30703D56410F0
:10743000FF2C03D91720FAF7AFF910BDFFF7DCFED8
:10744000E1B2044C200000F04FFF200000F04BFFA1
:107450000020F2E7F81A002070B5FFF7CDFE064DC8
:107460000021280000F040FF0400280000F03BFF4E
:1074700001206400204370BDF81A002010B5034AB3
:107480000F210348FEF790FE10BDC0467CF40000BB
:10749000F4F400000D4B70B51B6804000E001500DD
:1074A000002B01D1FFF794FEE1B2094C200001F05E
:1074B00066F8F1B2200000F063FFE9B2200000F0AE
:1074C0005FFF200001F0C6F870BDC046E01A002042
:1074D000181B002010B501240368234205D0416821
:1074E000214202D08268224203D10D20FAF754F9DA
:1074F00010BD5810802801D91520F7E74910FF2941
:1075000001D91620F2E75210FF2A01D91720EDE722
:10751000FFF7C0FF0020EBE7F7B50122140090420F
:1075200026DD0D682A4223D02D4B15411B684C687F
:10753000002B01D1FFF74CFE2A4EE9B2300001F0DA
:107540001EF827000122174014D01441FF2C02D945
:107550001720FAF721F9E1B2300000F011FF3000F6
:1075600001F078F80024A04202D02320FAF714F9A1
:107570002000FEBD042CF2D90F2523681D40092DE3
:107580001CD1636801925B100093009BBB42E6DD57
:10759000BB00E3189D68019B1D420BD06D10FF2DB1
:1075A00002D91720FAF7F8F8E9B2300000F0E8FE47
:1075B0000137EAE71720FAF7EFF8F9E7032DCED104
:1075C00027001A0992B25B0F92001D40551B3B1B0E
:1075D0009D42C4DD3979300000F0D2FE0137F6E774
:1075E000E01A0020181B0020154B70B51B68050021
:1075F0000E00002B01D1FFF7EBFD124CEDB229007C
:10760000200000F0BCFFF1B2200000F0B9FE002124
:10761000200000F0BFFF002801D0404270BD72B6CC
:1076200001222900200000F0A5FF62B6200000F032
:1076300098FE0028F2D0200000F098FEEEE7C04649
:10764000E01A0020181B002010B501240368234213
:1076500002D04168214203D10D20FAF79DF810BDF8
:107660005810802801D91520F7E74910FF2901D9C2
:107670001620F2E7FFF7B8FF40002043EFE70000D5
:1076800070B50D211D20FFF7AFFF184C5A280CD103
:1076900001222A2122703D38FFF7FCFE022001F072
:1076A00037FA0122124B1A6070BD0F211920FFF723
:1076B0009BFF332805D102238F22237020211A3803
:1076C000EAE70D211E20FFF78FFFC7280AD1032507
:1076D00000222A21A9382570FFF7DCFE2A002A2182
:1076E0001E20D9E700232370D8E7C04634000020CD
:1076F000EC1A002010B5002803DC1C20FAF74CF827
:1077000010BD01240B681C4001D10D20F6E75B1071
:10771000012B2BDD022B03D00224042B00DD0134CE
:10772000194B1B68002B01D1FFF7AAFF174B1B78E1
:107730005BB2022B1CD0032B1ED0012B11D1032CCA
:1077400000D1013C00222A211D20FFF7A3FE2200C8
:107750000E211D20FFF79EFE01222A211D20FFF78A
:1077600099FE022001F0D4F90020C9E70024D7E7F0
:10777000220123211920F2E7032C00D1013C220031
:107780000E211E20EBE7C046EC1A0020340000203A
:10779000204B10B51B680400002B01D1FFF770FFD0
:1077A0001D4B1B785BB2022B0AD0032B29D0012B77
:1077B0002CD121001D200124FFF716FF644205E0B3
:1077C000012C13D129211920FFF70EFF7F2801DD9D
:1077D0000138FF3803007F3301DA7F204042C8239D
:1077E0007F21584303F044F8604310BD032C0BD1B4
:1077F0002B211920FFF7F8FE043CE7E72D21192083
:10780000D9E721001E20D6E7052CF7D0012400205F
:107810006442E4E7EC1A00203400002010B5012097
:10782000FFF7B6FF43000120184310BD10B5032039
:10783000FFF7AEFF43000120184310BD10B505202F
:10784000FFF7A6FF43000120184310BD144B70B58D
:107850001B68002B02D10120FFF79AFF114B1B7808
:107860005BB2013301D1FFF70BFF0120FFF790FF5F
:1078700004000320FFF78CFF05000520FFF788FFB9
:107880006D43644340436419201805F001F801F08A
:10789000CBFC04F0C7FF43000120184370BDC04675
:1078A000EC1A002034000020F8B5514B05001B688D
:1078B000002B01D1FFF78CFC4E4C23787F2B00D896
:1078C00092E007210E20FFF78FFEC42833D101225A
:1078D0000E26494B10211A70484B30001A70267042
:1078E000FFF7D8FD802211213000FFF7D3FD0021E2
:1078F000615600291EDB424EC9B2300000F03FFE47
:107900003D4B3000197800F03BFD300000F0A2FE46
:1079100021780622300000F02DFEAC1D300000F072
:1079200020FD002806D0300000F020FD2870013531
:10793000A542F3D1F8BD0F211920FFF755FE3328DA
:107940000FD168222C4B1E261A7000222B4B60216F
:107950001A7030000C322670FFF79CFD0222612164
:10796000C2E700211820FFF73FFEFA281CD142226F
:10797000214B10261A700022204B4B211A70300028
:1079800001322670FFF786FD042001F0C1F838228D
:107990004C213000FFF77EFD0F2251213000FFF710
:1079A00079FD1B2252219FE70F211C20FFF71CFEAF
:1079B0003D289CD128221C2600270F4B20211A701D
:1079C0000E4B263A30001F702670FFF763FD3A0019
:1079D00022213000FFF75EFD3A0023213000FFF73F
:1079E00059FD402224217FE70021615683E7C046EC
:1079F000E01A00203500002037000020360000206B
:107A0000181B002073B5002606220021684605F0E9
:107A100073F86846FFF748FFFFF782F91A4B6A468A
:107A20009E576C466B4691781878D5785B781279BA
:107A30006479002E1FD000020902034329431BB2C0
:107A400009B2120211482243007812B240B2102843
:107A500002D15210DB10C910D8171B184340C817A9
:107A60000918414001205918D317D2185A408A18D2
:107A70005200104376BD1B022D02034329431BB263
:107A800009B22402DEE7C04636000020350000209F
:107A9000F8B501231C0098422BDD0F683B4228D02B
:107AA0004E6835001D4024D1042E22D90F223168A2
:107AB0000A40092A1DD173685C10202C00DD2024A7
:107AC000144B1B68002B01D1FFF782FB72B67F10AD
:107AD000F9B2114F2200380000F04CFD62B6A54209
:107AE00014DA380000F03DFC002804D101246D00B8
:107AF0002C432000F8BD380000F038FC0122AB0018
:107B00004000F31810439860AD18E8E764000125C1
:107B1000EEE7C046E01A0020181B002010B5054C07
:107B20002368002B02D01B20F9F736FE00202060CE
:107B300010BDC046F01A002010B5002803DC1C2040
:107B4000F9F72AFE10BD0B68DA0706D4042B04D916
:107B50000F221B681340032B01D02420F0E7034BB6
:107B600025201B68002BEBD01B20E9E7F01A002032
:107B700010B5002803DC1C20F9F70EFE10BD0B68C1
:107B8000DB0701D40D20F7E71B20F9F705FE0020E5
:107B9000F4E700001D4B70B51B680C00002B03D1EF
:107BA0002520F9F7F9FD70BD012801DC1C20F8E75C
:107BB00008680121084207D1042805D90F2302686B
:107BC0001340DD1E8D4201D92420EAE765680D428D
:107BD00001D11120E5E7042B0BD1FCF709FA05F0E0
:107BE00015FB63685B10013B01D4834208DB122064
:107BF000D7E7100980B252008000920F801AF0E798
:107C00001B20F9F7C9FD0120CDE7C046F01A00207E
:107C100010B50400802803DD2620F9F7BDFD10BD56
:107C2000002CFCDD1B20F9F7B7FDFEF79FFEFFF7E8
:107C300077F8012000F06CFFF2E7000010B5002893
:107C400005DC1C20F9F7A8FD0400200010BD184B2E
:107C50001B68002B01D12520F4E7012408680440AB
:107C60000FD04010FF2801D92820EBE71B20F9F79F
:107C700093FDFEF77BFEFFF753F8012000F048FF6D
:107C8000F4E70428E1D90F2102681140042906D144
:107C9000FCF7AEF905F0BAFAFFF7BAFFD5E703290A
:107CA000D3D1100980B2520F80000A40801AF3E746
:107CB000F01A0020044B10B51B682520002B00D0C3
:107CC0001B20F9F769FD10BDF01A002010B5034A1A
:107CD00006210348FEF768FA10BDC046A0F5000073
:107CE000D0F5000000207047012070470020704749
:107CF0000020704700207047012070470020704727
:107D00000020704700207047002070470020704717
:107D10000020704700207047002070470020704707
:107D2000704770477047000010B5034A0F210348A1
:107D3000FEF73AFA10BDC046F0F5000068F6000004
:107D40000378013B1F2B00D970470130F8E710B5CD
:107D5000FFF7F6FF0378002B0BD00130222B11D157
:107D60000378002B03D0421C222B03D11000FFF715
:107D7000E7FF10BD5C2B03D14378002B00D0821CA1
:107D80001000EDE73A2BF2D02C2BF0D07B2B0BD14F
:107D9000FFF7D6FF0378002BE9D07D2B01D101300E
:107DA000E5E7FFF7D4FFF5E720225B2B14D1FFF7BF
:107DB000C7FF0378002BDAD05D2BF0D0FFF7C7FFA9
:107DC000F7E7202BD3DD2C2BD3D0190091435D296D
:107DD000CFD0222BCDD001300378002BF1D1C6E7D4
:107DE000002210B5904216D0FFF7AAFF03780422B4
:107DF000222B10D0023A7B2B0DD0013A5B2B0AD0FC
:107E0000190030390232092905D92D2B05D14178C5
:107E1000303909290AD8100010BD0522742BFAD078
:107E20000132662BF7D001326E2BF4D0581E8341FD
:107E30005A42F0E770B5FFF783FF037801222D2B3C
:107E400001D18018023A00230A2502E06B43013079
:107E5000CB1801783039CCB2092CF7D95A4310002D
:107E600070BDF8B50C001500FFF76AFF0378222BF0
:107E700002D000232370F8BD0D236A1E21000825BF
:107E80000C260A279C4601300378222B02D10023BE
:107E90000B70F0E7002BFAD0441C5C2B0BD143781D
:107EA000841C622B0ED0662B0ED06E2B0ED0722B44
:107EB0000ED0742B0ED0002AE9DD0B70013A01318F
:107EC0002000E1E72B00F6E73300F4E73B00F2E7A0
:107ED0006346F0E70923EEE710B50400FFF737FF2C
:107EE000A04203D90378013B1F2B00D910BD0138F4
:107EF000F6E710B5002815D00378002B13D0FFF754
:107F00001FFF2021037802008B4300205D2B09D046
:107F10001000FFF71CFF03782C3B5A425341C01856
:107F2000FFF70EFF10BD1800FCE70300002070B53E
:107F30000C0081420EDD1A785B2A0BD1581CFFF72A
:107F4000FFFE0125AC4205D0FFF7D3FF002801D08A
:107F50000135F7E770BD70B50C001500002901D0A0
:107F600000230B70002820D00378002B1ED0FFF7D1
:107F7000E7FE037806002C2B03D10130FFF7E0FE6B
:107F80000600337800207D2B0FD0844204D02A00D5
:107F900021003000FFF765FF3000FFF7D8FE0378BF
:107FA0003A2B02D10130FFF7CBFE70BD1800FCE781
:107FB000F0B50D0004009DB02E78002E35D02E2196
:107FC000280005F00BF9071E14D0431B0193303E27
:107FD000092E14D82800FFF72DFF01002000FFF71D
:107FE000A4FF0400002C20D0002F1ED0019B0133E1
:107FF000ED18E1E7280005F009F90190E7E723789B
:108000007B2B11D1601C642203A9FFF7A4FF041E7F
:108010000BD0019A290003A805F0FFF80028E1D051
:108020002000FFF794FEEEE7002420001DB0F0BD15
:1080300070B5050000200C0081421DDD2800FFF70F
:10804000CFFE0300681C012B14D00020022B13D19B
:108050000022681C1100FFF77EFF012C0CD0FFF7F7
:1080600048FF00221100FFF776FF013CF5E7FFF71C
:1080700040FF013C012CFAD170BDF8B5050000208D
:108080000C0016001F0081420DDD2800FFF7A8FE3E
:1080900003000020022B06D1681C3A003100FFF7D4
:1080A0005AFF012C00D1F8BDFFF723FF3A00310041
:1080B000FFF751FF013CF4E710B50024A04218D0AF
:1080C000FFF73EFE03787B2B0AD10130002211001E
:1080D000FFF741FF00280CD0FFF739FE0134F5E728
:1080E0005B2B06D10130FFF704FF002801D00134DB
:1080F000F9E7200010BDF8B5002816DD0D68EB0784
:1081000013D56D10013D0124FDF716FA0026FF2757
:10811000644200280CD1002E21D0300005F076F802
:1081200001003000FCF784F9F8BD01256D42EAE753
:1081300003681A143A40152A0BD11B123B409C428B
:1081400000DA1C009D4201D106000836FDF7E8F870
:10815000DFE71D2AFAD1012400266442F6E7012058
:10816000013464002043DFE710B508680C00FBF71A
:108170003FFFFEF7B1FD002803DB6268024B800081
:10818000C250002010BDC046A02D002010B50868C8
:10819000FBF72EFFFEF7A0FD0123002802DB024BB8
:1081A0008000C358180010BDA02D002010B508682D
:1081B000FBF71EFFFEF790FDC043C00F800010BD0F
:1081C00010B5034A04210348FDF7EEFF10BDC04679
:1081D00004F70000FEF6000010B5FBF72BFEFBF7DE
:1081E000D9FEFEF74DF80448FEF782FAFDF702FAD1
:1081F000FEF762FB10BDC04653F7000010B5FBF759
:108200006BF910BD70B5002504AC24780573A94244
:1082100005D10A4B0A4A25210A4804F0E3FB016014
:108220000949920052589B0002715B58A400837167
:108230006358856043710223C37170BD6BF7000002
:10824000CAF7000079F7000028F80000037B002B34
:1082500004D14373837303610133037370470000D8
:108260001FB50191A02100240068C900D2B244507A
:10827000012A10D0A24209D0032A0AD0074A83500B
:10828000074B019AC250012343501FBD02221343E2
:10829000F4E70422FBE70622F9E7C0465405000094
:1082A0002405000010B50400FFF7D0FFA1222368C9
:1082B000A179D20099506179064A2000995021791C
:1082C00004329950044B19685A689B68FFF7C8FF3D
:1082D00010BDC0460C0500000C1B00201FB5FFF7A9
:1082E000BFFF05B000BD70470368074A99501A00E8
:1082F000FC32D1680029FCD0A321C90058580023C2
:10830000C0B2D3607047C0461C05000007B580228C
:10831000074BD2051A6000229A6002321A710F23AD
:108320000C3200930349023B0348FFF76BFF07BD84
:108330000C1B002000300040F81A0020F8B50500A2
:108340000E0017000024BC4208D02B68315D1B686A
:1083500028009847002801D00134F4E72000F8BD38
:10836000704710B51C3000F0AFF910BD10B51C30CF
:1083700000F09CF910BD10B51C3000F0ABF910BD39
:1083800070B5437E0D00002B01D1002070BD64301C
:10839000040000F0A8F90028F7D12000290000F01F
:1083A00076F90120F2E70000F7B50193FA230025E2
:1083B00004009B0083600B4B4560083303601C3056
:1083C0000F00160000F058F92000643000F054F956
:1083D0006B461B79276166756576A5762000A375C7
:1083E000FEBDC04608F80000012330B5A024C375C7
:1083F000837D13499B005A58437DC132114DFF3292
:10840000E40592009B005B581551CC22C133FF3329
:108410009B001D5104690C4B5204E2500522046973
:10842000243BE250837D04699B005A58A123DB0062
:10843000E250437D02699B005958044BD15030BD36
:1084400028F800000C060000240500000C050000C0
:10845000A022002310B50469D200A3500A4CA14207
:108460000FD90A4C8C425B4109495B420B40CD213C
:10847000C9045B18046907496350052103699950D1
:1084800010BDCC235B04F5E7A086010090D003006B
:10849000000098FD24050000F7B5040000200D0041
:1084A0000193824265D01600402A00D94026270059
:1084B0001C37380000F0F6F8B1232269DB00D550F4
:1084C00080220123216992008B50A27E002A03D1D1
:1084D00022691362226913600025731EAB4207D123
:1084E000019B002B04D08022022123699200995025
:1084F000012223691A622369FC33DA68002A02D157
:108500009A6A002AF9D09A6A002A0BD1DA60A3236A
:108510002269DB00D1583800C9B2013500F0B7F844
:10852000B542DAD3019B2269002B0FD11300FC3333
:108530009B6A002B0AD10133A376D3612369FC33F4
:10854000DA6C002AFCD00022DA640AE00023012160
:10855000A37651611A002369FC3399680029FCD085
:108560009A602369FC339A6A002A01D000229A6239
:10857000E8B2FEBD10B50123FFF78EFF10BD03006A
:10858000AC3310B504001970643000F08BF801238F
:10859000637610BD0023020070B5AC3243760D0047
:1085A0001178B12204000069D20081508022216933
:1085B00092008B5022690133136222699360260076
:1085C0006436300000F080F8002812D0300000F04F
:1085D0006DF81E4B2269D0502369FC331A6A002AB9
:1085E00002D19A6A002AF9D09A6A002A01D11A6245
:1085F000E5E723690122002D0DD11900FC31896ABC
:10860000002908D1DA612369FC33DA6C002AFCD036
:108610000022DA6407E05A612369FC339A68002A71
:10862000FCD000229A6000202369FC339A6A8242BF
:108630000BD098622169064A8B588B501800022B88
:1086400003D0181F431E9841033070BD1C05000065
:10865000C404000010B50121FFF79CFF10BD00000D
:1086600010B51323142202490248FFF79DFE10BDE6
:1086700000400040181B002010B5402200210400DB
:1086800004F03AFA002320002364636410BD10B59F
:108690003F24026C531C2340446C9C4201D0815403
:1086A000036410BD0023036443647047436C026C91
:1086B000934206D03F21C25C01330B40436410005B
:1086C000704701204042FBE7036C406C181A00D54C
:1086D00040307047436C026C934201D0C05C7047DD
:1086E00001204042FBE73F22036C406C0133134002
:1086F000181A43425841C0B27047000003210A488B
:1087000002680A430260094802680A430260084995
:10871000084A094B9B1A03DD043BC858D050FBDCC8
:1087200000F012F8F7F7F0FC240500405405004073
:1087300078FD00000000002070020020FEE7FEE748
:10874000FEE7FEE7FEE7FEE7014B024A1A607047CC
:10875000380000200024F4000120704710B50368A1
:108760001322DB69984710BD70470000054B026972
:10877000D1500369FC331A6A002AFCD00022012080
:108780001A6270471C050000030010B55C331A78AC
:108790001F231A401E3B19009140114AD167C22283
:1087A000042104699200A150026953600269D360F8
:1087B000A02300220169DB00CA5001230169094A94
:1087C0005B428B500169084A8B5001690C3A8B500F
:1087D000016908328B501430FFF764FF10BDC046AA
:1087E00004E100E00C0500001405000010B5143091
:1087F000FFF76AFF10BD10B51430FFF76BFF10BD17
:1088000010B51430FFF752FF10BD0000030070B523
:108810005E331A780469724BE25003005D331A78B4
:108820000469704BE250030061331C7802696E4B9F
:10883000012C00D09EE005005F352E78A225ED00CA
:108840005651020060321578A1220669D200B55057
:108850000269D4509623DB00994200D88CE096231D
:108860001B01994200D88AE096235B01994200D807
:1088700088E096239B01994200D885E0E1239B0183
:10888000994200D882E09623DB01994200D880E02B
:10889000E123DB01994200D87DE096231B02994237
:1088A00000D87AE0E1231B02994200D877E09623B2
:1088B0005B02994200D874E0E1235B02994200D840
:1088C00071E0E1239B02994200D86EE0474B994248
:1088D00000D86CE0E123DB02994200D86AE0E12293
:1088E000002312038A425B41414A5B4213408022CB
:1088F00052059B1801693F4A8B50A023042201694D
:10890000DB00CA5000210369FC33D9600369FC33E2
:108910001962012301690B6001698B60C12104693F
:10892000890062501F215C3002780A409340623116
:10893000314AFF3153500021415600293CDA0F23C0
:108940000B40083B2D4C9B089B001B190324214026
:10895000A140FC348C40DD69A5432C00C0258D402E
:1089600029002143D9611F23017819401E3B8B4008
:10897000136070BD00246CE79E23DB02BAE79D23E1
:108980001B03B7E71E4BB5E71E4BB3E7EC239B0376
:10899000B0E71D4BAEE71D4BACE71D4BAAE71D4BE7
:1089A000A8E71D4BA6E71D4BA4E71D4BA2E78023BC
:1089B000DB049FE71B4B9DE78C080F4BA400E418DA
:1089C00003230B40FF21C025DB009940AD00665911
:1089D0008E433100C0269E4033000B436351C2E7F3
:1089E0000C050000140500006C05000090D0030089
:1089F00000D0BEFE2405000000E100E000ED00E034
:108A000000B013000050270000A04E0000F07500D9
:108A100000509D0000F0EB0000903A0100E0D7010B
:108A200000B0AF0300705F07F7B5009308AB1B7889
:108A300000250193FA2304009B0083600E4B4560E0
:108A40000833036014300F001600FFF715FE2300F3
:108A50005C3327611E70009B084A9B0099582300D5
:108A60005D331970019B20009B009A5823005E33F0
:108A7000DD701A70FEBDC046ACF8000028F800009A
:108A8000036910B51A00FC32D2680400002A0AD02B
:108A9000A322D20099581430C9B2FFF7F8FD002282
:108AA0002369FC33DA6010BD10B50248FFF7E8FF18
:108AB00010BDC046D01B0020162307B5022200932C
:108AC0000249013B0248FFF7AFFF07BD002000400D
:108AD000D01B002010B5002801D004F0C9FA10BD49
:108AE0000849094A094B10B51B688858FA22190A27
:108AF0001B0618439200002301F0F2FF4904C00B4B
:108B0000084310BD0010014004050000341C002083
:108B100070B5041E09D0FFF7E3FF050000F014F85C
:108B2000FFF7DEFF401BA042F8D370BD0022044BCC
:108B30009A60044A13680133DBB213607047C04681
:108B4000FC100140341C00207047704710B500F045
:108B50005FF8FFF7FAFF0120FFF7DAFFFFF73CFBB2
:108B6000FFF74CFB024B002BFAD000E000BFF7E709
:108B700000000000F8B54C1EA1410125104B114F1B
:108B80008000C3584C4238680F499D40160001F0E0
:108B9000E5FD0A21704301F0E1FD2C4003002200B5
:108BA00029000A4800F016F8FA21094C89004443CC
:108BB000386801F0D3FD0100200001F0CFFDF8BDC1
:108BC00028F800003800002040420F001005005037
:108BD0001027000030B504680C40944206D1013BD8
:108BE000002BF8D112E0013B002B0FD004680C40A1
:108BF0009442F8D1002405680D40954204D1013417
:108C00009C42F8D1002002E0201C00E0181C30BD7E
:108C1000C420114B80001A5810491140C022120282
:108C20000A431A50C0218022490092025A501A6009
:108C30008023A3220021DB05D20099500122F930C4
:108C40009A60074BFF301950C12002318000195043
:108C5000403019501A60704700E100E0FF00FFFF4C
:108C600000100140014B18607047C046840000208E
:108C7000F7B5002320285AD8384B8000C258042A60
:108C80005BD007D8022A54D055D80423012A09D032
:108C900000234CE0062A54D051D31A2A53D0022381
:108CA0001B2AF5D12E4A116808294ED909294FD01F
:108CB0000A240226A02001252A4AC00015502A486D
:108CC0002A4D07681C20BF0007402948019700680B
:108CD0005759009027481B0207401F43C0230098A4
:108CE0009B020340FF2057515759000207401F4382
:108CF000019B1F43009B58016023184007433E43DC
:108D0000565101251C4B156058680028FCD00020E6
:108D10005860A1230125DB00D3585560A025ED0044
:108D200050511BB2A14202D015D2611ACB4018009B
:108D3000FEBD0823B6E71023B4E72023B2E74023A3
:108D4000B0E78023AEE70123ACE708240026B1E7B3
:108D50000C000126AEE7091B8B40E8E728F800006D
:108D600080000020007000403C000020040500004E
:108D700040000020FF00FFFFFC700040F0B52028FD
:108D80005BD8364B8000C258354B1E68002E30D160
:108D9000C227344BBF00D859334C03250440C020B0
:108DA00000022043D851C024802064008000185164
:108DB0002E4F18602E4B803CD859FF3CA043D85111
:108DC0000437D859A8432043D8510837D8590C350F
:108DD000A8438446072065462843D851A820C000F0
:108DE0001E50C1208026800076021E501C601C4B45
:108DF0001C60142500202B001E4C2E0046433659C3
:108E0000771C1BD14343E250A0230325C132FF321C
:108E10009200DB05D550184B1A68082A14D1142388
:108E20004343E3189A6812485132FF329200596066
:108E30001150DA68C1239B00C250F0BD9642E1D0C8
:108E400001300328D9D1F8E7082A02D9083AD140DD
:108E5000E5E708239A1A9140E1E7C04628F80000A8
:108E6000381C002000E100E0FF00FFFF04050000C7
:108E70000090004044000020840000202149F0B50B
:108E80004A6C2148002A14D0A025A12600230124E1
:108E9000ED05F600C258571C06D0C7187F68002F92
:108EA00002D027009740AF5114333C2BF2D100235E
:108EB0004B64A0230121DB0500260F009C461423F0
:108EC0004B43C3181A1F1268104C0E4D9200141910
:108ED0005219526C002A10D01A00143A1268551C0C
:108EE00009D0103B1B68FF2B05D03B009340654623
:108EF0001A00074BEA50FC34666401310429DED1C4
:108F0000F0BDC046FC9000404400002000900040AE
:108F10000C05000000B5202810D80C4A80008358AA
:108F200003290BD8A0220800C133FF33D2059B00D0
:108F300001F000FC020905070021D15000BD0C2101
:108F4000FBE70421F9E70321F7E7C04628F8000012
:108F500020280AD8074B8000C25801239340A02242
:108F6000D205002902D1044953507047A121C900FC
:108F7000FAE7C04628F800000C05000003000020B6
:108F8000202B0AD8A021A222C905D2008858034A62
:108F90009B009B58D84001231840704728F80000D8
:108FA000F7B506000D000C008B180193019B671BA1
:108FB0009C4207D0336821781B6830009847013401
:108FC0000028F3D13800FEBDF0B5C64600B5CB0F82
:108FD0009846404A4B005B0D9A1882B00D00040081
:108FE000132A2FDC002A49DB3B4F17413E000E407D
:108FF000064323D07F08390029400C430AD0374963
:10900000BD438C4663445C425C418023DB021341D8
:10901000E4071D434146CE0031492B008E19220042
:10902000346875682000290001F000FF009001916C
:109030000098019922002B0003F090F802B004BCC4
:109040009046F0BD332A08DD8023DB009A42F5D13B
:1090500002000B0001F0EAFEF0E7224A94460122EA
:1090600063445242DA400242E8D052080242D1D070
:1090700094438022D2051A411443CBE74B005B088E
:109080000343DBD00B031B0B1C43634223438024AD
:109090004D0C24031B0B23406D042B431900434646
:1090A000DA000F4B9B181C685D6802000B00200063
:1090B000290001F0BBFE0090019100980199220067
:1090C0002B0003F04BF842464B005B08D6073343B6
:1090D0001900B3E701FCFFFFFFFF0F00EEFBFFFFEE
:1090E000E0F80000EDFBFFFFF8B5274A4B005B0DF1
:1090F0009A180C000700132A10DC002A36DB234BD9
:1091000013410B423AD080242403144100206418F8
:109110009C430600250030002900F8BD332A0EDDEF
:1091200080230600DB000D009A42F4D102000B0000
:109130003800210001F07AFE06000D00EBE7144D27
:109140000600AC46012563446D42DD40AC466346F3
:109150000D000342DFD033239A1A323B9340181894
:10916000874200D94C1C63469843D2E7C90FCC070D
:109170000020531CCDD1074B1C43CAE706000D004D
:109180000028C0D1C7E7C04601FCFFFFFFFF0F006A
:10919000EDFBFFFF0000F03F30B5214A4B0087B0E8
:1091A0005B0893421EDD1F4A934205DD02000B005F
:1091B00002F0D4FF07B030BD02AA00F095F80323F7
:1091C0001840049A059B012813D002281DD00028BE
:1091D00014D00298039900F06FFB80231B069C4675
:1091E0006144E7E7002300220093002301F0DEF84A
:1091F000E0E70298039900F05FFBDBE701240298A7
:109200000399009401F0D2F8D4E70124029803995D
:10921000009401F0CBF880231B069C466144C9E70B
:10922000FB21E93FFFFFEF7FF0B54746CE4680B513
:109230008DB004000D0000F067FA294B06001B7882
:109240000F005BB29846013310D022002B002000A3
:10925000290003F0CBFA8146002807D10022002321
:109260002000290001F014FC002806D1300039004C
:109270000DB00CBC90469946F0BD01230293194BEA
:109280000694079503934B460A9343460494059529
:10929000002B15D0002300221900100002F0E2F884
:1092A000434608900991022B0ED103F0B9FB21230C
:1092B00003600A9B0193002B0CD1089E099FD5E700
:1092C000002300240893099402A801F0C1F90028A2
:1092D000EFD1EAE703F0A4FB0A9B01930360ECE7FC
:1092E00088000020F0F80000F0B54E464546DE4606
:1092F0005746E0B5E14B4C008FB090468946640874
:109300009C4200DC87E0DE4B9C4222DCDD4A0029E7
:1093100000DC92E0DC4B02F021FFDB4B06000F008B
:109320009C4200D17EE1D94AD94B02F017FF0200DE
:109330000B00414630000A604B60390002F00EFF1E
:10934000D34BD24A02F00AFF434601259860D96008
:109350006BE0D04B9C4200DC8FE0CF4B9C4200DDA9
:1093600055E1CE4A231592469A4451460905631A9F
:1093700019001D00040003F055FA03F089FA0200F9
:109380000B00200029000892099302F0E7FE00225A
:10939000C34B02F071FC0F00060003F043FA03F028
:1093A00077FA04000D0002000B00300039000A9427
:1093B0000B9502F0D3FE0022B94B02F05DFC0022B7
:1093C00000230C900D9101F05DFB002800D192E18B
:1093D000002300222000290001F054FB43424341B6
:1093E0000133B04A41460192022208A80092524637
:1093F00000F07CFB4B460500002B16DA802243462A
:109400001206944642465B68454263445360D36803
:109410006344D36009E00B00020041460A604B60E0
:109420000022002300258A60CB6028000FB03CBCDE
:1094300090469946A246AB46F0BD934B01F0F6FC30
:10944000914B06000F009C4200D13DE18F4A904BAA
:1094500001F0ECFC02000B00414630000A604B605A
:10946000390002F07BFE894A894B01F0DFFC0125BF
:1094700043466D429860D960D7E701F049F88A4ABF
:109480008A4B06000F0002F0F7FB0022884B01F028
:10949000CDFC03F0C7F9050003F0FAF9794A7A4BDD
:1094A0000490059102F0E8FB02000B003000390047
:1094B00002F054FE754A06000F0004980599744B9B
:1094C00002F0DAFB029003911F2D00DCC7E0029A44
:1094D000039B3000390002F041FE83468A46534622
:1094E0005B0024155B0DE31A102B6CDD04980599C5
:1094F000D322674B520502F0BFFB02000B00300085
:1095000039000292039302F029FE0A0001001300C1
:109510000691079202003900300002F01FFE029A05
:10952000039B02F01BFE06000F0004980599614A98
:10953000614B02F0A1FB32003B0002F00FFE069EE1
:10954000079F0B000200390030000292039302F0E3
:1095500005FE4B005B0D83468A46E41A312C32DD52
:1095600004980599B822544B920502F085FB03003C
:109570000C000200029303940B000698079902F076
:10958000EDFD02000B0006000F000698079902F09F
:10959000E5FD029A039B02F0E1FD484A0290039127
:1095A00004980599464B02F067FB029A039B02F070
:1095B000D5FD02000B00300039000292039302F047
:1095C000CDFD83468A465A465346414630000A60DE
:1095D0004B60390002F0C2FD029A039B02F0BEFD0F
:1095E00044460B000200A260E3604B46002B00DB08
:1095F0001BE75B46236080231B0653446360802384
:109600001B069C466144A060E1606D420DE70B00C3
:10961000020002F0A3FD434600259860D96018605F
:10962000596002E7D3221A4B520502F097FD214AF6
:10963000214B0D00040002F091FD02000B00414699
:1096400020000A604B60290002F088FD1A4B194A7D
:1096500002F084FD434601259860D960E5E60200EA
:109660000B003000390002F079FD6B1E154A9B009B
:109670009B5883468A46A342A5D130E7FB21E93FA8
:109680007BD9024000004054FB21F93F3163621A4C
:1096900061B4D03DFB213941FFFFEF7FEAFBFFFFC3
:1096A0000000704178F9000083C8C96D305FE43F65
:1096B0000000E03F7370032E8A19A33BC1492025A7
:1096C0009A837B39F8F80000D3220C4B520501F045
:1096D000ADFB0B4A0B4B04000D0001F0A7FB020091
:1096E0000B00414620000A604B60290002F036FD65
:1096F000034A044BB9E6032373E6C04661B4D03D88
:109700007370032E8A19A33BF8B54746CE46674BC4
:1097100080B50A000F00190005003940994200D1B8
:109720009BE004000100002F69DD3F1500D1B4E08B
:109730005F4B12039C468023120B5B0313435B00B9
:10974000CA0F67449B184A00F80703D5D20F5B0085
:109750009B188A0079108C460021802016248946A7
:1097600080030D189D4202DC29185B1B8144D50F34
:109770005B00013C5B1952004008002CF1D1002035
:109780008046802020250027000609E08B425CD01F
:10979000D40F5B00013DE31852004008002D16D0A5
:1097A000C4198B42F2DD27180E00002C49DB5B1A2E
:1097B000A242894149425B1A121BD40F5B00013D52
:1097C00080443100E31852004008002DE8D11343D3
:1097D0004ED143465B0837494A46884649465210AF
:1097E0004244C90702D5802109060B4361460F0593
:1097F000BD18180029000CBC90469946F8BD7B00A6
:109800005B0803433900002BF5D0002F3CD1E30A5D
:10981000153A6405002BFAD08020400303423FD163
:10982000002700E00F005B00791C0342FAD02500FE
:1098300020208D40401A2900D71B2200C2401A4325
:1098400076E7FE43F60F8E19B1E79442A0D82718A9
:10985000002CF6DB1E000023AEE702003B002800D0
:10986000390002F009FA2A003B0001F0DFFAC2E7F2
:109870004346013303D0434601335B08ABE7012382
:1098800098460023C144A6E73B00020002F066FCB4
:1098900002000B0001F0E6FDADE713000022BBE77C
:1098A0000127210020207F42C6E7C0460000F07F4C
:1098B00001FCFFFF0000E03FF0B54746CE4680B513
:1098C00087B000920193754B4F00814688467F0810
:1098D0009F4263DC02F0A6FF002800D1D4E04A4694
:1098E00043464846414602F0C7F904000D006C4A61
:1098F0006C4B02F0C1F96C4A6C4B01F097FA2200F4
:109900002B0002F0B9F96A4A6A4B02F027FC2200E8
:109910002B0002F0B1F9684A684B01F087FA220087
:109920002B0002F0A9F9664A664B02F017FC2200F0
:109930002B0002F0A1F9644A644B01F077FA22008F
:109940002B0002F099F9029003910022604B200055
:10995000290002F091F9029A039B06000F002000F3
:10996000290002F089F9009A019B04000D00484685
:10997000414602F081F902000B002000290002F0AC
:10998000EDFB02000B003000390002F0E7FB0200A3
:109990000B0000204F4902F0E1FB70E002000B00D9
:1099A00002F06AF904000D003D4A3E4B02F064F9F2
:1099B0003D4A3E4B01F03AFA22002B0002F05CF9DE
:1099C0003B4A3C4B02F0CAFB22002B0002F054F948
:1099D000394A3A4B01F02AFA22002B0002F04CF9E6
:1099E000374A384B02F0BAFB22002B0002F044F950
:1099F000354A364B01F01AFA2B00220002F03CF9EE
:109A0000354B029003919F429FDD344B00229F42D1
:109A10003DDC334900207B182E4916001F0002F060
:109A20009DFB049005910022294B2000290002F0A3
:109A300023F932003B0002F091FB029A039B0600DF
:109A40000F002000290002F017F9009A019B040082
:109A50000D004846414602F00FF902000B002000BD
:109A6000290002F07BFB02000B003000390002F0FD
:109A700075FB02000B000498059902F06FFB07B01C
:109A80000CBC90469946F0BD00201249F7E7154BF3
:109A9000002604920593144FC5E7C046FFFF3F3EE2
:109AA000D43888BEE9FAA8BDC4B1B4BD9EEE213E4B
:109AB000AD529C804F7E923E9015CB19A001FA3E8C
:109AC0007751C1166CC1563F4C5555555555A53F5C
:109AD0000000E03F0000F03F3233D33F0000E93F99
:109AE0000000E0FF0000E73F0000D23FF0B5DE4697
:109AF0004E4645465746E0B5DC4CA5440D91140052
:109B00001900A49A0993DA4B9200D6584D1E03907F
:109B10001821E01E0696029500F0AAFEC34301003C
:109B2000DB1719404B1C9A009B1ADB001B190B9189
:109B300005934C1B771918D4A59BA5009C463F198B
:109B400022AE6544013707E0286802F0A1FE013427
:109B500003C60435BC4208D0002CF5DA00200021F1
:109B6000013403C60435BC42F6D1069B002B01DA52
:109B700000F0FDFB069B03990133DB009A46099B2D
:109B8000DA00944600920022914672AA0492B94AE1
:109B90006144934688469AAB63449B44029B002BE6
:109BA00000DABCE15D4600260027039C4D442A688C
:109BB0006B6803CC02F060F802000B003000390043
:109BC00001F034F9083D06000F004445EFD1049B35
:109BD0004B441E605F6008239C46E144D145DDD1C3
:109BE0000EA804218446494261448C46069A93009B
:109BF0009C44614684460A910399083B63448C4621
:109C00000C93009B009263449B46009A0498D100F9
:109C100003008C46634408911E685F68002A33DDA8
:109C2000954980468C466244D300984470AB9A466E
:109C30000EAB99460022914B3000390002F01CF81F
:109C400002F0F0FD02F024FE00228D4B04000D0016
:109C500002F012F802000B003000390002F07EFA28
:109C600002F0E0FD4B4601C39946434620001A68C6
:109C70005B68290001F0DAF808235B429C46E04467
:109C800006000F00D045D5D1059B30001A003900E1
:109C9000984600F0DFFCFF2300229B0504000D0026
:109CA00001F0EAFF00F038FC0022764B01F0E4FFFF
:109CB00002000B002000290002F050FA0D00040001
:109CC00002F0B0FD814602F0E3FD02000B0020002F
:109CD000290002F043FA060040460F00002800DC8D
:109CE000EEE0009B18215A1E92000EAB9B58091AF9
:109CF0001D000D41A9448D405D1B0EAB9D501723E7
:109D00001B1A1D41002D2DDD01239C46009BE144C3
:109D1000002B00DC1CE20E9C0123002C00D0B5E0DF
:109D2000009A012A09D099000EAA54580133002C38
:109D300000D0ACE0009A9A42F5D1059B002B0EDDD5
:109D4000012B00D1A8E1022B09D1009B0EA95A1EBC
:109D500092000EAB9B5807939B029B0A8B50022DDF
:109D600000D1C1E0002300223000390000F08AFE5B
:109D7000009B002800D194E2069A591E8A4210DC0A
:109D8000414A0A9894460EAA6344944600229B00D6
:109D900063441C68043B22438342FAD1002A00D06A
:109DA000C0E0069B0EAA013B9B00D358002B00D0BD
:109DB000B3E001220C9B043B596801320029FAD020
:109DC000009B9C466244110007921A0001338B42AB
:109DD00046DC0B9863468046A59C4344A046099CFC
:109DE0009B00A1464A449844D30022AA9146049A73
:109DF00099449446089BA59A6344844661449446DA
:109E00009A468B00634400934346586802F040FD35
:109E10004B4618605960029B002B24DB4D46039C87
:109E20000026002701E0286869680CCC01F024FFB7
:109E300002000B003000390000F0F8FF083D06007A
:109E40000F005C45EFD153469E60DF6004239C46C3
:109E50000433E0449C46009BE144E2449845D3D15E
:109E6000079B0093D1E600260027ECE794FDFFFF57
:109E7000C0FA000018FEFFFFFFFFFF1F0000703E4A
:109E80000000704100002040FFFFFF3F00218022C2
:109E90005204141B0EAA5450009999420EDD0EA8CC
:109EA00084469B000EAA8900D25861446344CF487F
:109EB00000E01A68821A04C38B42FAD101243CE7FD
:109EC000059B002B06D1009B0EAA013B9B00D55899
:109ED000ED1517E70022C64B300000F0F7FD002813
:109EE00000D024E100253DE732003B000020C149BD
:109EF00002F034F906000F00002C00D132E7059A79
:109F00000020BC4900F0A6FB02000B003000390025
:109F100002F024F906000F0024E7012250E7002692
:109F2000002754E64B46059A079388468B000EA9F6
:109F3000CB58183A08950592002B0DD18C46414616
:109F4000AD4B43449B006344043B58680139183AC5
:109F50000028F9D088460592059A0020A54900F00E
:109F600079FB434604000D00002B00DA05E29E0059
:109F70000EAB9C464346DB0066449C46059370ABA3
:109F80009946049F67440097306802F081FC2200E4
:109F90002B0001F071FE002238607960974B2000A1
:109FA000290001F069FE083F04000D00043EB94598
:109FB000EAD14AAB03939B4600239A46069B42464E
:109FC000994643460132029204934B46002B00DA35
:109FD000AAE080208A4B009D9846C005894900264A
:109FE0000027002408E008239C460835E044544537
:109FF00011DC4346186859682A686B6801F03CFE1A
:10A0000002000B003000390000F010FF01340600A0
:10A010000F00A145E7DA5B46C0C39B4601239C467F
:10A02000009BE244083B0093029B9A45CDD1049BE0
:10A030009846A49B022B00DD8EE0002B37DC1FD15D
:10A04000059B00271D00039B00249C461E006544C1
:10A05000083E2A686B683800210000F0E7FE083DE2
:10A0600007000C00AE42F4D1089B002B03D08023E4
:10A070001B069C4664443A0023000D990A604B601D
:10A080000720079B18409B239B009D443CBC9046A7
:10A090009946A246AB46F0BD009B0EA95A1E9200FF
:10A0A0000EAB9B5807935B025B0A8B5057E6434607
:10A0B000002B00DA70E100200021DB004AAAD6184C
:10A0C00048AF32687368083E00F0B0FEB742F8D17E
:10A0D000089B002B00D025E10B0002004A984B9909
:10A0E0000D9C2260636002F039F8434607000C00C3
:10A0F000002B13DD01254CAEB14638002E002100A7
:10A100004C4601360CCC00F091FEA146B045F7DA82
:10A11000089B07000C00002B00D015E13A0023003B
:10A120000D998A60CB60ABE70026002773E7012317
:10A130009C46009BE1440225002B00DDEBE532004C
:10A140003B0000202B4902F009F806000F0009E649
:10A150000024F2E54AAB0393A49B032B00D08FE7C6
:10A160004346002B00DC14E1039ADB009B461300FE
:10A1700091465B441E685F68234B43440293DB00B7
:10A18000994448AB9A464B465C681B68180021000E
:10A1900032003B000090019100F048FE04000D00E9
:10A1A00002000B000098019901F0D8FF3B0032003B
:10A1B00000F03CFE4B469860D9601C605D6008234F
:10A1C0005B429C46E14426002F00CA45DBD1434652
:10A1D000012B00DCE3E0039A13005B441E685F6818
:10A1E000029BDB0099464A44904610E0FFFFFF00C7
:10A1F0000000E03F0000F03FFFFFFF3F0000703E27
:10A2000080FA0000FB21F93FFFFFFF1F98464346FD
:10A210005C681B681800210032003B00009001912F
:10A2200000F004FE04000D0002000B0000980199EC
:10A2300001F094FF32003B0000F0F8FD4346039A22
:10A240009860D9601C605D60083B26002F009A4230
:10A25000DCD14D4694460026002447460835654427
:10A260002A686B683000210000F0E0FD083D060020
:10A270000C00AF42F4D1039B4A9F5D689968D8688F
:10A28000089B002B65D08022120694460D9B6544E6
:10A29000604464441F605D609960D8601E615C61C9
:10A2A000EEE69A464B460793059B30005A4239002A
:10A2B000089500F0CFF900223A4B06000F0000F09D
:10A2C00005FC002824D0384B00223000390001F072
:10A2D000D3FC02F0A7FA52460400950002F0D8FA27
:10A2E0000022304B01F0C8FC02000B0030003900A6
:10A2F00001F034FF02F096FA0EAA50510122059B9C
:10A30000524418339046059393000EAAD45023E686
:10A310005346300039009C0002F084FA0EAB18510D
:10A32000D04619E680230D9A1B06CB1810605360A7
:10A330000B0002004A984B9901F010FF43460700BA
:10A340000C00002B00DDD5E680231B069C466444F0
:10A35000E4E62B003A000D9D2A606B600A000300C2
:10A36000AA60EB60320023002A616B6188E6099BDA
:10A37000DB00009372AB049332E4A49B022B00DD5C
:10A38000E8E6002B00DD92E600D079E60027002405
:10A390006AE6002600246EE70020002198E60026E9
:10A3A000340068E7000070410000703EF0B5CE4612
:10A3B000474680B587B000920193474A4B008146DB
:10A3C00088465B08934207DC4146484602F02AFA79
:10A3D0004146031E484666D04A46434648464146E3
:10A3E00001F04AFC04000D0002000B004846414603
:10A3F00001F042FC394A3A4B06000F0020002900C8
:10A4000001F03AFC374A384B01F0A8FE22002B003D
:10A4100001F032FC354A364B00F008FD22002B00DB
:10A4200001F02AFC334A344B01F098FE22002B0045
:10A4300001F022FC314B324A00F0F8FC0E9B0290F6
:10A440000391002B34D00098019900222D4B01F08C
:10A4500013FC029A039B049005913000390001F02F
:10A460000BFC02000B000498059901F077FE220016
:10A470002B0001F001FC009A019B01F06FFE224AC3
:10A4800004000D00214B3000390001F0F5FB020003
:10A490000B002000290000F0C9FC02000B00484618
:10A4A000414601F05BFE07B00CBC90469946F0BDFA
:10A4B00002000B002000290001F0DEFB124A134BC2
:10A4C00001F04CFE32003B0001F0D6FB4A46434609
:10A4D00000F0ACFCE7E7C046FFFF3F3E7CD5CF5A1B
:10A4E0003AD9E53DEB9C2B8AE6E55A3E7DFEB15715
:10A4F000E31DC73ED561C119A0012A3F1111813F5B
:10A50000A6F810110000E03F495555555555C53F77
:10A5100049004B0819007047474AF0B54F4691462D
:10A520004B005B0D99444646D6464A46C0B50500E9
:10A530000C000E0088460700132A27DC002A4BDB9C
:10A540003E4B13419A460B0052461340034318D02A
:10A550003B4A3C4B2800210000F068FC002200230D
:10A5600000F0AAFA002847D0002C04DA80234A46DB
:10A570005B03134198444646534600279E433800E8
:10A5800031001CBC90469946A246F0BD332A08DD36
:10A590008023DB009945F4D102000B0000F046FC5B
:10A5A000EFE7294A9446012263445242DA40924638
:10A5B0000242E6D0224A234B2800210000F036FC5C
:10A5C0000022002300F078FA002815D0002C1EDBB2
:10A5D000534646469F430FE0194A1A4B2800210074
:10A5E00000F024FC0022002300F066FA002803D0CB
:10A5F000002C04DB0027002638003100C1E764008E
:10A60000640825430027002DF6D0104EF4E74B4692
:10A61000142B0BD03422D21A012393405D19BD4272
:10A6200008D201239C462F00E044D1E7133B9C460F
:10A63000E044CDE72F00CBE701FCFFFFFFFF0F0059
:10A640009C7500883CE4377EEDFBFFFF0000F0BF07
:10A65000002070474B0070B55B0D14000A00002B02
:10A660001AD14B005B08034315D0234B002201F0A5
:10A6700003FB224B9C422DDB0A004B005B0D363B5B
:10A680001F4DE318AB422ADC002B0DDD1D4C1B05D2
:10A6900022401A43110070BD1B4DAB42F0D10200A5
:10A6A0000B0000F0C3FBF6E71D00353519DA174B38
:10A6B00002009C4209DD0B001548164900F032F8F3
:10A6C000134A144B01F0D8FAE5E70B00124813497E
:10A6D00000F028F8104A114B01F0CEFADBE7020037
:10A6E000E9E7084C363322401B05134319000022CA
:10A6F0000B4B01F0C1FACEE700005043B03CFFFF26
:10A70000FE070000FFFF0F80FF07000050C300009E
:10A710009C7500883CE4377E59F3F8C21F6EA50192
:10A720000000903C30B54A00DB0FDB0752081A43AB
:10A73000110030BD02B4714649084900095C490066
:10A740008E4402BC7047C04603B4714649084000BD
:10A750004900095A49008E4403BC7047002243084F
:10A760008B4274D303098B425FD3030A8B4244D3D9
:10A77000030B8B4228D3030C8B420DD3FF2209021B
:10A7800012BA030C8B4202D31212090265D0030BDA
:10A790008B4219D300E0090AC30B8B4201D3CB03D0
:10A7A000C01A5241830B8B4201D38B03C01A524112
:10A7B000430B8B4201D34B03C01A5241030B8B4214
:10A7C00001D30B03C01A5241C30A8B4201D3CB02FF
:10A7D000C01A5241830A8B4201D38B02C01A5241E4
:10A7E000430A8B4201D34B02C01A5241030A8B42E7
:10A7F00001D30B02C01A5241CDD2C3098B4201D3FF
:10A80000CB01C01A524183098B4201D38B01C01A7C
:10A81000524143098B4201D34B01C01A52410309F3
:10A820008B4201D30B01C01A5241C3088B4201D3A2
:10A83000CB00C01A524183088B4201D38B00C01A4F
:10A84000524143088B4201D34B00C01A5241411A76
:10A8500000D20146524110467047FFE701B5002083
:10A8600000F0F0F802BDC0460029F7D076E7704747
:10A8700003460B437FD4002243088B4274D3030961
:10A880008B425FD3030A8B4244D3030B8B4228D302
:10A89000030C8B420DD3FF22090212BA030C8B4228
:10A8A00002D31212090265D0030B8B4219D300E0C8
:10A8B000090AC30B8B4201D3CB03C01A5241830B4D
:10A8C0008B4201D38B03C01A5241430B8B4201D3FD
:10A8D0004B03C01A5241030B8B4201D30B03C01A26
:10A8E0005241C30A8B4201D3CB02C01A5241830AA0
:10A8F0008B4201D38B02C01A5241430A8B4201D3CF
:10A900004B02C01A5241030A8B4201D30B02C01AF8
:10A910005241CDD2C3098B4201D3CB01C01A52415F
:10A9200083098B4201D38B01C01A524143098B42E8
:10A9300001D34B01C01A524103098B4201D30B01D1
:10A94000C01A5241C3088B4201D3CB00C01A5241F6
:10A9500083088B4201D38B00C01A524143088B42BB
:10A9600001D34B00C01A5241411A00D20146524154
:10A97000104670475DE0CA0F00D04942031000D373
:10A980004042534000229C4603098B422DD3030AC8
:10A990008B4212D3FC22890112BA030A8B420CD3D8
:10A9A000890192118B4208D3890192118B4204D301
:10A9B00089013AD0921100E08909C3098B4201D381
:10A9C000CB01C01A524183098B4201D38B01C01ABB
:10A9D000524143098B4201D34B01C01A5241030932
:10A9E0008B4201D30B01C01A5241C3088B4201D3E1
:10A9F000CB00C01A524183088B4201D38B00C01A8E
:10AA00005241D9D243088B4201D34B00C01A524164
:10AA1000411A00D20146634652415B10104601D3F1
:10AA20004042002B00D54942704763465B1000D37B
:10AA3000404201B5002000F005F802BD0029F8D021
:10AA400016E770477047C046D0400B1C1141203AB2
:10AA500003D49C4613411843634652429340184323
:10AA60007047C0468446101C62468C46191C6346DB
:10AA700000E0C0461FB501F097F8002801D400217E
:10AA8000C8421FBD10B500F0EFFF4042013010BDBD
:10AA900010B501F089F8002801DB002010BD01206D
:10AAA00010BDC04610B501F07FF8002801DD002080
:10AAB00010BD012010BDC04610B501F011F80028EE
:10AAC00001DC002010BD012010BDC04610B501F012
:10AAD00007F8002801DA002010BD012010BDC04693
:10AAE000F0B5CE46474615042D0C2E0080B5070460
:10AAF000140C3F0C9946030C7E435D43674363434C
:10AB00007F19340CE4199C46A54203D980235B02CB
:10AB10009846C4444B4643435143250C3604654490
:10AB2000360C2404A4195B19591820000CBC90465B
:10AB30009946F0BDF0B54E4657464546DE46E0B56F
:10AB400043025B0A450083B00F1C99462D0EC60FC9
:10AB5000002D57D0FF2D24D08020DB00C0041843E7
:10AB6000002381469A469B467F3D7C027A00FB0F7C
:10AB7000640A120E984623D0FF2A4BD0E3008024AB
:10AB80000020E4047F3A1C43AD186B1C4746019338
:10AB9000534677403A000F2B48D87D499B00CB584D
:10ABA0009F46002B00D085E008339A46063B9B4623
:10ABB0007C027A00FB0FFF25640A120E9846DBD157
:10ABC000002C00D090E0524601231A439246012007
:10ABD000DBE74C4658461700022824D0032800D152
:10ABE000CFE00022002301284DD15802D205400AAF
:10ABF000FF071043384303B03CBC90469946A24639
:10AC0000AB46F0BD002B5BD104239A46033B0025E5
:10AC10009B46AAE7FF35002C60D1524602231A4317
:10AC200092460220B1E7FF220023DEE74B461B0CD1
:10AC30009C464B462604360C180461463300220C11
:10AC40006446000C43434E435043544380191A0C4E
:10AC50001218964203D9802149028C4664441B0491
:10AC60001B0C1004C01883015E1EB341800E1843F4
:10AC7000130C1B199B0103431C00230179D50123ED
:10AC800062081C401443019A7F32002A4DDD63079D
:10AC900004D00F232340042B00D00434230103D518
:10ACA0003C4B019A1C408032FE2ABCDCA3015B0AAB
:10ACB000D2B29AE70C239A46093BFF259B4654E7FC
:10ACC000180001F071FE4A46431F76259A40002382
:10ACD0006D4291462D1A9A469B4646E752460323FB
:10ACE0001A439246032050E7200001F05DFE431F07
:10ACF0002D1A9C40763D002047E780230027DB0388
:10AD0000FF2272E7424666E74C463200584662E749
:10AD100080234A46DB031A4222D01C4220D123431F
:10AD20005B025B0A4746FF225FE701239A1A1B2A50
:10AD300021DC23000199D3409E318C401A0023006E
:10AD40005C1EA34113435A0704D00F221A40042A61
:10AD500000D004335A0111D49B015B0A002244E75E
:10AD600080234A46DB0313435B025B0A3700FF2262
:10AD70003BE7019587E70022002336E70122002305
:10AD800033E78023DB0323435B025B0AFF222CE7CC
:10AD9000D0FA0000FFFFFFF770B500283DD0C317C1
:10ADA000C5185D40C40F280001F0FEFD9E22121A56
:10ADB000962A07DCD2B2082833DD083885406802BD
:10ADC000400A23E0992A0BDD052329001B1AD940EC
:10ADD00003001B339D402B005D1EAB4119430D004A
:10ADE000052801DD431F9D402B000F490B406E07D6
:10ADF00009D00F263540042D05D004335D0102D55E
:10AE00009F220B40121A9B01580AD2B24002D2056F
:10AE1000400AE4071043204370BD002400220020B4
:10AE2000F4E76802400AF1E7FFFFFFFBF0B54F4689
:10AE30004646D6460C000903C0B5490A470F5E00D6
:10AE400039431F03DB0F9C4665007B0A570F1F43E6
:10AE50006D0DE40F760DA146C000B846D200AB1BC5
:10AE600064457BD0002B5FDD002E00D0A4E03E00C7
:10AE7000164300D112E15E1E002E00D09EE1871A1B
:10AE80004346B84280410125C91A4042091A0B02C3
:10AE900000D431E149024E0A002E00D16EE13000AB
:10AEA00001F082FD0300083B1F2B00DD61E1202241
:10AEB0003900D21A9E40D1409F400E439D4200DD92
:10AEC00051E15D1B6B1C1F2B00DD7CE12021C91AA9
:10AED0003D0030008F408840DD40791E8F413100B9
:10AEE00007222843D940002507433A40002A09D0C9
:10AEF0000F233B40042B05D03B1DBB42BF417F428B
:10AF0000C9191F000B0200D426E26A1CC64B550566
:10AF10006D0D9A4200D106E1C44AFF080A4053076A
:10AF200052023B43120B8EE0002B00D0B8E06B1CAA
:10AF30005B055B0D012B00DC30E1871A4346B8420C
:10AF4000B641CB1A76429E1B330200D54CE13B0042
:10AF50003343A1D100220024002570E0002B00DC47
:10AF6000E5E0002E00D183E0AF4EB54260D08026F0
:10AF700036043743B846382B00DC3EE143461343E2
:10AF80001F007A1E97413F188742804140420918AE
:10AF90000B0200D4B0E0A44B01359D4200D1C3E0C8
:10AFA000A24A7B080A4001210F401F435108D307E2
:10AFB00007221F433A4099E79B4EB54238D080267E
:10AFC00036043743B846382B00DDDCE01F2B00DCAD
:10AFD00030E11E004746203EF740BC46202B04D0FF
:10AFE0004026F31A46469E403243170063467A1EB7
:10AFF00097411F43CCE0002B00D104E243461343AA
:10B0000000D159E14B07C00818438023C9081B032E
:10B01000194208D04546ED081D4204D14346D008E8
:10B02000590708432900420FC9007F4D1143C00052
:10B030004B07CA087C49C00803438D4268D01203FD
:10B040006D05120B6D0D002112031800130B0A0D74
:10B0500012051A43764B2D0513402B435B00E40782
:10B060005B08234319001CBC90469946A246F0BDDC
:10B070003E00164312D05E1E002E00D000E187185D
:10B080008742804141444042091801250B0233D5D3
:10B09000022585E764463300414610001D00C7E7DE
:10B0A000002D00D0DAE00C000443F3D05C1C00D18A
:10B0B0009FE15D4CA64200D12FE1DB43382B00DD40
:10B0C00066E11F2B00DD83E120240500E41A0F0058
:10B0D000DD40D940A0404346A7405B1A441EA04132
:10B0E00098462F433843171ABA4292414346524278
:10B0F000991A64463500CAE607223A40002A00D071
:10B10000F6E64B07CA084849FF083B438D4296D1F3
:10B110001900114300D19EE1802109030A43120363
:10B12000120B414D8FE71500002200238BE7002B07
:10B1300000D0C7E06B1C5F057F0D012F00DCF1E044
:10B14000394DAB4200D1B9E085180A0085428941EA
:10B150004244494251180722CF076D082F4349083E
:10B160003A401D00C2E607223049ED1A31403A400C
:10B17000BCE63E002838864000279FE6380001F0F4
:10B1800013FC20308EE6434613431F007A1E97417E
:10B19000C71BB84280414042091A78E60E003B00C6
:10B1A00006431343002D61D1002E00D0F4E0002BA4
:10B1B00000D11BE164463900100039E71A4FBB4249
:10B1C0007AD03300FFE630001F3DE840202B03D04B
:10B1D0004021CB1A9E4037437B1E9F4107220743E5
:10B1E0003A400021002589E7171A4346BA42B64182
:10B1F000591A76428E1B64464EE61F2B00DDADE0E9
:10B2000020264746F61AB740B9461700B246DF4037
:10B210004E463E4337005646B240561EB241174393
:10B220004246DA408918AEE6FF070000FFFF7FFFC5
:10B23000FFFF0F8020264746F61AB740B946170091
:10B24000B246DF404E463E4337005646B240561E99
:10B25000B24117434246DA40891A99E77F4CA64229
:10B260005BD0802424045B42214327E7002E0CD1CD
:10B27000002B00D1CBE0644639001000774DD7E6B3
:10B28000764FBB4218D0330075E6002B14D04B0725
:10B29000C00818438023C9081B03194207D0FC08C3
:10B2A0001C4204D17907D0080843E14621004C46EE
:10B2B000420FC9001143C000684DB9E61D000022CD
:10B2C0000023C0E6002D5BD10D00054300D1E2E66E
:10B2D0005D1C00D1B0E0614DAE421FD0DB43382B86
:10B2E00071DC1F2B00DD96E020250F00ED1AAF402A
:10B2F000B9460700AA46DF404D463D432F0055465C
:10B30000A840D940451EA84188440743BF1897422A
:10B3100092415142414435003AE664463500414687
:10B32000100085E60B000343002D00D063E6002BE0
:10B33000F5D04346134300D17AE68718874280410F
:10B3400007224144404209183A400B0200D4D5E696
:10B35000434B01351940C9E5380069E61E004746F0
:10B36000203EF740BC46202B04D04026F31A464628
:10B370009E403243170063467A1E97411F4302E600
:10B38000364DAE42CAD080252D045B422943A6E744
:10B390000843411E8841A6E6002B00D148E6871AE3
:10B3A0004346B842B641CB1A76429E1B33024BD578
:10B3B000171A4346BA429241591A5242891A072231
:10B3C00064463A4092E501430F00791E8F419DE7A4
:10B3D0001C000F00203CE740202B03D04024E31A40
:10B3E00099400843411E884138437CE600220024EE
:10B3F00025E6171A4346BA429241591A5242891A0F
:10B400006446350043E541461000144D10E68022A5
:10B410000024120380E61D000F00203DEF40BC46D3
:10B42000202B03D04025EB1A9940084307006346C0
:10B43000781E87411F4369E7871897429B41414423
:10B440005B42C9183500A3E53B003343CED0072249
:10B4500031003A4052E600231A00F4E5FF070000ED
:10B46000FFFF7FFFF0B55746DE464E464546E0B546
:10B47000834607000E03480085B092461C00360B39
:10B48000400DCD0F002800D19DE0954B984239D05A
:10B490008023F6001B041E43924A7B0F33439946D8
:10B4A000944603006344009300230026FF000293A8
:10B4B00023031B0B98466300E40F52465B0D019477
:10B4C00000D1B3E086498B4200D19EE04246D100D4
:10B4D000802212040A435146490F11438B46814989
:10B4E00052468C4600996344CB1A0021D200009347
:10B4F0002B0063409A460F2E00D905E17A4BB60027
:10B500009B599F465B463343994600D0B8E00223DF
:10B510000826002700900293CAE7CB463A0002991A
:10B520000195019B9A46022927D0032900D180E288
:10B53000012944D06D49009B8C4663441C00002CBB
:10B5400038DD530700D013E2D2085B46DB0109D592
:10B550005946674B19408B468021C9008C46009B99
:10B5600063441C00634B9C4207DC5B4664055F0739
:10B570005B0217431B0B620D02E000230027584AB1
:10B5800000211B031C0B0B0D1B05234314055A4AFA
:10B59000380013401C4353466400DB0764081C4317
:10B5A000210005B03CBC90469946A246AB46F0BD92
:10B5B0000122524201231B1B382B00DCADE100228B
:10B5C00000230027DCE75B46334399465ED0002E1C
:10B5D00000D18AE1300001F0E7F903000B3B1C2B9E
:10B5E00000DD7BE11D22D31A5A460100DA400839FA
:10B5F0008E4013005F46334399468F403F4B0026F1
:10B600001B1A00930023029352E7414653460B4313
:10B610003B499B468C46009B634400935B46002B52
:10B620003BD1022300221E43022161E7434613431C
:10B630009B4637D04346002B00D162E1404601F0E3
:10B64000B3F903000B3B1C2B00DD53E10200414624
:10B65000083A914088461D21CB1A5146D9400B002B
:10B6600041460B439B46534693401A00009B254995
:10B670009C46604403008C4663440093002137E7F6
:10B680000323B14600900C26029311E70023009398
:10B6900001330426002702930AE70323C3461E430F
:10B6A000032125E701331E430022012120E7002367
:10B6B0009A46802300271B03094A61E780234946F5
:10B6C0001B03194200D1E2E05946194200D0DEE0E6
:10B6D0000B431B0317001B0BA246014A50E7C04651
:10B6E000FF07000001FCFFFF10FB0000FF0300004C
:10B6F000FFFFFFFEFE070000FFFF0F800DFCFFFFB6
:10B7000001F8FFFFF3030000D94500D9CBE000D1D9
:10B71000C6E03C0048460027009B013B00935B4687
:10B72000160E1B021E431302984633041B0C994647
:10B73000310C0191FFF798F84A4642430B04210C63
:10B74000050019438A4207D98919013D8E4203D861
:10B750008A4201D9851E8919881A0199FFF784F850
:10B7600009048C464A46210464464243090C0300FE
:10B7700021438A4204D98919013B8E4200D8F1E065
:10B780002D041D43AB464346891A4246280C120439
:10B790001D0C5B46140C22001B041B0C5A43039423
:10B7A0006B434443029568431B19150CEB189C42EC
:10B7B00003D980246402A44660441C0C15041B04B5
:10B7C0002D0C20185D19814277D373D00C1AA24A30
:10B7D0007D1BAF42BF419446009B7F426344E01B08
:10B7E0001C00864200D1DBE00199FFF73DF84A4694
:10B7F00042430B04290C070019438A4207D98919CF
:10B80000013F8E4203D88A4201D9871E8919881ABE
:10B810000199FFF729F809044A46894629044D464B
:10B820004243090C030029438A4207D98919013B85
:10B830008E4203D88A4201D9831E89193F04891A8E
:10B840003A00039F1A43380013041B0C58438146E7
:10B850000298150C6F43434345434846000C844609
:10B86000DB1963449F4203D980204002844665442B
:10B8700048461F0C00041B04000C7D191818A9422F
:10B8800000D284E000D17FE001231A4357E68023F1
:10B890004A461B0313431B031B0BAA466F4A6FE662
:10B8A000BA4200D935E74B46DC0758087B081C43F1
:10B8B000FF0734E70024AF4289D247444745A441FB
:10B8C0005B466442A4196418013BA6421ED2A04202
:10B8D0006DD800D1B6E0241A9B4678E703005A469B
:10B8E000283B9A400027914688E6584601F05CF8CC
:10B8F000203072E603005246283B9A4093460022CD
:10B90000B4E6504601F050F820309AE6A642E2D163
:10B91000B845DCD9341A9B4659E71F2B65DC504CDF
:10B920000099A4465C46614408008C4011008240A6
:10B93000D940501E82410C4314435A46DA4013004A
:10B94000620709D00F222240042A05D02200141DCC
:10B950009442894149425B181A0262D501220023B0
:10B9600000270DE68A4200D80AE7831E891907E7F7
:10B970000F231340042B00D1E6E5171D9742924197
:10B9800053429B44FA08E0E5002800D1D7E571183E
:10B99000531EB14227D3A94215D358D01A0073E7DA
:10B9A000002B00DC04E6012300229B44CDE50223AA
:10B9B0004744474589415B429C46494289190C19D5
:10B9C000E344241A03E743465F0047459B41B846DA
:10B9D0005B429E19023A8919A94200D054E74045BA
:10B9E00000D051E7ABE51A00F6E71F215F46494258
:10B9F0000C1BE740202B07D01A49009B8C46634460
:10BA000018005B4683401A43501E82413A43072781
:10BA10000023174009D00F210023114014000429EE
:10BA200095D122005F075B021B0BD208174300224F
:10BA3000A6E5802359461B030B431B0317001B0B72
:10BA4000064A9DE5BD42B2D89B460024BFE680452C
:10BA5000B9D31A00C3E7C046FF030000FF07000088
:10BA60001E0400003E040000F0B54F464646D64690
:10BA70008446C0B58046194E18030F034D00000BD5
:10BA80005C0082463F0B6D0DC90F9146640DDB0FC4
:10BA90000120B5420AD0B44203D0A54201D1574596
:10BAA0000CD01CBC90469946A246F0BD66463E436B
:10BAB000F7D1AC42F5D154461443F2D10120C84528
:10BAC000EFD1994207D0002DEBD163461F433800D8
:10BAD000471EB841E5E70020E3E7C046FF07000046
:10BAE000F0B54F464646D6464D00C0B50E03C90FC9
:10BAF0008A462C491F035C008046360B6D0D91462B
:10BB00003F0B640DDB0F8D421ED08C4216D0002DF2
:10BB10001ED130438446002C01D13A4323D06246E3
:10BB2000002A1AD09A4529D05146022001390840EE
:10BB300001381CBC90469946A246F0BD390011431D
:10BB4000E5D002204042F4E73043FAD1AC420FD0B6
:10BB5000002C0FD13A43E7D00CE00122013B934384
:10BB600018000130E5E763460020002BE1D0DBE759
:10BB70003A43E6D19A45D7D1A542D5DCA54205DBAB
:10BB8000BE42D1D808D00020BE42D2D250460123B6
:10BB9000013898430130CCE7C845C5D80020C845D6
:10BBA000F4D3C6E7FF070000F0B54F464646D64639
:10BBB0004D00C0B50E03C90F8A462E491F035C0015
:10BBC0008046360B6D0D91463F0B640DDB0F8D42A9
:10BBD00018D08C4211D0002D18D130438446002C4F
:10BBE0001ED13A431CD163460020002B30D0514671
:10BBF00002200139084001382AE039001143EAD017
:10BC0000022025E03043FBD1AC4226D0002C26D1C7
:10BC10003A4324D15146022001390840013817E047
:10BC20006246002A0FD09A45E1D1A54205DBBE420B
:10BC3000DDD819D00020BE420AD250460123013877
:10BC40009843013004E00122013B93431800013086
:10BC50001CBC90469946A246F0BD3A43D0D19A45C5
:10BC6000C5D1A542C3DCE0E7C845C0D80020C8451F
:10BC7000E3D3EDE7FF070000F0B55746DE464E463A
:10BC80004546E0B5834606000F03480087B092465C
:10BC90001D003F0B400DCC0F002800D16FE0DE4BA4
:10BCA000984238D08023FF001B041F43730F3B438F
:10BCB0000193DA4B0027994600239B46F600814406
:10BCC0002B0369001B0B52469846490DED0F0029C6
:10BCD00000D185E0D04B994200D173E04346DA00B1
:10BCE00080231B0413435246CC48520F844613430F
:10BCF000524600206144D2008944210069400091ED
:10BD00008C46012149448A460F2F00D990E0C4494E
:10BD1000BF00CF59BF465B463B43019300D06AE169
:10BD200002230827002681469B46C9E73200584671
:10BD3000019B61460091022800D175E0032800D1E3
:10BD4000FEE1012800D02CE1002300270026002579
:10BD50003F032A0D3F0BB34812053A4302401B052F
:10BD60001343009A5B00D1075B080B4330001900B6
:10BD700007B03CBC90469946A246AB46F0BD5B4638
:10BD80003B43019300D12FE1002F00D1A5E1380002
:10BD900000F00AFE03000B3B1C2B00DD96E11D2288
:10BDA000D31A5A460100DA405E4608398F40130024
:10BDB0008E403B4301939C4B00271B1A994600235E
:10BDC0009B467DE7414653460B4393498C46E144ED
:10BDD000002B00D01AE102220220174300228CE738
:10BDE000134300D10DE14346002B00D181E14046D1
:10BDF00000F0DAFD02000B3A1C2A00DD72E10100BE
:10BE0000434608398B4098461D239A1A5346D3401F
:10BE10001A004346134352468A404946081A82494B
:10BE200089468144002068E77B4B002700268EE787
:10BE3000140C1204120C1100370C3604350C794323
:10BE400028008C462E006043604483465643210000
:10BE5000300C80465846794340440291844506D9C7
:10BE60008846802149028C46E044414602913604CE
:10BE7000010C360C00048B4681191E0C1B041B0C94
:10BE80000391190079438C46280075436544A84600
:10BE90005843050C45447743A94203D98021490200
:10BEA0008C466744290C8C4639000004000C2D0494
:10BEB0002D186144AB4405915946049101990F0432
:10BEC0003F0C080C390051434243904602008C4617
:10BED000090C8B4662437C4344445C44A04503D92F
:10BEE0008021490288464244210C88466146090463
:10BEF000090C8C4639005943434370437E430F0C71
:10BF0000F6182404BE19644442448C46B34203D953
:10BF100080235B0298464044029B61469846049BFE
:10BF2000370443449B46AB45AD416B420D04059934
:10BF30002D0C8C467F196744FD18A8465D462D19C7
:10BF4000A542A44193466442A446C344DC448F42C4
:10BF5000BF4198459B4193459241A445A4415B4212
:10BF60007F421F43360C52426442BF192243BF181E
:10BF7000624638184302D20D039913436A020A43FA
:10BF8000501E82416146ED0D2A434E023243D901D3
:10BF900000D4B3E00126500832400243DE073243AA
:10BFA0005B08224C5444002C62DD510709D00F205D
:10BFB0001040042805D0101D9042924152429B1817
:10BFC0000200D90104D580241948E40003405444F8
:10BFD0001848844200DD27E75E075B02D2081F0B8A
:10BFE000630516435B0DB2E600239946013304272F
:10BFF00000269B4664E60323019781460C279B4657
:10C000005EE6012201201743002276E60323032087
:10C010001F43434671E6C046FF07000001FCFFFFD7
:10C0200050FB0000FFFF0F800DFCFFFFFF0300002F
:10C03000FFFFFFFEFE0700000023802700933F0361
:10C040000026434B83E6019B3200A446584670E627
:10C05000AC466EE6802701993F0339422DD03B4222
:10C060002BD11F433F033F0B00951600384B6EE664
:10C0700001252D1B382D00DD66E61F2D40DC3548DF
:10C080001C005044160082408440EE40501E824105
:10C0900034431443EB40620709D00F222240042AA4
:10C0A00005D02200141D9442804140421B181A0200
:10C0B0003ED501230027002649E68027019B3F0348
:10C0C0001F433F033F0B0094214B40E603005A46B9
:10C0D000283B9A40002601926DE6584600F064FC29
:10C0E000203057E603005246283B9A4013000022B6
:10C0F00093E6504600F058FC20307BE6CA4650E7F5
:10C100001F201E004042041BE640202D03D0124C8D
:10C110005444A3401A43501E82413243072600274D
:10C12000164009D00F200023104014000428B9D174
:10C1300022005E075B021F0BD2081643002306E6AF
:10C1400080273F031F433F033F0B1600004BFEE5D4
:10C15000FF0700001E0400003E040000F8B557462B
:10C160004E464546DE460C000903E0B5490A460F37
:10C170005F0031431E03DB0F760A9B46530F3343A8
:10C18000C84E6500C000E40FD2006D0DA246814686
:10C190007F0D9C469046B74200D1B9E05B46012630
:10C1A00073409B46EE1BA34500D183E0002E63DD68
:10C1B000002F00D0B1E06346134300D123E1731E8A
:10C1C000002B00D0BAE1861A6346B04280410125B7
:10C1D000C91A4042091A0B0200D447E149024B0A2E
:10C1E00098464346002B00D189E1404600F0DCFB35
:10C1F0000300083B1F2B00DD7CE120223000D21A17
:10C200004146D040994002009E400A439D4200DDD5
:10C210006AE15D1B6B1C1F2B00DD94E120211000E7
:10C220003500C91A8E40DA408840DD40711E8E41CB
:10C23000110007222843002506433240002A09D076
:10C240000F233340042B05D0331DB342B641764251
:10C2500089191E000B0200D43DE26A1C914B550562
:10C260006D0D9A4200D119E18F4AF6080A4057072E
:10C2700052023743120B9BE0002E00D0C5E06E1C2B
:10C280007605760D012E00DC48E16746861ACB1B49
:10C29000B042BF417F42B8461F004346FF1A3B00F1
:10C2A000B8461B0200D55FE137439AD10022002433
:10C2B000002579E0002E00DCFAE0002F00D18DE0AF
:10C2C000784B9D4267D0802367461B041F43BC46C2
:10C2D000382E00DC52E1634613435A1E93411E1868
:10C2E00086428041404209180B0200D4BEE06D4BEB
:10C2F00001359D4200D1D2E06B4A73080A4001210A
:10C300000E401E435108D30707221E43324095E7D3
:10C310001E00164300D045E740E7624B9D423AD0ED
:10C32000802367461B041F43BC46382E00DDEBE02C
:10C330001F2E00DC3AE133006746203BDF403B0024
:10C34000202E05D04027BF1B6646BE403243904694
:10C350004646721E96413343DAE0002B00D114E2C8
:10C360006346134300D168E180234E07C008C90823
:10C370001B030643194208D06046C008184204D186
:10C3800063460100D2085E071643F3009946C900D0
:10C39000720F444D11434B46DE08424B4F07374363
:10C3A000CA089D4200D16EE012036D05120B6D0D9F
:10C3B00000211203130B0A0D12051A433B4B2D05E6
:10C3C00013402B435B00E4075B082343380019004C
:10C3D0003CBC90469946A246AB46F8BD6346134323
:10C3E00011D0731E002B00D007E1861886428041D1
:10C3F00061444042091801250B0237D502257BE72D
:10C400003E00614691463500C5E75C46002D00D0F0
:10C41000E1E00B000343F3D0731C00D1ACE1214BEE
:10C420009F4200D13AE1F343382B00DD6FE11F2B2F
:10C4300000DD8CE120250E00ED1AAE40B04606006E
:10C44000AA46DE40454635432E005546D940A84011
:10C450006346451EA8415B1A9C463043161AB242F9
:10C46000924163465242991A3D00B4E60722324097
:10C47000002A00D0E4E60B4BF6084F073743CA0802
:10C480009D4200D090E73B00134300D1A6E18023FA
:10C490001B031A431203120B024D89E715000022F9
:10C4A000002785E7FF070000FFFF7FFFFFFF0F80EA
:10C4B000002E00D0C7E06B1C5E05760D012E00DC5F
:10C4C000F0E0C84DAB4200D1B9E085180A008542C2
:10C4D00089416244494251180722CE076D082E4314
:10C4E000490832401D00A9E6BF49ED1A1140072254
:10C4F0003240A3E6320028388240002686E630002B
:10C5000000F052FA203073E6634613435A1E9341FB
:10C51000C61AB04280414042091A5CE60E006746E6
:10C5200006431743002D5ED1002E00D0F3E0002F0C
:10C5300000D11EE15C46614691462CE7A94FBE4200
:10C540007BD01E00F1E610001F3DE840202B03D0F9
:10C550004021CB1A9A401643731E9E410722064380
:10C5600032400021002583E7161A6346B24280411B
:10C57000591A40420B1A98465C4632E61F2E00DDDF
:10C58000ABE02027BB1B9A4663465746BB40994603
:10C5900013004F46F3401F433B005746BA40571E17
:10C5A000BA4113436246F240891898E62027BB1B24
:10C5B0009A4663465746BB40994613004F46F340A0
:10C5C0001F433B005746BA40571EBA4113436246C9
:10C5D000F240891A9CE7834B9F425FD080252D044F
:10C5E0007342294320E7002E0CD1002F00D1D0E068
:10C5F0005C46614691467B4DCDE67A4FBE421CD0EB
:10C600001E0065E6002F18D0C0084E0706438020A4
:10C61000C9080003014208D06346DC08044204D183
:10C620002100DA46D2085E071643F300994601243A
:10C630005346C900720F11431C406A4DABE61D0002
:10C6400000220027B4E6002D59D10B00034300D18E
:10C65000D6E6731C00D1B2E0624B9F421ED0F3437A
:10C66000382B6FDC1F2B00DD97E020250E00ED1A24
:10C67000AE40B0460600AA46DE40454635432E0091
:10C680005546A840D940451EA8418C440643B618DB
:10C6900096429241514261443D0025E63D0061468B
:10C6A000914678E60B000343002D00D055E6002BA1
:10C6B000F5D06346134300D16DE68618864280416B
:10C6C00061444042091800220B0200D4D0E6464BD8
:10C6D00001351940B2E5B1465DE633006746203BBF
:10C6E000DF403B00202E05D04027BF1B6646BE40E2
:10C6F000324390464646721E96413343EFE5394B2E
:10C700009F42CBD080252D0473422943A8E70843DC
:10C71000411E8841A2E6002F00D13CE66346861AFE
:10C72000CF1AB0429B415B42FB1A98461B024ED582
:10C73000161A6346B2429241591A5242891A5C460D
:10C7400000227BE501430E00711E8E419FE71D0014
:10C750000E00203DEE40B046202B04D04025EB1AC1
:10C7600099400843814648464346411E8841184344
:10C7700074E60022002417E6161A6346B24292417C
:10C78000591A5242891A3D0025E561469146154DD8
:10C7900001E680220024120379E61D000E00203DF0
:10C7A000EE40B046202B04D04025EB1A99400843B8
:10C7B00081464E464346711E8E411E4367E78618EA
:10C7C00096429B4161445B42C9183D008CE5474657
:10C7D0003743CED007224146324049E600273A008F
:10C7E000E6E5C046FF070000FFFF7FFF70B50C4E77
:10C7F0000D031C0349005B002D0B490D240B5B0D41
:10C80000B14208D0064900208B4203D114432000D6
:10C81000441EA04170BD05430120002DFAD1F1E76F
:10C82000FF07000030B5144D0A034B00120B5B0DDF
:10C83000C90F0024AB4211DD104CA34210DC802450
:10C84000640322430E4CE41A1F2C0CDD0D48C31A5E
:10C85000DA4013005C42002900D11C00200030BDEA
:10C86000094BCC18FAE7094DE040AC4663449A40C6
:10C8700013000343EEE7C046FE0300001D04000062
:10C880003304000013040000FFFFFF7FEDFBFFFFF8
:10C8900070B500282DD0C317C5185D40C40F2800FF
:10C8A00000F082F8154B1B1A5B055B0D0A2815DD9D
:10C8B0000B38854000222D032D0B002110002D0385
:10C8C0000A0D2D0B12052A430D4D1B052A4013435B
:10C8D0005B00E4075B082343190070BD02002900D8
:10C8E000153291400A000B21081AC5402D032D0B6B
:10C8F000E3E70024002300250022DEE71E040000F9
:10C90000FFFF0F804100090E4B1C70B5DBB24602E1
:10C91000750AC40F012B14DDE0239B006D07360B55
:10C92000CB1800210A0D280012051C4D32435B056F
:10C930002A405B0813435B00E4075B0823431900AC
:10C9400070BD002914D1002D1ED0280000F02CF855
:10C950000A281CDC0B232A001B1ADA4003001533BB
:10C960009D400F4B12031B1A5B05160B5B0DD8E79E
:10C97000002D06D0320B802636036D071643094B77
:10C98000CFE7084B0026CCE700230026C9E70300C9
:10C990002A000B3B9A400025E3E7C046FFFF0F80CB
:10C9A00089030000FF0700001C2101231B0498429B
:10C9B00001D3000C10391B0A984201D3000A083930
:10C9C0001B09984201D30009043902A2105C4018E7
:10C9D0007047C0460403020201010101000000008B
:10C9E0000000000030B51C00094B05001B6885B035
:10C9F000D868084B002A01D1074B1A000292019314
:10CA000000912B002200054900F026F800F0A6FD59
:10CA10008C00002090FB0000F8E600009DFB000069
:10CA2000014B18687047C0468C000020084B10B5B9
:10CA30000400002B02D0002100E000BF054B186865
:10CA4000836A002B00D09847200001F05DFBC046B0
:10CA500000000000CCFB00000EB403B5010003ABE6
:10CA6000044804CB0068019300F076F802B008BCDB
:10CA700003B018478C00002070B500260C4D0D4CFB
:10CA8000641BA410A64209D1002601F03FFB0A4D09
:10CA90000A4C641BA410A64205D170BDB300EB582C
:10CAA00098470136EEE7B300EB5898470136F2E7B6
:10CAB0005C0200205C0200205C0200206C0200206E
:10CAC000002310B59A4200D110BDCC5CC454013390
:10CAD000F8E710B5884202D98B18984203D3002397
:10CAE00007E08B5C8354013AFBD210BDCC5CC4548C
:10CAF00001339A42FAD1F8E703001218934200D1A9
:10CB0000704719700133F9E7936810B5013B9360E2
:10CB1000002B04DA9469A34207DB0A2905D01368C5
:10CB2000581C10601970080010BD00F04BFC01008B
:10CB3000F9E7F8B506000F001400D518AC4201D192
:10CB4000002007E021783A003000FFF7DDFF0134D4
:10CB5000431CF3D1F8BD0000F0B59FB002900F0068
:10CB600016000593002805D083690493002B01D19A
:10CB700000F0F4FD7B4B9F425BD1029B5F68BB8959
:10CB80001B0762D53B69002B5FD0002306AC6361B5
:10CB9000203363761033A37635002B78002B01D039
:10CBA000252B5CD1AB1B04930CD0320039000298CA
:10CBB000FFF7BFFF431C00D1C4E06269049B9446A9
:10CBC000634463612B78002B00D1BBE0012200237A
:10CBD0005242626002A9543252186E1C2360E36014
:10CBE000A3601370A365317805225F4800F0D4FE7E
:10CBF000751C002835D12268D30604D5532302A919
:10CC00005B1820211970130704D5532302A95B1860
:10CC10002B21197033782A2B2CD0350000210A20C3
:10CC2000E3682A786E1C303A092A64D900292ED08C
:10CC300026E04E4B9F4202D1029B9F689FE74C4BE0
:10CC40009F429CD1029BDF6899E73900029800F06F
:10CC50000FFC002899D0012040421FB0F0BD0135E3
:10CC60009BE7414B2268C01A012383401343236092
:10CC70002E00B8E7059B191D1B680591002B01DBF1
:10CC8000099304E05B42E3600223134323602B78A3
:10CC90002E2B0AD16B782A2B35D1059B02351A1D14
:10CCA0001B680592002B2BDB0793324E2978032259
:10CCB000300000F071FE002806D04023801B834026
:10CCC0002268013513432360297806222A486E1C06
:10CCD000217600F061FE00283AD0284B002B25D1A8
:10CCE0000722059B07339343083305936369039A2F
:10CCF0009B18636150E7434301219B18350090E77F
:10CD000001235B42D0E700230A201A00013563604B
:10CD100029786E1C3039092903D9002BC5D0079218
:10CD2000C3E74243012352183500F1E705AB0093F6
:10CD30003A00134B2100029800E000BF0390039BD0
:10CD40000133D3D1BB895B0600D584E70B9884E718
:10CD500005AB00933A000A4B2100029800F080F8DE
:10CD6000ECE7C04624FC0000D0FB000044FC0000BF
:10CD700004FC0000D6FB0000DAFB0000000000000D
:10CD800033CB0000F7B5150001938A680B6900905A
:10CD90000C00934200DA130022002B604332127819
:10CDA000002A01D001332B6023689B0602D52B6833
:10CDB00002332B60062723681F4027D0230043330C
:10CDC0001B785A1E93412268920630D422000199A2
:10CDD00043320098089EB047431C25D006232068A4
:10CDE0002A68E16803400025042B03D18D1AEB4328
:10CDF000DB171D40A3682269934201DD9B1AED18E1
:10CE00000027BD4220D1002010E00137E3682A68E6
:10CE10009B1ABB42D2DD22000123193201990098EE
:10CE2000089EB047431CF0D101204042FEBD302097
:10CE3000E1184331087021005A1C45310978A218C5
:10CE4000433202331170C1E7220001231A320199E3
:10CE50000098089EB047431CE6D00137D1E7000098
:10CE6000F0B589B004920A00433205930390029210
:10CE70000A7E0C000E9B6E2A00D186E01FD8632A22
:10CE800033D008D8002A00D18CE0582A4DD0250094
:10CE900042352A7030E0642A01D0692AF7D1196836
:10CEA00025680A1D280629D508681A60002803DAB3
:10CEB0002D23029A404213706B4E0A274FE0732ACB
:10CEC00074D008D86F2A1FD0702AE0D120220968B8
:10CED0000A43226003E0752A16D0782AD7D12200AF
:10CEE000782145321170614E22E025001A684235E2
:10CEF000111D196013682B70012365E008681A6022
:10CF00006906D3D500B2D1E719682568081D1860F5
:10CF100008682E0605D5544E08276F2A1BD00A270D
:10CF200019E06D06F7D580B2F5E745314E4E0A702F
:10CF300018682268011D00681960150621D5D307FD
:10CF400002D520231A4322601027002803D1202372
:10CF500022689A4322602300002243331A706368D8
:10CF6000A360002B58DB0422216891432160002834
:10CF700054D1029D002B5AD02500337842352B70B6
:10CF800055E05506DBD580B2D9E71A680D68101D4B
:10CF90004969186013682E0601D5196002E06D0614
:10CFA000FBD519800023029D23614FE01A68111DF3
:10CFB0001960156800216268280000F0EDFC002867
:10CFC00001D0401B6060636823610023029A1370E4
:10CFD0003CE023692A0004990398059DA847431C57
:10CFE0003ED023689B0715D4079BE068984239DA46
:10CFF000180037E022000123193204990398059E96
:10D00000B047431C2CD00135E368079A9B1AAB420A
:10D01000F0DCE9E70025F7E70028ADD0029D3900F4
:10D02000FDF722FC735C013D2B700028F7D1082F1F
:10D0300009D12368DB0706D563682269934202DCC5
:10D040003023013D2B70029B5B1B2361059B07AACC
:10D0500000932100049B0398FFF794FE431CB8D172
:10D060000120404209B0F0BDE1FB0000F2FB0000EE
:10D070000D4B70B51C680500A36B002B0FD1182059
:10D0800000F06EFC094BA0630360094B0122436072
:10D09000084B83600B2383810023026143610022DC
:10D0A000A36B1D615A6170BD8C0000200E33CDABA7
:10D0B00034126DE6ECDE0500124B10B51C68A36B54
:10D0C000002B0FD1182000F04BFC0F4BA063036026
:10D0D0000E4B012243600E4B83600B2383810023A0
:10D0E00002614361A46B0B4A206961690A4BFDF739
:10D0F000F7FC01220023801859412061616148003A
:10D10000400810BD8C0000200E33CDAB34126DE60C
:10D11000ECDE05002D7F954C2DF451580CB430B544
:10D12000164B9DB00C1E1D6808DA8B2301202B6066
:10D1300040421DB030BC08BC02B01847822302A98F
:10D140009B008B810023029008619C4200D0631EEB
:10D150008B604B6101235B42CB81209A21AB28007D
:10D16000019300F055FD431C01DA8B232B60002C4A
:10D17000DFD00023029A1370DBE7C0468C0000204A
:10D180000EB400B50B499CB01DAB02900690079100
:10D1900004910948094904CB0591006802A901934B
:10D1A00000F036FD0023029A13701CB008BC03B0D7
:10D1B0001847C046FFFFFF7F8C0000200802FFFFDA
:10D1C000020010B51378541C002B05D1CC5CD4544C
:10D1D0000133002CFAD110BD2200F3E7C9B2037865
:10D1E000002B04D08B4200D170470130F7E74B424F
:10D1F000594149420840F7E702780B78002A03D0EA
:10D20000013001319A42F7D0D01A70470023C25C36
:10D210000133002AFBD1581E7047002330B59A42D3
:10D220000AD0013AC45CCD5CAC4204D1934202D036
:10D230000133002CF6D1631B180030BD30B505005A
:10D24000002A00D130BD0C78013A6B1C2C700131E2
:10D25000002C05D19A189A42F4D01C700133FAE7D9
:10D260001D00EDE710B50378002B0FD10B785A4263
:10D2700053415B42184010BD0023CA5C002AFAD01B
:10D28000C45C944201D10133F7E701300378002BED
:10D29000F2D11800EFE70000F0B51F000E0087B0D4
:10D2A0000590019102920C98347800F0EAFA082275
:10D2B00000194378751C134036D12D2C36D1B51C7E
:10D2C00074780126002F62D0102F09D1302C07D19D
:10D2D00020222B789343582B54D110276C78023599
:10D2E0002D4B3900F31818000393FDF7BDFA049194
:10D2F00001210023494202008C46180021003039E8
:10D3000009291AD80C00A74223DD591C09D063460D
:10D31000824206D302D10499A14202DB0123784361
:10D3200020182C780135E9E72E00BCE72B2C01D022
:10D330001E00C7E7B51C7478FAE7210041391929A6
:10D3400001D8373CDFE721006139192901D8573C62
:10D35000D9E75A1C08D1059A23331360029B03981E
:10D36000002B09D107B0F0BD002E00D04042029A38
:10D37000002AF7D0002B01D06B1E0193029B019A6B
:10D380001A60EFE73024002FAAD10827A8E7302C35
:10D390009ED00A27A4E7C046FFFFFF7F37B51300E2
:10D3A000064A05001068046A002C00D1044C0A00EB
:10D3B00000942900FFF770FF3EBDC0468C0000209E
:10D3C000F0000020F8B505000E001400002804D07D
:10D3D0008369002B01D100F0C1F9224B9C422DD171
:10D3E0006C68A369A360A3891B0731D52369002B4F
:10D3F0002ED023682269F7B2981A6369F6B2834285
:10D4000005DC2100280000F03BF9002826D1A368A4
:10D410000130013BA36023685A1C22601F706369BE
:10D42000834204D0A389DB071AD50A2E18D1210024
:10D43000280000F025F9002812D00FE00A4B9C428A
:10D4400001D1AC68CDE7094B9C42CAD1EC68C8E772
:10D450002100280000F00CF80028CAD001267642EE
:10D460003000F8BD24FC000044FC000004FC000077
:10D47000364B70B51D6806000C00002D05D0AB6959
:10D48000002B02D1280000F069F9314B9C420FD1EA
:10D490006C680C23E25E93B219072DD4D90611D41F
:10D4A00009230120336037331343A381404270BD09
:10D4B000284B9C4201D1AC68EBE7274B9C42E8D15A
:10D4C000EC68E6E75B0713D5616B002908D0230001
:10D4D0004433994202D0300000F06AFA00236363BB
:10D4E0002422A3899343A3810023636023692360DB
:10D4F0000823A2891343A3812369002B0BD1A02108
:10D500008022A389890092000B40934203D021001E
:10D51000300000F0E1F90123A289134011D000236B
:10D52000A36063695B42A361002023698342BED18B
:10D530000C23E25E1306BAD540231343A3810138BE
:10D54000B5E7920700D46369A360EDE78C00002083
:10D5500024FC000044FC000004FC000010B5062080
:10D5600000F090FC012000F0CFFD0000F7B58A89A3
:10D5700005000C00130760D44B68002B04DC0B6C17
:10D58000002B01DC0020FEBDE76A002FFAD000234B
:10D590002E682B6080235B01216A1A4034D0606DB5
:10D5A000A3895B0706D56368C01A636B002B01D0A3
:10D5B000236CC01A0200216A00232800E76AB847DA
:10D5C000A189431C06D12B681D2B30D82B4ADA4089
:10D5D000D3072CD50023636023692360CB0405D5D2
:10D5E000431C02D12B68002B00D16065616B2E605B
:10D5F0000029C7D023004433994202D0280000F00C
:10D60000D7F900206063BEE701232800B847431C18
:10D61000C6D12B68002BC3D01D2B01D0162B01D1F6
:10D620002E60AFE74023A2891343A381ABE74023D9
:10D630000B430120A3814042A5E70F69002FA1D031
:10D640000B680F60DB1B01930023920700D14B692D
:10D65000A360019B002B00DC94E7019B3A00216A48
:10D660002800A66AB047002803DC4023A2891343A0
:10D67000DFE7019B3F181B1A0193EAE701004020F6
:10D680000B6970B505000C00002B01D1002070BDA6
:10D69000002804D08369002B01D100F05FF80B4B08
:10D6A0009C4209D16C680C22A35E002BEED02100B5
:10D6B0002800FFF75BFFEAE7054B9C4201D1AC680D
:10D6C000F1E7044B9C42EED1EC68ECE724FC00004F
:10D6D00044FC000004FC0000002310B504000360BB
:10D6E0004360836081814366C281036143618361DA
:10D6F000190008225C30FFF7FFF9054B24626362D2
:10D70000044BA362044BE362044B236310BDC04689
:10D71000C5DE0000EDDE000025DF000051DF000067
:10D7200010B5024900F08CF810BDC04681D600004B
:10D7300070B568254A1E55430E002900743100F06B
:10D7400081F9041E08D000212A00016046600C30D7
:10D75000A0606832FFF7D0F9200070BD836913B56F
:10D760000400002B28D18364C3640365134B144A5F
:10D770001B6882620193984201D1012383612000DA
:10D7800000F020F86060200000F01CF8A06020008D
:10D7900000F018F80022E06004216068FFF79CFFA9
:10D7A00001220921A068FFF797FF02221221E068F9
:10D7B000FFF792FF0123A36113BDC046CCFB00001D
:10D7C00021D70000F8B51C4B07001E68B369002B79
:10D7D00002D13000FFF7C2FF4836B4687368013BDE
:10D7E00004D53368002B07D03668F6E70C22A55E17
:10D7F000002D0DD06834F2E704213800FFF798FFC0
:10D8000030600028F0D10C2304003B602000F8BDFC
:10D8100020000A4B656625606560A560E3602561B0
:10D820006561A561082229005C30FFF765F9656331
:10D83000A563A564E564E9E7CCFB00000100FFFFF8
:10D84000F7B504000700002601914834002C01D1EF
:10D850003000FEBD6368A5680093009B013B009308
:10D8600001D52468F2E7AB89012B08D90E22AB5E03
:10D87000013304D029003800019B984706436835DE
:10D88000EBE7EC300068704770B50E001D000E230A
:10D89000C95E96B01400002907DA00232B60B38913
:10D8A0001B0611D48023DB000FE06A4600F088FBE2
:10D8B0000028F2DBF022019B12021340054A9B185C
:10D8C0005A4253412B60EDE740230020236016B0FD
:10D8D00070BDC04600E0FFFFF7B502268B8905004A
:10D8E0000C00334206D02300473323602361012319
:10D8F0006361F7BD01AB6A46FFF7C6FF00990700F9
:10D90000280000F09FF8002808D10C22A35E9A0599
:10D91000EFD4032293431E43A681E4E70F4BAB628F
:10D920008023A28920601343A381009B206163614F
:10D93000019B002B0DD00E23E15E280000F052FB6E
:10D94000002806D00322A38993431A00012313431E
:10D95000A381A0893843A081CBE7C04621D700002E
:10D9600010B5034B0100186800F06CF810BDC046FC
:10D970008C00002082B0002900D101A9101E06D021
:10D98000002B06D013780B601078431E984102B02C
:10D99000704702204042FAE7C9B28218904201D192
:10D9A0000020704703788B42FBD00130F6E700007F
:10D9B00070B50500002910D00C1F2368002B00DA79
:10D9C000E418280000F034FB1D4A1368002B05D131
:10D9D00063601460280000F02CFB70BDA34209D9DD
:10D9E000216860188342F3D118685B684118216090
:10D9F000EEE713005A68002A01D0A242F9D919684B
:10DA00005818A0420BD12068091858181960824292
:10DA1000E0D110685268411819605A60DAE7A042F4
:10DA200002D90C232B60D5E721686018824203D10C
:10DA3000106852684118216062605C60CAE7C046A5
:10DA40003C1C0020032370B5CD1C9D430835060007
:10DA50000C2D1ED20C25A9421DD8300000F0E8FA8A
:10DA6000254A14682100002919D1244C2368002B71
:10DA700003D1300000F0CAF920602900300000F026
:10DA8000C5F9431C2BD10C233000336000F0D1FAD0
:10DA900003E0002DDFDA0C233360002070BD0B683B
:10DAA0005B1B19D40B2B03D90B60CC18256003E04A
:10DAB0004B688C420DD11360300000F0BAFA2000A0
:10DAC00007220B30231D9043C31AE7D05A42E2507D
:10DAD000E4E763600C00EFE70C004968C3E7032349
:10DAE000C41C9C43A042E1D0211A300000F08EF902
:10DAF000431CDBD1C7E7C0463C1C0020401C002073
:10DB0000F8B507000D001600002905D11100FFF738
:10DB100099FF04002000F8BD002A03D1FFF748FF59
:10DB20003400F7E700F086FA2C00B042F2D2310060
:10DB30003800FFF787FF041EECD029003200FEF703
:10DB4000BFFF29003800FFF733FFE3E7F0B58E6829
:10DB500085B007000C00039201939E423CD89023AD
:10DB60008A89DB001A4234D00325096923685B1ACD
:10DB70000293636902985D43EB0F5D19019B6D1081
:10DB800001331B18AB4200D91D00530532D52900C3
:10DB90003800FFF757FF061E09D10C233B604023D6
:10DBA0000120A28940421343A38105B0F0BD029A2F
:10DBB0002169FEF785FFA389144A1A408023134385
:10DBC000A381029B2661F61826606561019EED1A0D
:10DBD000A560019B9E4200D9019E320003992068F6
:10DBE000FEF777FFA36800209B1BA36023689E19A4
:10DBF0002660DAE72A003800FFF782FF061EE0D130
:10DC000021693800FFF7D4FEC7E7C0467FFBFFFF5E
:10DC1000F0B59FB0029005938B890F0016001B068C
:10DC200011D50B69002B0ED14021FFF70BFF386097
:10DC30003861002805D10C23029A013813601FB007
:10DC4000F0BD40237B61002306AC63612033637623
:10DC50001033A37635002B78002B01D0252B46D12D
:10DC6000AB1B04930CD0320039000298FFF76EFF13
:10DC7000431C00D1AEE06269049B94466344636137
:10DC80002B78002B00D1A5E00122002352426260D4
:10DC900002A9543252186E1C2360E360A360137013
:10DCA000A365317805225448FFF776FE751C0028DD
:10DCB0001FD12268D30604D5532302A95B18202163
:10DCC0001970130704D5532302A95B182B2119706F
:10DCD00033782A2B16D0350000210A20E3682A78F1
:10DCE0006E1C303A092A4ED9002918D010E00135AF
:10DCF000B1E7414B2268C01A0123834013432360DC
:10DD00002E00CEE7059B191D1B680591002B01DB3A
:10DD1000099304E05B42E3600223134323602B7802
:10DD20002E2B0AD16B782A2B35D1059B02351A1D73
:10DD30001B680592002B2BDB0793304E29780322BA
:10DD40003000FFF729FE002806D04023801B8340C7
:10DD500022680135134323602978062228486E1C67
:10DD60002176FFF719FE00283CD0264B002B25D149
:10DD70000722059B07339343083305936369039A8E
:10DD80009B18636166E7434301219B183500A6E7B2
:10DD900001235B42D0E700230A201A0001356360AB
:10DDA00029786E1C3039092903D9002BC5D0079278
:10DDB000C3E74243012352183500F1E705AB009356
:10DDC0003A00114B2100029800E000BF0390039B32
:10DDD0000133D3D1BB890B985B0600D42FE7012018
:10DDE00040422CE705AB00933A00074B2100029814
:10DDF000FFF736F8EAE7C046D0FB0000D6FB00008C
:10DE0000DAFB0000000000004DDB0000002370B5CD
:10DE1000064C05000800236000F060F9431C03D1A4
:10DE20002368002B00D02B6070BDC046D02F00208F
:10DE300070B504000D001F2904D9162303600120CA
:10DE4000404270BD436C002B04D08A009B181A68B6
:10DE5000002A08D1200000F031F82A00010020003B
:10DE600000F01AF8EDE70020012AEAD0511C03D196
:10DE7000162301302360E4E7002428001C6090474B
:10DE80002000DEE710B5034B01001868FFF7D0FF54
:10DE900010BDC0468C000020002370B5064C050064
:10DEA00008001100236000F001F9431C03D123682E
:10DEB000002B00D02B6070BDD02F002010B500F0DB
:10DEC000E5F810BD70B50C000E25495F00F0BAF8FA
:10DED000002803DB636D1B18636570BDA389024ACC
:10DEE0001340A381F9E7C046FFEFFFFFF8B51F001D
:10DEF0008B8905000C001600DB0505D50E23C95ED5
:10DF00000022022300F080F8A389054A280013406C
:10DF1000A38132000E23E15E3B0000F02BF8F8BD38
:10DF2000FFEFFFFF70B50C000E25495F00F06CF8A5
:10DF3000A389421C03D1054A1340A38170BD8022EE
:10DF400052011343A3816065F8E7C046FFEFFFFF6E
:10DF500010B50E23C95E00F021F810BD0B1E04D0D1
:10DF6000FF2A04D98A2303608B3B180070470A708C
:10DF70000123FAE770B50500080011000022064CE5
:10DF800022601A0000F0B8F8431C03D12368002B6C
:10DF900000D02B6070BDC046D02F0020002370B58C
:10DFA000064C05000800236000F060F8431C03D114
:10DFB0002368002B00D02B6070BDC046D02F0020FE
:10DFC000002370B5064C050008001100236000F026
:10DFD00055F8431C03D12368002B00D02B6070BD83
:10DFE000D02F0020002370B5064C050008002360E8
:10DFF00000F054F8431C03D12368002B00D02B60A1
:10E0000070BDC046D02F002070B50500080011007B
:10E010000022064C22601A0000F050F8431C03D185
:10E020002368002B00D02B6070BDC046D02F00208D
:10E03000704770470B1F1B68181F002B01DA0B5825
:10E04000C018704770B50500080011000022064C8A
:10E0500022601A0000F03AF8431C03D12368002B19
:10E0600000D02B6070BDC046D02F00205822012068
:10E07000014B40421A607047D02F002058220120E7
:10E08000014B40421A607047D02F002058220120D7
:10E09000014B40421A607047D02F00205822024B9B
:10E0A00000201A607047C046D02F0020582201205F
:10E0B000014B40421A607047D02F002058220120A7
:10E0C000014B40421A607047D02F00205822012097
:10E0D000014B40421A607047D02F0020044A136859
:10E0E000002B00D1034B1818106018007047C04671
:10E0F000441C0020D82F002058220120014B404210
:10E100001A607047D02F0020FEE7C046F8B5C04621
:10E11000F8BC08BC9E467047F8B5C046F8BC08BCC1
:10E120009E4670476461746100000000C0E1000019
:10E13000EF010000C9E10000E50A0000CFE10000A6
:10E14000E3020000D7E10000990B0000DEE10000CF
:10E15000D50C0000E3E1000009050000E9E1000042
:10E16000F5060000F4E1000053030000F9E10000AF
:10E170002D0F000005E200001F0200000FE200006A
:10E18000110A00001DE20000950600002AE20000CE
:10E190008108000036E200005506000072616E64DE
:10E1A0006F6D00616C6C006C6173740066616C7300
:10E1B00065007472756500252E3135732E2E2E0084
:10E1C0006D616B654C6973740072616E67650061A7
:10E1D00064644C6173740064656C657465006A6F97
:10E1E000696E0073706C697400636F707946726F4A
:10E1F0006D546F0066696E64006A6F696E53747265
:10E20000696E677300756E69636F6465417400754C
:10E210006E69636F6465537472696E67006E6577CB
:10E2200042797465417272617900617342797465F3
:10E23000417272617900667265654D656D6F7279C4
:10E2400000000000B1E2000021140000B6E200006E
:10E250003F140000D7E1000043140000BCE20000BE
:10E2600025140000C6E2000047140000CFE20000C1
:10E270004B140000D9E200004F140000E2E200005D
:10E2800053140000EDE2000057140000F9E2000012
:10E290002914000002E30000371400000CE3000022
:10E2A0002D14000017E300003B14000066696C6544
:10E2B000006F70656E00636C6F736500656E644F10
:10E2C0006646696C6500726561644C696E650072D2
:10E2D00065616442797465730072656164496E7446
:10E2E0006F00617070656E644C696E65006170707E
:10E2F000656E6442797465730066696C6553697A0A
:10E30000650073746172744C697374006E6578741F
:10E31000496E4C6973740073797374656D496E66E8
:10E320006F00000048180000581800007218000024
:10E33000EE180000261900005A190000921900007A
:10E34000B8190000FC1900003E1A0000921A0000E3
:10E35000D61A0000381B0000801B0000A61B00001E
:10E36000DE1B0000241C00004A1C0000781C00007A
:10E37000A61C0000B23300006C1D00003E1E000011
:10E38000B41E0000201F00006C1F00008C1F000046
:10E39000AE1F0000062100004A210000C22100003B
:10E3A000F02100002222000070220000D82200008C
:10E3B000402300009C230000FA2300006C2400008E
:10E3C000DE2400003A25000094250000D42500003A
:10E3D0001A26000060260000A8260000FC26000087
:10E3E000502700008E270000142800004A28000053
:10E3F00092280000DA280000222900005C29000091
:10E40000AC290000F4290000562B0000781C000005
:10E41000DE1B00005C2A000048180000922A000061
:10E42000BE2A0000F42A0000202B0000481800003B
:10E43000481800004818000048180000D22B0000BF
:10E44000142C00005A2C0000AA2C0000D62C00002E
:10E450004E2D0000D62D0000042E000048180000AC
:10E4600048180000282E0000582E0000882E0000BA
:10E47000BE2E0000E82E00001E2F0000482F0000D6
:10E48000702F0000982F0000C82F0000F82F000008
:10E49000223000004C3000007C300000A63000002C
:10E4A00048180000481800004818000048180000EC
:10E4B00048180000D6300000023100002E31000064
:10E4C0005A31000098310000CE31000004320000C3
:10E4D0003A320000703200009C320000C832000066
:10E4E000FE320000481800004818000048180000DC
:10E4F000481800004818000048180000481800009C
:10E50000481800004818000048180000481800008B
:10E51000481800002A3300002A330000523400005B
:10E52000883400005B2564206974656D206C697314
:10E53000745D002825642062797465732900286F52
:10E54000626A65637420747970653A2025642900D5
:10E55000537461636B20756E646572666C6F7700CF
:10E56000626F6F6C65616E006E756D6265720073CF
:10E570007472696E67006C697374006279746520E7
:10E580006172726179000000070000000300000062
:10E590001AE60000B135000022E6000061360000F6
:10E5A0002BE60000E13A000034E60000B53500003B
:10E5B0003DE60000E53A000045E60000793800003D
:10E5C0004EE60000C93800005CE60000A9370000F4
:10E5D00067E600006D3C000072E60000F1360000C6
:10E5E0007DE60000E13B000089E6000055370000B1
:10E5F00095E600003D3C0000000000000100000026
:10E600000200000003000000040000000A000000F7
:10E610006D6963726F3A62697400686173546F6EFA
:10E620006500706C6179546F6E6500686173536545
:10E6300072766F00736574536572766F0064616300
:10E64000496E697400646163577269746500736F21
:10E650006674577269746542797465007371756187
:10E6600072655761766500736574557365724C45C4
:10E670004400616E616C6F675265616400616E6138
:10E680006C6F675772697465006469676974616C5F
:10E6900052656164006469676974616C577269747A
:10E6A0006500474320746F6F6B2025642075736588
:10E6B00063733B206672656520256420776F726402
:10E6C00073003C496E74656765723E003C4C69732B
:10E6D000743E003C4F626A6563743E003C4279744C
:10E6E0006541727261793E000D0A564D2050616E8F
:10E6F00069633A2025730D0A006D69736300000099
:10E7000045E70000CD4600004EE7000099470000B5
:10E7100056E700005D4700005AE70000B51700000B
:10E7200069E700002146000071E70000C7450000CE
:10E730007BE700005D45000087E700005F440000C4
:10E740006E756C6C00686578546F496E7400726504
:10E750007363616C650073696E0062726F616463FC
:10E76000617374546F494445006A736F6E476574F2
:10E77000006A736F6E436F756E74006A736F6E56C6
:10E78000616C75654174006A736F6E4B6579417495
:10E790000000000088E800000948000090E8000040
:10E7A0000D4800009AE800002B480000A3E8000094
:10E7B00035480000AEE800003F480000BAE800001D
:10E7C00049480000C8E8000053480000D0E80000B5
:10E7D0005D480000D6E8000067480000EBE8000054
:10E7E0007148000000E900007B4800000CE90000CF
:10E7F000854800001CE900008F48000028E900005F
:10E800009948000035E90000A34800003EE90000F7
:10E81000AD48000046E90000B748000054E9000098
:10E82000C148000065E90000CB48000078E900001D
:10E83000D548000086E90000DF48000095E90000A7
:10E84000E9480000A8E90000F3480000BEE9000024
:10E85000FD480000CAE9000007490000DAE90000AD
:10E8600011490000E9E900001B490000F7E9000038
:10E8700025490000FFE900001748000007EA0000F2
:10E88000214800006E65740068617357694669002D
:10E890007374617274576946690073746F70576955
:10E8A00046690077696669537461747573006D79A0
:10E8B0004950416464726573730073746172745378
:10E8C0005349447363616E00676574535349440050
:10E8D0006D794D414300687474705365727665724A
:10E8E0004765745265717565737400726573706FF6
:10E8F0006E64546F487474705265717565737400FA
:10E9000068747470436F6E6E6563740068747470BD
:10E910004973436F6E6E65637465640068747470E8
:10E9200052657175657374006874747052657370A4
:10E930006F6E7365007564705374617274007564F2
:10E940007053746F700075647053656E64506163CA
:10E950006B657400756470526563656976655061B6
:10E96000636B65740075647052656D6F74654950B2
:10E97000416464726573730075647052656D6F7481
:10E9800065506F727400776562536F636B65745383
:10E990007461727400776562536F636B65744C6168
:10E9A00073744576656E7400776562536F636B654B
:10E9B0007453656E64546F436C69656E74004D5199
:10E9C0005454436F6E6E656374004D5154544973D3
:10E9D000436F6E6E6563746564004D5154544469B1
:10E9E00073636F6E6E656374004D5154544C617364
:10E9F000744576656E74004D515454507562004DE7
:10EA0000515454537562004D515454556E73756290
:10EA1000001A1B1C03040607090A17181900000036
:10EA2000000008080800080A4A4000000A5FEA5F80
:10EA3000EA0ED92ED36E19324489330C924C924D82
:10EA4000080800000004880808040804848488007A
:10EA50000A448A4000048EC480000000048800003C
:10EA60000EC000000000080001224488100C9252E1
:10EA7000524C048C84848E1C824C901E1EC2449284
:10EA80004C06CA525FE21FF01EC13E02448ED12ED8
:10EA90001FE24488100ED12ED12E0ED12EC4880034
:10EAA0000800080000048004880244880482000EE4
:10EAB000C00EC008048244880ED126C0040ED13591
:10EAC000B36C0C925ED2521C925C925C0ED0101011
:10EAD0000E1C9252525C1ED01C901E1ED01C901018
:10EAE0000ED013712E12525ED2521C8808081C1FC1
:10EAF000E242524C1254981492101010101E113B06
:10EB000075B131113935B3710C9252524C1C925C73
:10EB100090100C92524C861C925C92510ED00C823A
:10EB20005C1FE4848484125252524C1131312A44C5
:10EB3000113135BB7112524C9252112A4484841EF9
:10EB4000C488101E0EC808080E10080482410EC2A8
:10EB500042424E048A400000000000001F0804806A
:10EB60000000000ED2524F10101C925C000ED0100C
:10EB70000E02424ED24E0C925C900E06C81C8808C3
:10EB80000ED24EC24C10101C925208000808080207
:10EB90004002424C10149814920808080806001B02
:10EBA00075B131001C925252000C92524C001C92D2
:10EBB0005C90000ED24EC2000ED010100006C804A9
:10EBC0009808080EC807001252524F0011312A440B
:10EBD00000113135BB00124C8C9200112A44980070
:10EBE0001EC4881E06C48C848608080808081808F5
:10EBF0000C881800000C8360000000000100000079
:10EC000002000000030000000400000005000000F6
:10EC100006000000070000000800000009000000D6
:10EC20000A0000000B0000000C0000000D000000B6
:10EC30000E0000000F000000100000001200000095
:10EC40001400000016000000180000001A00000068
:10EC50001C0000001E000000200000002300000037
:10EC600026000000290000002C0000002F000000FA
:10EC700032000000360000003A0000003E000000B4
:10EC800042000000460000004B0000005000000061
:10EC9000550000005A0000006100000068000000FC
:10ECA0006F000000760000007D000000840000007E
:10ECB0008B0000009200000099000000A0000000FE
:10ECC000A7000000AE000000B5000000BC0000007E
:10ECD000C3000000CA000000D1000000D8000000FE
:10ECE000DF000000E6000000ED000000F40000007E
:10ECF000FB000000FF00000050ED0000494900004B
:10ED00005BED00001D4F000065ED0000294B000089
:10ED100072ED00008D4C000079ED0000DD4C00002C
:10ED200082ED00002D4D00008EED0000254C00000E
:10ED30009FED0000B54B0000AFED00001D4E000040
:10ED4000BCED0000814B0000646973706C61790058
:10ED50006C696768744C6576656C006D62446973B4
:10ED6000706C6179006D62446973706C61794F6693
:10ED700066006D62506C6F74006D62556E706C6FE2
:10ED800074006D62447261775368617065006D62F2
:10ED90005368617065466F724C6574746572006D7E
:10EDA00062456E61626C65446973706C6179006E76
:10EDB000656F506978656C53656E64006E656F5061
:10EDC0006978656C53657450696E004E6F74206588
:10EDD0006E6F75676820726F6F6D206576656E2047
:10EDE000616674657220636F6D70616374696F6EC4
:10EDF00000436F6D70616374656420466C61736875
:10EE000020636F64652073746F72650A25642062E5
:10EE10007974657320757365642028256425252918
:10EE2000206F6620256400426164207265636F7202
:10EE30006420666F756E6420647572696E67206900
:10EE40006E697469616C697A6174696F6E002564BA
:10EE50002025642025642028256420776F72647340
:10EE600029002564207265636F7264732C20256409
:10EE700020776F7264732C206D617849442025647B
:10EE80002C20636F6D70616374696F6E20637963AA
:10EE90006C657320256400526573746F726564201D
:10EEA00025642073637269707473005374617274A3
:10EEB000656400726164696F0000000051EF00003A
:10EEC000355900005EEF0000315C00006EEF00007D
:10EED000B15B00007CEF0000C55D000087EF000023
:10EEE0004D59000097EF0000C9590000ABEF00003A
:10EEF000B1590000BAEF0000755F0000C6EF0000D6
:10EF0000F35E0000CFEF0000975E0000DAEF000034
:10EF1000115E0000E5EF00004D5E0000EEEF000026
:10EF2000815E0000F7EF00005D59000006F0000070
:10EF3000915900000FF000006D590000253038781D
:10EF4000006E6F6E65006F74686572007061697243
:10EF50000064697361626C65526164696F006D651C
:10EF60007373616765526563656976656400706196
:10EF7000636B657452656365697665007061636B88
:10EF8000657453656E64007265636569766564498E
:10EF90006E74656765720072656365697665644D58
:10EFA000657373616765547970650072656365693F
:10EFB000766564537472696E670073656E64496E3A
:10EFC00074656765720073656E6450616972007381
:10EFD000656E64537472696E67007365744368612B
:10EFE0006E6E656C0073657447726F757000736543
:10EFF00074506F776572007369676E616C537472D9
:10F00000656E677468006465766963654944006C81
:10F010006173744D657373616765494400556E6B28
:10F020006E6F776E207072696D6974697665205BAA
:10F0300025733A25735D00000000000096300777C5
:10F040002C610EEEBA51099919C46D078FF46A70DC
:10F0500035A563E9A395649E3288DB0EA4B8DC79FC
:10F060001EE9D5E088D9D2972B4CB609BD7CB17E7C
:10F07000072DB8E7911DBF906410B71DF220B06A4C
:10F080004871B9F3DE41BE847DD4DA1AEBE4DD6D5C
:10F0900051B5D4F4C785D38356986C13C0A86B645C
:10F0A0007AF962FDECC9658A4F5C0114D96C06637C
:10F0B000633D0FFAF50D088DC8206E3B5E10694C5C
:10F0C000E44160D5727167A2D1E4033C47D4044B9C
:10F0D000FD850DD26BB50AA5FAA8B5356C98B2427C
:10F0E000D6C9BBDB40F9BCACE36CD832755CDF45FC
:10F0F000CF0DD6DC593DD1ABAC30D9263A00DE512C
:10F100008051D7C81661D0BFB5F4B42123C4B3561B
:10F110009995BACF0FA5BDB89EB802280888055F9B
:10F12000B2D90CC624E90BB1877C6F2F114C6858FB
:10F13000AB1D61C13D2D66B69041DC760671DB01E9
:10F14000BC20D2982A10D5EF8985B1711FB5B606BB
:10F15000A5E4BF9F33D4B8E8A2C9077834F9000FFB
:10F160008EA8099618980EE1BB0D6A7F2D3D6D089B
:10F17000976C6491015C63E6F4516B6B62616C1C8B
:10F18000D83065854E0062F2ED95066C7BA5011BBB
:10F19000C1F4088257C40FF5C6D9B06550E9B7125B
:10F1A000EAB8BE8B7C88B9FCDF1DDD62492DDA151B
:10F1B000F37CD38C654CD4FB5861B24DCE51B53A3B
:10F1C0007400BCA3E230BBD441A5DF4AD795D83D3B
:10F1D0006DC4D1A4FBF4D6D36AE96943FCD96E347B
:10F1E000468867ADD0B860DA732D0444E51D03335B
:10F1F0005F4C0AAAC97C0DDD3C710550AA4102276B
:10F2000010100BBE86200CC925B56857B3856F203A
:10F2100009D466B99FE461CE0EF9DE5E98C9D9299A
:10F220002298D0B0B4A8D7C7173DB359810DB42EDA
:10F230003B5CBDB7AD6CBAC02083B8EDB6B3BF9A26
:10F240000CE2B6039AD2B1743947D5EAAF77D29DB2
:10F250001526DB048316DC73120B63E3843B649492
:10F260003E6A6D0DA85A6A7A0BCF0EE49DFF099392
:10F2700027AE000AB19E077D44930FF0D2A3088702
:10F2800068F2011EFEC206695D5762F7CB676580B2
:10F2900071366C19E7066B6E761BD4FEE02BD389B2
:10F2A0005A7ADA10CC4ADD676FDFB9F9F9EFBE8E12
:10F2B00043BEB717D58EB060E8A3D6D67E93D1A152
:10F2C000C4C2D83852F2DF4FF167BBD16757BCA632
:10F2D000DD06B53F4B36B248DA2B0DD84C1B0AAFD2
:10F2E000F64A0336607A0441C3EF60DF55DF67A852
:10F2F000EF8E6E3179BE69468CB361CB1A8366BCE2
:10F30000A0D26F2536E2685295770CCC03470BBB31
:10F31000B91602222F260555BE3BBAC5280BBDB231
:10F32000925AB42B046AB35CA7FFD7C231CFD0B5D1
:10F330008B9ED92C1DAEDE5BB0C2649B26F263ECC3
:10F340009CA36A750A936D02A906099C3F360EEBD1
:10F350008567077213570005824ABF95147AB8E291
:10F36000AE2BB17B381BB60C9B8ED2920DBED5E571
:10F37000B7EFDC7C21DFDB0BD4D2D38642E2D4F1C1
:10F38000F8B3DD686E83DA1FCD16BE815B26B9F651
:10F39000E177B06F7747B718E65A0888706A0FFFB1
:10F3A000CA3B06665C0B0111FF9E658F69AE62F871
:10F3B000D3FF6B6145CF6C1678E20AA0EED20DD771
:10F3C0005483044EC2B30339612667A7F71660D091
:10F3D0004D476949DB776E3E4A6AD1AEDC5AD6D9D1
:10F3E000660BDF40F03BD83753AEBCA9C59EBBDEF1
:10F3F0007FCFB247E9FFB5301CF2BDBD8AC2BACAA1
:10F400003093B353A6A3B4240536D0BA9306D7CD10
:10F410002957DE54BF67D9232E7A66B3B84A61C430
:10F42000021B685D942B6F2A37BE0BB4A18E0CC3F0
:10F430001BDF055A8DEF022D416C6C207461736BDC
:10F44000732073746F7070656400763137300020FC
:10F450002573202573004D656D6F727920636C658F
:10F4600061726564004E6F20667265652074617319
:10F470006B20656E7472696573000000FCF4000017
:10F480004D78000009F500009971000015F50000A5
:10F490001D7800001BF500002D78000021F500000C
:10F4A0003D78000027F50000F57600003DF50000EE
:10F4B000057A00004BF50000CD71000055F5000005
:10F4C000917A00005DF500001975000066F50000F6
:10F4D000F572000077F50000D573000083F5000099
:10F4E000A97200008CF500002973000094F500005B
:10F4F0002174000073656E736F72730061636365DE
:10F500006C65726174696F6E0074656D70657261AF
:10F51000747572650074696C74580074696C745900
:10F520000074696C745A00736574416363656C653B
:10F53000726F6D6574657252616E6765006D6167AB
:10F540006E657469634669656C6400746F756368A1
:10F5500052656164006932635265616400693263B7
:10F56000577269746500693263536574436C6F63E5
:10F570006B53706565640073706945786368616E8C
:10F5800067650073706953657475700072656164B6
:10F59000444854006D6963726F70686F6E65000057
:10F5A000B1E20000717B0000B6E200001D7B0000AC
:10F5B000D7F50000B57C0000D9E20000397B0000DF
:10F5C000DCF500003D7C0000E2F50000957B0000CA
:10F5D00073657269616C0072656164007772697449
:10F5E0006500777269746542797465730000000084
:10F5F0006CF60000E57C00007AF60000F57C000067
:10F6000087F60000E97C000090F60000F97C00001D
:10F610009AF60000FD7C0000A3F60000017D0000CA
:10F62000A8F60000057D0000ADF60000097D000091
:10F63000B9F600000D7D0000C0F60000117D00004D
:10F64000C9F60000157D0000CEF60000197D00000F
:10F65000D9F600001D7D0000E3F60000ED7C0000FF
:10F66000EDF60000F17C000074667400656E616266
:10F670006C65446973706C61790073657442616391
:10F680006B6C6967687400676574576964746800B7
:10F690006765744865696768740073657450697854
:10F6A000656C006C696E65007265637400726F75DD
:10F6B0006E6465645265637400636972636C6500AF
:10F6C000747269616E676C65007465787400746645
:10F6D00074546F756368656400746674546F756301
:10F6E000685800746674546F756368590074667462
:10F6F000546F7563685072657373757265007661D7
:10F700007273000024F70000AD8100002EF70000A6
:10F710008D81000037F700006981000043F7000089
:10F72000F7800000766172457869737473007661C2
:10F73000724E616D6564007365745661724E616DE1
:10F740006564007661724E616D65466F72496E64E4
:10F7500065780057656C636F6D6520746F204D6927
:10F7600063726F426C6F636B732100705F737069BB
:10F7700020213D204E554C4C002F686F6D652F6742
:10F7800069742F2E706C6174666F726D696F2F7063
:10F7900061636B616765732F6672616D65776F7208
:10F7A0006B2D61726475696E6F6E6F726469636EE2
:10F7B0007266352F6C69627261726965732F53507E
:10F7C000492F5350492E63707000535049436C6168
:10F7D00073733A3A535049436C617373284E5246DF
:10F7E0005F5350495F547970652A2C2075696E7497
:10F7F000385F742C2075696E74385F742C207569BD
:10F800006E74385F742900000000000000000000E2
:10F81000818300003D830000638300006D8300004E
:10F8200077830000618300000300000002000000F5
:10F8300001000000040000000500000011000000AD
:10F840000C0000000B000000120000000A00000085
:10F85000060000001A00000014000000170000005D
:10F86000160000001500000010000000FFFFFFFF61
:10F87000FFFFFFFF000000001E0000001900000055
:10F880001800000007000000080000000900000048
:10F890000D0000000E0000000F0000001C00000022
:10F8A0001B0000001D00000013000000000000000D
:10F8B000000000006D870000A18F0000ED870000B0
:10F8C00001880000F7870000698700005D8700005D
:10F8D0000D880000898700005987000000000000A3
:10F8E000000000000000304300000000000030C3B2
:10F8F0007371727400000000FB21F93FFB21094085
:10F900007CD91240FB2119407A6A1F407CD92240E1
:10F91000BBFD2540FB2129403A462C407A6A2F4006
:10F920005C4731407CD932409C6B3440BBFD354054
:10F93000DB8F3740FB2139401BB43A403A463C400C
:10F940005AD83D407A6A3F404C7E40405C47414037
:10F950006C1042407CD942408CA243409C6B444096
:10F96000AC344540BBFD4540CBC64640DB8F4740ED
:10F97000EB584840FB21494083F9A200444E6E00F9
:10F98000FC291500D1572700DD34F50062DBC000EB
:10F990003C999500419043006351FE00BBDEAB00F3
:10F9A000B761C5003A6E2400D24D42004906E0001E
:10F9B00009EA2E001C92D100EB1DFE0029B11C00AB
:10F9C000E83EA700F535820044BB2E009CE9840088
:10F9D000B4267000417E5F00D69139005383390010
:10F9E0009CF439008B5F840028F9BD00F81F3B00B0
:10F9F000DEFF97000F980500112FEF000A5A8B00C9
:10FA00006D1F6D00CF7E360009CB2700464FB70033
:10FA10009E663F002DEA5F00BA277500E5EBC70040
:10FA20003D7BF100F739070092528A00FB6BEA0038
:10FA30001FB15F00085D8D00300356007BFC46005F
:10FA4000F0AB6B0020BCCF0036F49A00E3A91D0098
:10FA50005E619100081BE60085996500A0145F00B7
:10FA60008D40680080D8FF0027734D0006063100E6
:10FA7000CA561500C9A873007BE260006B8CC000F9
:10FA800000000040FB21F93F000000002D44743EBF
:10FA9000000000809846F83C0000006051CC783BA4
:10FAA00000000080831BF0390000004020257A38D8
:10FAB000000000802282E336000000001DF369355B
:10FAC0000200000003000000040000000600000027
:10FAD0002CAC0000D6AB0000D6AB000004AD00009B
:10FAE000D2AB0000D2AB0000FAAC000004AD0000C5
:10FAF000D2AB0000FAAC0000D2AB000004AD0000B5
:10FB000008AD000008AD000008AD000010AD000019
:10FB100008B700007AB50000BEB5000022B50000AD
:10FB2000BEB50000AEB60000BEB5000022B50000B4
:10FB30007AB500007AB50000AEB6000022B500002C
:10FB40001AB500001AB500001AB50000BCB60000D6
:10FB500030BE000032BD000032BD000050C00000C9
:10FB60002CBD00002CBD000038C0000050C00000BB
:10FB70002CBD000038C000002CBD000050C00000AB
:10FB800046C0000046C0000046C0000054C000004F
:10FB90002C2066756E6374696F6E3A200061737312
:10FBA000657274696F6E2022257322206661696C0C
:10FBB00065643A2066696C6520222573222C206CCE
:10FBC000696E65202564257325730A009000002066
:10FBD000232D302B2000686C4C0065666745464736
:10FBE00000303132333435363738394142434445B9
:10FBF0004600303132333435363738396162636428
:10FC00006566000000000000000000000000000029
:10FC100000000000000000000000000000000000E4
:10FC200000000000000000000000000000000000D4
:10FC300000000000000000000000000000000000C4
:10FC400000000000000000000000000000000000B4
:10FC500000000000000000000000000000000000A4
:10FC600000000000504F5349580000202020202061
:10FC7000202020202828282828202020202020205C
:10FC8000202020202020202020202088101010104C
:10FC900010101010101010101010100404040404A0
:10FCA00004040404041010101010101041414141CC
:10FCB00041410101010101010101010101010101B4
:10FCC00001010101010110101010101042424242C6
:10FCD0004242020202020202020202020202020284
:10FCE00002020202020210101010200000000000A8
:10FCF0000000000000000000000000000000000004
:10FD000000000000000000000000000000000000F3
:10FD100000000000000000000000000000000000E3
:10FD200000000000000000000000000000000000D3
:10FD300000000000000000000000000000000000C3
:10FD400000000000000000000000000000000000B3
:10FD500000000000000000000000000000000000A3
:10FD60000000000000000000000000000000000093
:08FD70009803FF7F0100000071
:10FD7800FFFFFFFFE803000001000000E803DC05C7
:10FD8800DC05DC05DC050000FFFFFFFFFFFFFFFFD0
:10FD98001800000019FCFFFFFFFFFFFF0200000032
:10FDA80040420F00FFFF01FF0024F40002000000A2
:10FDB80003000000FFFFFFFF00000000010000003B
:10FDC8000000020001000000FFFFFFFF000000002C
:10FDD800020000000000040002000000FFFFFFFF17
:10FDE80000000000030000000000080003000000FD
:10FDF8000A00000008000000010000009000002038
:10FE08000000000024FC000044FC000004FC00008A
:10FE180000000000000000000000000000000000DA
:10FE280000000000000000000000000000000000CA
:10FE380000000000000000000000000000000000BA
:10FE480000000000000000000000000000000000AA
:10FE5800000000000000000000000000000000009A
:10FE68004300000000000000000000000000000047
:10FE7800000000000000000000000000000000007A
:10FE88004300000000000000000000000000000027
:10FE9800000000000000000000000000000000005A
:10FEA8004300000000000000000000000000000007
:10FEB800000000000000000000000000000000003A
:10FEC80043000000000000000000000000000000E7
:10FED800000000000000000000000000000000001A
:10FEE80043000000000000000000000000000000C7
:10FEF80000000000000000000000000000000000FA
:10FF080043000000000000000000000000000000A6
:10FF180000000000000000000000000000000000D9
:10FF28004300000000000000000000000000000086
:10FF380000000000000000000000000000000000B9
:10FF48005DDF000075D90000000000006AFC0000B9
:10FF5800BEE10000F8E60000F8E60000F8E6000060
:10FF6800F8E60000F8E60000F8E60000F8E6000011
:10FF7800F8E60000F8E60000FFFFFFFFFFFFFFFFC5
:10FF8800FFFFFFFFFFFF0000010041534349490005
:10FF98000000000000000000000000000000000059
:10FFA80000000000000000000000415343494900E0
:10FFB8000000000000000000000000000000000039
:10FFC800000000000000000000000000E900000040
:10FFD8000D83000061860000B98A0000C10000009E
:04000003000086FD76
:00000001FF
